:100000000040002021720000617200006372000055
:1000100000000000000000000000000000000000E0
:1000200000000000000000000000000065720000F9
:10003000000000000000000067720000697200000C
:100040006B720000315300009D7600006B7200005F
:100050006B720000000000006B7200006B72000009
:100060006B720000757A0000313200006B72000084
:100070006B7200006B7200006B7200006B7200000C
:100080006B720000217700006B7200006B72000041
:100090006B7200006B7200006B7200006B720000EC
:1000A0006B7200006B720000000000000000000096
:1000B0000000000000000000000000000000000040
:1000C00010B5064C2378002B07D1054B002B02D02E
:1000D000044800E000BF0123237010BD6802002027
:1000E0000000000010E60000044B10B5002B03D008
:1000F0000349044800E000BF10BDC04600000000F6
:100100006C02002010E60000164B002B00D1144BAF
:100110009D46402292029A1A924600218B460F4633
:100120001348144A121A0BF0F1FA0F4B002B00D0AF
:1001300098470E4B002B00D0984700200021040068
:100140000D000D48002802D00C4800E000BF0BF065
:100150009DFA2000290007F0F3FA0BF071FAC0466F
:100160000000080000400020000000000000000027
:1001700068020020C82F00200000000000000000DE
:1001800002000120104011D1042A0ED91368180969
:1001900080B2002809D001388000031D11180979A8
:1001A000002902D001309842F8D170470020FCE7C6
:1001B0000378002B03D05AB2002A01DB01307047CC
:1001C0003F229343C03B59424B41C01803789343AD
:1001D000802BF4D10130F9E710B500240378002B0F
:1001E00001D1200010BDFFF7E3FF0134F6E770B541
:1001F000002204000D00411C092003F043FB0028ED
:1002000006D001236200134343600023A34200DBB6
:1002100070BD9A00A958821891600133F6E770B555
:10022000012803DC1C2001F073F870BD01230D6868
:1002300011201D42F7D04868184206D1042804D97D
:100240000F2302681340042B01D00E20EBE703F0CC
:1002500077F96D100400002D03DDFFF7BDFFA84204
:1002600006DA1220DFE72000FFF7A2FF0400013DBD
:10027000012DF8D120787F2809DDDF280BDCF82359
:100280003F22DB00800118406378134018430123AC
:1002900040001843C9E7EF280BDCFC226378120109
:1002A0009B0113403F220007000C0343A07810403D
:1002B000ECE7F72812DCFC22637892021B03134060
:1002C000E0228004520310403F221843E378134099
:1002D000FC220343A07812018001E8E7012040429C
:1002E000D5E7F8B54D680F00EB0706D4042D04D907
:1002F0000F232E683340092B03D00B2001F008F8A0
:10030000F8BD6B683609B6B25C10731EA3420FD8F5
:100310000321200009F0B6F86421642803DC010001
:10032000032800DA03212800891903F0DDFA05000B
:100330002B6800201B099BB2013B9C42E0D23A682B
:10034000A31C9B005A510123013464001C436C60C0
:10035000D6E7F0B585B0012803DC1C2000F0D8FFFB
:1003600012E001274B683A000093022806D08B6800
:100370003B4203D05F10002F00DC17000125009BDB
:100380002B4203D00120404205B0F0BD009B042B5E
:10039000F8D91B680C680F261900314004292AD1AE
:1003A0002C4205D1042C03D923681E40042E01D011
:1003B0000E20D3E70098FFF7E3FEB842E2DB009897
:1003C00003F0BEF80600200003F0BAF80100781E22
:1003D00030180BF051FD041ED4D03378002B01D01F
:1003E000A64202D36800012521E03000FFF7E0FEBD
:1003F00001350600F1E709293ED1009B5B685B10DF
:1004000001939F42BEDC2C422ED1042C2CD92368B0
:100410003340042B28D1200003F092F80396029079
:100420007E1C009AB300D058844202D17800284341
:10043000AAE728420ED104280CD90368039A134076
:10044000042B07D103F07CF8010002980BF0DEFCCE
:100450000028EBD0019B37009E42E1DD92E71F00B0
:10046000019B9F4200DD8DE77B1C00999A008A5812
:10047000A242F4D17800B6E7032900D082E71A0936
:1004800092B25B0F92000B40D31A01939F4200DDA2
:1004900078E72C4229D1042C27D922681640032E54
:1004A00019D1100980B2520F80003240251D801AE8
:1004B000019B2E181B1A0193009B781E0433019A8E
:1004C000904200DD5EE72A001918B2420FD316D120
:1004D0000130400087E7042E07D1200003F030F8F8
:1004E00005002000FFF74CFEE2E70F2036E70C780E
:1004F000A4461478A44502D101310132E5E7013068
:10050000DDE710B503F000F843000120184310BDEB
:10051000C30711D404280FD90F2302681340032BFB
:100520000AD119400133591AC0234907DB05194084
:10053000024B1A40114301607047C046FFFFFF9F06
:10054000F7B507000E001C20012F06DD4C680123C3
:1005500022001A40009203D10D2000F0D9FE53E092
:10056000022F02D08A681A42F6D0012335681D4254
:1005700000D0A9E0042D00D8A6E01C41002C00DC2E
:100580001C000F2029680840092828D16B685B10DF
:100590000093022F05D0B368009A5B109A4200DDE9
:1005A0000093009B01221D1B0135EB43DB171D400F
:1005B000691C092003F066F9071E09D001236D00AC
:1005C0001D4303003268083345600099A14201DAF7
:1005D0003800FEBD0134A100515802C3F5E70428DC
:1005E00045D1280002F0ACFFFFF7F6FD0190022F85
:1005F00004D0B3685B10984200DD0193019BA342D5
:1006000004DA002003F0B0F90700E1E7280002F067
:1006100097FF0700009BA34221DB2800009702F010
:100620008FFF05003800FFF7C3FD019B0134070071
:10063000A342F7DA009BC41A200003F095F9071EC5
:10064000C6D002F07DFF0190306802F079FF2200F1
:10065000009B591B411801980BF03CF8B8E7380093
:10066000FFF7A6FD009B070001330093D2E70328A4
:100670002AD10B099BB2490F9B000140591A022F46
:1006800004D0B2685210914200DD1100A14205DA97
:1006900000220320110003F0F5F8B5E703200E1B3C
:1006A000331DD9170140C9188910002203F0EAF858
:1006B000071E00D18CE7013631000334FFF728FF15
:1006C000381D29193200C7E7212046E7F8B5002870
:1006D00005DC1C2000F01CFE05002800F8BD0126EA
:1006E0000C6826400FD06410E343DB171C40E11C6C
:1006F00089100022032003F0C5F8051EEDD021006B
:10070000FFF706FFE9E7042C01D80025E5E70F23F2
:1007100022681340042B1BD12000FFF731FDC31CBE
:1007200007000320D9170140C9188910320003F0CF
:10073000A9F8051ED1D03900FFF7EAFE200002F02B
:10074000FFFE2B1D01003A0018000AF0C3FFC4E7AA
:10075000092BDAD10320636832005F10FB1CD91724
:100760000140C918891003F08DF8051ECDD039005D
:10077000FFF7CEFEFF20BE42AFDA0122B300E3183E
:100780009B68134208D01341FF2B00DD0300D943BF
:10079000C917AA190B4013710136ECE710B57F2970
:1007A00002DC0170013010BD1A4B99420CDC402371
:1007B0008A115B42134303703F230B40802149425F
:1007C000194341700230EEE7134B994210DC2023AD
:1007D0000A135B4213433F24802203708B11524261
:1007E0002340214013430A43437082700330DAE709
:1007F0000A4B9942D7DCF0230370603B4370113BF6
:100800008A11FF3B1A4382703F2211401943C17085
:100810000430C8E7FF070000FFFF0000FF0F0100E2
:10082000F0B50D0085B0002803DC1C2000F070FD41
:100830000DE009680122080010400AD002AC114105
:100840002000FFF7ABFF011B200003F099F8040024
:100850001AE004293FD90F230C682340092B3AD111
:100860004B685B10019303239C46019B9A420EDD6B
:1008700003F07AF8041E07D02E68012502F060FE0E
:100880002F00019B9D421DDD200005B0F0BD01320F
:100890009300CC580123234001D10D20C6E76410FA
:1008A0007F2C0DDD0D4E0223B44209DD0C4E634654
:1008B000B44205DD00270B4EE30FA6427B419B00AF
:1008C000C018D2E70135AB00F1583942E5D04910E4
:1008D000FFF764FFD5E72120A8E7C046FF07000027
:1008E000FFFF0000FF0F010010B5040001200840C9
:1008F00010D104290DD90F230A681340042B08D105
:10090000080002F01DFE010020000BF07FFA4342B8
:10091000584110BD0020FCE7F7B50F00012803DCAB
:100920001C2000F0F5FCFEBD01264D682E4006D1CE
:10093000042D04D90F222B681A40092A01D00B205C
:10094000EFE76A681B099BB25410A34200D85C1EF3
:1009500039681E48FFF7C8FF01230190002813D112
:1009600039681B48FFF7C0FF002811D0002C0DD0BC
:100970000123621C013C9C409200535123436B6055
:1009800004E00136B200AB50B442FADA0020CAE704
:100990003B680D20DA07C4D55B10002B11DD9C42AB
:1009A0000FDB9B00A200291DEB1889180433994224
:1009B00009D10123013C9C40AA181C4353606C6080
:1009C000E4E71220ADE758681860EFE79FCD00001C
:1009D000A3CD0000002310B50C000B70C30705D594
:1009E0000D49421020000BF0D5F908E00B49002812
:1009F00002D0042804D10A4920000BF0EBF910BD05
:100A00000428FCD90F2302681340042BF7D102F00D
:100A100097FD04490200E5E79CD70000A8CD00003F
:100A2000AECD0000B3CD0000F0B593B0060002914A
:100A30001C20012E1DDD029B01251B681C002C4083
:100A400000D0ADE0042B00D8E6E01A680F231A406E
:100A5000092A4AD10394039A029992008A581700EE
:100A60002F4005D1042A03D910681840092806D060
:100A7000222000F04DFC0190019813B0F0BD5268A7
:100A80005210A418039A013203929642E3D1611CDA
:100A9000012202F0F7FE0190002802D10023019309
:100AA000EAE7019B6400190025435D600831029A62
:100AB000BB00D05802684368120992B25B109A4298
:100AC00000D8531E0022934209DCDA43D2171340A8
:100AD0009B00C918039B01379F42E8DBCCE79400D9
:100AE0000519AD6801320D51EDE72700032A59D1F0
:100AF0000193029ABB00D3582B42B9D1042BB7D92A
:100B0000186801990140032939D1020992B2430FB3
:100B100092000B40D31A1C190137BE42E9D10320C1
:100B2000E31CD9170140C9188910002202F0AAFE5F
:100B300001900028B2D000252100FFF7E9FC019BBD
:100B40001E1D029AAB00D45801231C421FD1042C55
:100B50001DD90F2123681940032918D1180980B223
:100B60005B0F80000B40C01A0023834213DBC3439A
:100B7000DB17184001353618BD42E2DB7CE704295B
:100B800000D075E71800FFF7FBFA2418C4E720002F
:100B9000FFF7F6FAE8E7E2181279F2540133E4E7D6
:100BA00000273C000F25029ABB00D35801221342B4
:100BB00034D1042B32D9186801002940042935D1D9
:100BC0001800FFF7DDFA24180137BE42EBD12000F0
:100BD00002F0CAFE0190002800D15FE7029FB60034
:100BE000BB19041D029301233D681D4229D1042D28
:100BF00027D90F262B681E40042E37D12800FFF777
:100C0000BFFA0600280002F09BFC01002000320021
:100C10000AF060FDA41922E02700C3E7180005A927
:100C2000FFF7D8FE05A80BF0FBF8CCE7032900D0AE
:100C30001EE7020992B2430F92000B40D31A1C190F
:100C4000C2E705A92800FFF7C5FE05A80BF0E8F8E4
:100C500005A90500020020000AF03CFD6419029B72
:100C60000437BB42BFD10023237005E7032EF6D122
:100C70001A0992B25B0F92001E40961B291DC5E710
:100C8000F0B50D0097B0002806DC1C2000F040FBFA
:100C90000700380017B0F0BD0C68012123000B409D
:100CA000009306D1042C04D922680F331A40092A74
:100CB00001D00B20EAE7626852100392002A03DC9D
:100CC000009802F051FEE3E7504A019201280BD050
:100CD0006868084208D1042806D902681340042B2A
:100CE00002D102F02DFC019001980BF099F806005A
:100CF0000F27039B0834013B05935E43039B02903F
:100D00009B00E318049301232068184273D1042840
:100D100071D901680B003B409C46042B03D1FFF7BF
:100D20002FFA861909E0032B6CD162460B099BB29E
:100D3000490F9B0011405A1A9619049B0434A34290
:100D4000E1D1300002F010FE071EA2D02B680793FD
:100D5000029B002B03D0686802F0F2FB0190380080
:100D600002F0EEFB0400009B079A9B00D3189E68DC
:100D7000300002F0E5FB0123334005000693002B11
:100D800001D1042E04D809A93000FFF723FE09ADD4
:100D900028000BF045F8069B0490002B0ED1042E82
:100DA0000CD90F2133681940032907D11A0992B2CF
:100DB0005B0F92000B40D31A351D04932000049A58
:100DC00029000AF087FC049BE418029B002B0AD040
:100DD000059B009A934206DD2000029A01990AF0D1
:100DE00079FC029BE418009B01330093009A039B5B
:100DF0009342B8D14DE709A9FFF7ECFD09A80BF024
:100E00000FF88EE702F09CFBF9E7C04640D20000E5
:100E100010B50024A04207DD0B6801341C4003D04C
:100E20005C10E343DB171C40611C0122092002F027
:100E300029FD002803D0012364001C43446010BD39
:100E40000A6870B510000125284034D1042A32D92F
:100E50000F24136849681C40092C17D154681B09DA
:100E60009BB22C41A34200D85C1E844205DC0220C8
:100E70000133984206DB00200FE085005519A96078
:100E80000130F2E7840011510130F2E7032C12D156
:100E9000294203D1132000F03BFA70BD4910FF290D
:100EA000F8D81B099BB204329B00D3189342E2D9B5
:100EB00011700132FAE70B2000F02AFADBE700009C
:100EC0000123F7B500254E680F0033400093AB4275
:100ED0000ED11D00042E0BD90F2233681A40092AA7
:100EE00010D172681B099BB25510AB4200D85D1E31
:100EF0003968CB0717D54C10002C01DDA5421DDA4F
:100F0000122032E0042A04D13000FFF739F905003D
:100F1000EEE7009D032AEBD11D09ADB25B0FAD00DA
:100F20001340ED1AE4E72E48FFF7DEFC002814D04A
:100F30000AF0CCFE290008F08BFB4C1C009B002B18
:100F40004CD1042E4AD932680F331340092B10D1EB
:100F50000134A400A4592000FEBD39682148FFF7E0
:100F6000C3FC2C000028E9D1113000F0D1F90400B5
:100F7000F1E7042B2AD1300002F0E2FA0500FFF776
:100F80002BF9A042BCDB012C1ADC300002F0D8FAAD
:100F900000902800FFF70CF9461B300002F0E4FC3B
:100FA000041ED8D002F0CCFA0190786802F0C8FA9A
:100FB000009B3200E91A411801980AF08BFBCAE73E
:100FC0002800FFF7F5F8013C0500DCE7032B05D10D
:100FD0003419E478023B64001C43BCE70B20C4E7EF
:100FE00098CD0000A3CD0000F7B54D680F002A0092
:100FF00001210A402FD1042D2DD90F242B68BE6862
:101000001C40092C14D169681B099BB24C10019239
:10101000A34200D85C1E39682A48FFF765FC002807
:101020002DD00F232A681340092B1DD1012317E06F
:10103000032C10D10E4203D1132000F069F9FEBD3C
:1010400072100192FF2AF7D81A0992B25B0F920030
:101050001C40141BDFE70B20EFE701339A00AE5072
:101060009C42FADA0020EAE7032BFBD12B00013384
:101070005A1BA242F6DC6A461279DA70F7E7396841
:10108000CB0706D54910002901DD8C4209DA122070
:10109000D3E70D48FFF728FC2100002801D11130CB
:1010A000CBE70F232A681340092B03D101318900B4
:1010B0004E51D7E7032BD5D16B461B796D18EB70DA
:1010C000D0E7C0469FCD0000A3CD000010B501249D
:1010D000086820421AD1042818D90F21026811404B
:1010E000092901D1406810BD032908D113099BB219
:1010F000500F9B000840181A40002043F3E70429D2
:1011000004D102F01DFAFFF767F8F5E70B2000F0B5
:10111000FFF8E8E710B5034A0B21034804F0CAF9C9
:1011200010BDC04640CD000038CD00000020704703
:10113000042070470120704710B5002002F014FC15
:1011400010BD00207047002070470020704700202D
:101150007047002070470020704700207047002033
:101160007047000010B5034A0C21034804F0A2F9AF
:1011700010BDC04628CE000088CE00007047000099
:1011800010B50124044002D04410200010BD0428F2
:1011900010D90F2302681340042B07D102F0D0F9B5
:1011A00021000A220AF004FF0400EEE7032B01D11C
:1011B0000430F5E70D22014B1A70E6E7A802002083
:1011C000012210B5024018D1042802D903681A0977
:1011D00092B201230B4012D1042902D90B681B09DA
:1011E0009BB20024934206D104309B000431C31803
:1011F000984206D30124200010BD0022E9E7002315
:10120000EFE704780A78002C01D1002AF2D00130EF
:1012100001319442ECD00024EDE70000F7B507005F
:10122000009101933049314B002A02D002220A700A
:10123000013A00261A601B68CE54BE4200DBF7BD9F
:10124000009AB300D058294B274D1C68C8239B0037
:1012500065191C1B0123184206D0254A43102100A2
:1012600028000AF065FD09E0224A002802D004287F
:101270001BD1214A210028000AF05AFD1A4C2000F7
:101280000AF0CEFD194A019B1060002B0BD07B1E8B
:10129000B34208DD194B984205D8431C1360202245
:1012A00022540022E2540136C7E7042819D90F233B
:1012B00001680B40042B04D102F042F9104A0300EC
:1012C000CDE7092B03D143680E4A5B10C7E7032B18
:1012D00008D10A0992B2490F92000B40D31A0A4A68
:1012E000BDE70123094ABAE7A9020020CC05002086
:1012F0009CD70000A8CD0000AECD00001F03000069
:10130000C7DD0000F8D0000007D1000012D10000B6
:10131000014B187000207047A802002070B501F042
:101320006FFE094C0100251D1F2228000AF090FDC8
:1013300028000AF075FD04230430800800011843DA
:101340002060200070BDC04684020020C368F0B554
:101350009D00836889B05D19030018330693036903
:10136000069A9F00069B0290DF19436901939B0038
:10137000D3180393CD4B1B78002B26D17F222B68EB
:10138000CB491C1213409B005B58043501929F46C9
:10139000029B587804F0C8FC0023029A137027E0DF
:1013A000C24B1B78002B10D12B68019A1C121340E2
:1013B000BF4A9B009B580435E9E7069B3A1DD11AAA
:1013C000BA4BD82928DD1A221A70029BB74C9B68A9
:1013D00021780193EA1A029B92109B7812021A4319
:1013E000029B587804F0A8FC0023029A2370137023
:1013F000029B069A9B680193ED1A029BAD10DD607B
:10140000069BFE1A029BB6101E61039B9B1A029A52
:101410009B10536109B0F0BD1B783C60002B01D0DC
:101420001700D2E72B6801991C120B40A0499B00C2
:101430005B5817000435AAE7069B3A1DD11A9B4B4F
:10144000D82902DD1A221A70BFE728681B78291DE7
:101450003860002B02D017000D00B6E76B680199C9
:101460001C120B4092499B005B58170008358EE711
:10147000069B3A1DD11A8D4BD82902DD1A221A700B
:10148000A3E7A4001B782C193C60002B01D01700A7
:101490009BE72B6801991C120B4085499B005B5808
:1014A0001700043573E7069B3A1DD11A7F4BD829E4
:1014B00002DD1A221A7088E77E49A40061581B7861
:1014C0003960002B01D017007FE72B6801991C12AF
:1014D0000B4077499B005B581700043557E7043FE2
:1014E000744B3A68A400E250704B1B78002B00D07C
:1014F0006BE72B68019A1C1213406D4A9B009B58A6
:10150000043544E76B4BA400E058FFF739FE043F75
:1015100006003868FFF734FE36180120654B760068
:101520000643E650614B1B78002B00D04DE72B683B
:10153000019A1C1213405E4A9B009B58043526E713
:10154000069B3A1DD11A594BD82902DD1A221A706E
:101550003BE70698039C0121A04202D221000C39EE
:1015600009681B783960002B01D017002DE72B6824
:1015700001991C120B404E499B005B581700043523
:1015800005E7069B3A1DD11A484BD82902DD1A22DD
:101590001A701AE70699039881420FD203000C3B98
:1015A0001B6845495B106418E41AA40023583B608B
:1015B0003E4B1B78002B05D0170006E71821197049
:1015C0000023F4E72B6801991C120B4038499B005B
:1015D0005B5817000435DAE6069B039A934219D24A
:1015E00013000C3B1B68344A043FA4185B10E31A39
:1015F000039A39689B0099502C4B1B78002B00D024
:10160000E3E62B68019A1C121340294A9B009B5861
:101610000435BCE61822254B1A70EDE7069B039AA9
:1016200093422DD2244B3E1FE31814000C3C04932C
:101630002368049A5B10D31A039A9B009858FFF70B
:101640009FFD07903068FFF79BFD2468049B6410A2
:101650001C1B079BA4001F1801207F00039B07434E
:10166000E7503700114B1B78002B00D0ADE62B68FC
:10167000019A1C1213400E4A9B009B58043586E6C3
:1016800018220A4B1A70EDE7069B3A1DD11A074B38
:10169000D82902DD1A221A7097E60399A40061582E
:1016A0001B783960002B09D017008EE6A8020020B5
:1016B000F8CE0000942D0020FDFFFF3F2B6801991C
:1016C0001C120B40CF499B005B58170004355EE6A7
:1016D000043F039B3A68A400E250CB4B1B78002BDD
:1016E00000D072E62B68019A1C121340C54A9B0079
:1016F0009B5804354BE6039BA4001C192368043F48
:1017000038685E10FFF73CFD36180120BE4B7600AE
:101710001B7806432660002B00D056E62B68019A02
:101720001C121340B74A9B009B5804352FE6069BBA
:10173000A4003F1BB44CBB420CD82378002B00D034
:1017400043E62B68019A1C121340AE4A9B009B583B
:1017500004351CE6AD4801F0E3FE2378002B00D0F1
:1017600033E62B68019A1C121340A64A9B009B5833
:1017700004350CE6A300ED18002C00DA38E6A24B85
:101780001B78002B00D020E62B68019A1C12134016
:101790009C4A9B009B580435F9E5043F3B68042BA9
:1017A00004D1A300ED18002C00DA21E6964B1B783B
:1017B000002B00D009E62B68019A1C121340914AB5
:1017C0009B009B580435E2E5043F3B68042B04D0A2
:1017D000A300ED18002C00DA0AE68B4B1B78002BD7
:1017E00000D0F2E52B68019A1C121340854A9B0039
:1017F0009B580435CBE53E1F3068C3070AD540101F
:101800000138002809DB01234000A40018432D19EA
:101810003060EDE5FFF7B4FCF2E77B4B37001B7857
:10182000002B00D0D1E52B68019A1C121340754A99
:101830009B009B580435AAE53A00069B0C32D31A4C
:10184000D82B03DD1A22704B1A70BEE5FF2361000E
:101850005B001940FE3BFF3B194339600299069833
:101860008968241204916D1A0299AD1089782D02AD
:101870000D4303999D40091A891099401D430B435C
:10188000BB60029B7D609C70E4B2614BE4000392FC
:10189000E358029A93605C4A1278002A03D0083316
:1018A0001D00039F91E51D00019A9B680C351C12D9
:1018B0001340544A9B009B58039F68E53B1F1C68DC
:1018C000039A069B934232D10A20E30711D4042CD9
:1018D00018D90F2322681340042B16D1200001F0E1
:1018E0002FFE0AF09DFAC8239B00984200D91800E9
:1018F0000630643003F018FE00280FD1043D069B2B
:10190000039375E50720042CF3D02000431E984173
:10191000FA234042FF3318400730EAE7029B2100D8
:10192000587804F01BFA0023029A1370E7E7039B30
:10193000039A0C3B1B6802995B109B00D31A0C3B6B
:101940001C601F1D1300083B1B685A108A70D2B21E
:101950002F49D2005B0055589B0A029A9B00956064
:10196000ED18039B069A043B1B685B109B00D31881
:101970000393254B1B78002B00D026E52B68019A9A
:101980001C1213401F4A9B009B580435FFE43B1F69
:101990001868FFF7F5FBA40006003F1B1E2827DC94
:1019A00000280DDC184B1B78002B00D00DE52B68B0
:1019B000019A1C121340134A9B009B580435E6E41D
:1019C00001F00CFB033E361801F008FB114B801BA5
:1019D0009842F9D80C4B1B78002B00D0F5E42B680B
:1019E000019A1C121340074A9B009B580435CEE411
:1019F0000123029A137001F0F1FA029B0A3886194A
:101A00005E60F5E4F8CE0000A802002024D10000BA
:101A10009C2500203F420F003B1F1868FFF7B0FBDA
:101A2000A40006003F1B00280DDCCF4B1B78002BC9
:101A300000D0CAE42B68019A1C121340CB4A9B00C9
:101A40009B580435A3E4CA4B984203DD1D22C64BC4
:101A50001A70BAE40123029A137001F0BFFAFA2354
:101A60009B005E43029B0A3E30185860C0E4A3000E
:101A7000FF1A002320001A003900FFF7CFFBBD4EEC
:101A8000BD4C3168200001F07BFFBC4B3168186011
:101A9000200004F005F83168200004F066F9B24B2C
:101AA0001B78002B00D090E42B68019A1C12134085
:101AB000AE4A9B009B58043569E4AB4BA4001B78ED
:101AC0003F1B002B00D080E42B68019A1C121340AE
:101AD000A64A9B009B58043559E4029803F088FD00
:101AE000A14B1B78002B00D06FE42B68019A1C12CD
:101AF00013409E4A9B009B58043548E43B1F1B68DB
:101B0000002B3ED13B000C3B1B68DA072CD539007B
:101B100001225B105800083902430A60002B44DDA3
:101B2000012259001143381F016039000839096842
:101B30001141CB1A39000C390968114224D09B1885
:101B40009340A4001343039AA350874B1B78002BA8
:101B500000D03AE42B68019A1C121340834A9B0080
:101B60009B580435FFF713FC042B06D90F211A6884
:101B70000A40092A01D15B68C9E719227A4B1A7019
:101B800023E45B10013BC9E7042909D90F200A6847
:101B90000240092A04D102339B005B58A400D2E71B
:101BA0001922714B1A70FFF710FC0435CDE7A30022
:101BB000069AFB189B1AD82B13DC0122631E002CFB
:101BC00014DC694B1B78002B01D0FFF7FEFB2B6860
:101BD000019A1C121340654A9B009B580435FFF77D
:101BE000D6FB1A22604B1A70FFF7EFFB3A601C001D
:101BF0000437E3E7069A3B1D9B1A5B4ED82B03DDA7
:101C00001A233370FFF7E1FB069B039AA40093426B
:101C10002AD23B1F1868FFF7B3FA011E21DD039B90
:101C20000C3B1A68521082421BDB9007801A544BFF
:101C30004018C018039B8000C2583B1B1A604A4BD7
:101C40003F1B1B780437002B01D0FFF7BEFB2B682E
:101C5000019A1C121340454A9B009B580435FFF71C
:101C600096FB20233370EAE71823FBE7434BA400DD
:101C70001A683B1B1F001A603B4B04371B78002B74
:101C800001D0FFF7A2FB2B68019A1C121340374AC0
:101C90009B009B580435FFF77AFB3B1F1A68042A08
:101CA00011D1A4002D19304B1B78002B01D0FFF768
:101CB0008CFB2B68019A1C1213402C4A9B009B58EA
:101CC0000435FFF764FB1F00EDE73A1F1368042B90
:101CD00004D0002313603A00A4002D19224B1B7876
:101CE000002B02D01700FFF770FB2B6801991C1224
:101CF0000B401E499B005B5817000435FFF747FB5C
:101D0000A3009C46FE1A002C17DC1C22164B1A70EE
:101D1000002333606346FF1A134B04371B78002BF4
:101D200001D0FFF752FB2B68019A1C1213400F4A97
:101D30009B009B580435FFF72AFB002033685A109C
:101D40008300F15801230B4003D10D21064A117085
:101D5000DFE749108A4200DD0A0001308442EFDCEF
:101D6000012352001343D4E7A8020020F8CE00005C
:101D700080EE3600CC050020A902002008000020DB
:101D8000FCFFFF3FA3009C46FE1A002C17DC1C2220
:101D9000DB4B1A70002333606346FF1AD84B0437BD
:101DA0001B78002B01D0FFF710FB2B68019A1C1247
:101DB0001340D44A9B009B580435FFF7E8FA0020F3
:101DC00033685A108300F15801230B4003D10D21D1
:101DD000CB4A1170DFE749108A4200DA0A0001306D
:101DE0008442EFDC012352001343D4E73B00083B5D
:101DF0001868FFF7C5F93B1F06001868FFF7C0F920
:101E00000023864200DA0433A4003A1B1700136053
:101E1000BB4B04371B78002B01D0FFF7D6FA2B6899
:101E2000019A1C121340B74A9B009B580435FFF7D8
:101E3000AEFA3B00083B1868FFF7A2F93B1F06000B
:101E40001868FFF79DF9F30FC217B0425341A40081
:101E50003A1B17009B001360A94B04371B78002B1B
:101E600001D0FFF7B2FA2B68019A1C121340A54A61
:101E70009B009B580435FFF78AFA3B00083B186823
:101E80003B1F1968A600BE1B0423814202D0042810
:101E900002D80023336018E001239C461842F8D191
:101EA0000F2302681A40042AF3D163461942F0D185
:101EB0000429EED90B680B321340042BE9D1FFF74C
:101EC0007FF9431E9841800030608D4BA4001B7841
:101ED0003F1B0437002B01D0FFF777FA2B68019ADC
:101EE0001C121340874A9B009B580435FFF74FFA9A
:101EF0003B00083B18683B1F1968A600BE1B002367
:101F0000814202D0042802D80423336018E0012360
:101F10009C461842F8D10F2302681A40042AF3D1D4
:101F200063461942F0D10429EED90B680B321340F5
:101F3000042BE9D1FFF744F9434258418000306057
:101F40006F4BA4001B783F1B0437002B01D0FFF719
:101F50003CFA2B68019A1C1213406A4A9B009B585A
:101F60000435FFF714FA3B00083B1868FFF708F93F
:101F70003B1F06001868FFF703F9F317C20F8642EC
:101F80005341A4003A1B17009B0013605C4B0437BD
:101F90001B78002B01D0FFF718FA2B68019A1C124E
:101FA0001340584A9B009B580435FFF7F0F93B005B
:101FB000083B1868FFF7E4F83B1F06001868FFF7B6
:101FC000DFF80023864200DD0433A4003A1B17002B
:101FD00013604B4B04371B78002B01D0FFF7F5F94A
:101FE0002B68019A1C121340464A9B009B580435EB
:101FF000FFF7CDF93B1F1B68A400043B5A1E934119
:102000003A1B17009B0013603D4B04371B78002BD5
:1020100001D0FFF7DAF92B68019A1C121340394AF4
:102020009B009B580435FFF7B2F93B00083B18684A
:10203000FFF7A6F83B1F06001868FFF7A1F8321853
:102040000120A4003B1B1F00520002431A602C4BCE
:1020500004371B78002B01D0FFF7B7F92B68019AE2
:102060001C121340274A9B009B580435FFF78FF939
:102070003B00083B1868FFF783F83B1F0600186811
:10208000FFF77EF8321A0120A4003B1B1F0052000C
:1020900002431A601A4B04371B78002B01D0FFF75C
:1020A00094F92B68019A1C121340164A9B009B5806
:1020B0000435FFF76CF93B00083B1868FFF760F840
:1020C0003B1F06001868FFF75BF802000120A40020
:1020D0003B1B1F007243520002431A60084B043737
:1020E0001B78002B01D0FFF770F92B68019A1C12A6
:1020F0001340044A9B009B580435FFF748F9C0463B
:10210000A8020020F8CE00003B1F1868FFF738F83F
:10211000061E17D11F23EE4A1370A4003B1B1F009D
:102120001E60EB4B04371B78002B01D0FFF74DF9F5
:102130002B68019A1C121340E64A9B009B580435F9
:10214000FFF725F93B00083B1868FFF719F8310045
:1021500007F098F9012640000643DEE73B1F1868A8
:10216000FFF70EF8061E17D11F23D94A1370A400DB
:102170003B1B1F001E60D64B04371B78002B01D081
:10218000FFF723F92B68019A1C121340D14A9B00D8
:102190009B580435FFF7FBF83B00083B1868FEF737
:1021A000EFFF310007F054FA012649000E43DEE745
:1021B0003B1F1868FEF7E4FFC21780185040012249
:1021C000A4003B1B1F00400010431860C04B0437A5
:1021D0001B78002B01D0FFF7F8F82B68019A1C122E
:1021E0001340BC4A9B009B580435FFF7D0F8A3006E
:1021F000FE1A3068012C24D1FEF7C2FF0494079028
:1022000009F064FD0799002900DC012107F020FA9C
:10221000049BA400C918012349001943AC4B3F1B80
:102220001B7831600437002B01D0FFF7CEF82B6804
:10223000019A1C121340A74A9B009B580435FFF7D4
:10224000A6F8FEF79DFF04907068FEF799FF049BC7
:102250000130C31A0793D3E7A300FE1A3100200010
:10226000049301F013FD049B3060FF1A984B043770
:102270001B78002B01D0FFF7A8F82B68019A1C12DD
:102280001340944A9B009B580435FFF780F83B00AD
:10229000083B1868FEF774FF3B1F06001868FEF73E
:1022A0006FFF02000120A4003B1B1F0032405200C0
:1022B00002431A60864B04371B78002B01D0FFF7CE
:1022C00084F82B68019A1C121340824A9B009B5889
:1022D0000435FFF75CF83B00083B1868FEF750FF39
:1022E00006003B1F1868FEF74BFF32000243012037
:1022F000A4003B1B1F00520002431A60744B0437BA
:102300001B78002B01D0FFF760F82B68019A1C1294
:102310001340704A9B009B580435FFF738F83B0088
:10232000083B1868FEF72CFF06003B1F1868FEF7F5
:1023300027FF320042400120A4003B1B1F00520037
:1023400002431A60624B04371B78002B01D0FFF761
:102350003CF82B68019A1C1213405E4A9B009B5864
:102360000435FFF714F83B1F1868FEF709FFC04358
:102370000122A4003B1B1F00400010431860544B77
:1023800004371B78002B01D0FFF71FF82B68019A48
:102390001C1213404F4A9B009B580435FEF7F7FF71
:1023A0003B00083B1868FEF7EBFE06003B1F186871
:1023B000FEF7E6FE3200824051000122A4003B1BE2
:1023C0001F000A431A60424B04371B78002B01D0D0
:1023D000FEF7FBFF2B68019A1C1213403D4A9B003D
:1023E0009B580435FEF7D3FF3B00083B1868FEF707
:1023F000C7FE06003B1F1868FEF7C2FE320002410E
:1024000051000122A4003B1B1F000A431A60304BFD
:1024100004371B78002B01D0FEF7D7FF2B68019AF9
:102420001C1213402B4A9B009B580435FEF7AFFF4C
:102430003B000C3B1868FEF7A3FE3B00083B060080
:102440001868FEF79DFEF1170200C317300007F071
:1024500051F93B1F049005911868FEF791FE0200A8
:102460000498059907F0FAF843000120A4003E1BE8
:1024700037001843164B30601B780437002B01D00F
:10248000FEF7A3FF2B68019A1C121340114A9B0010
:102490009B580435FEF77BFFA300FE1A3100200095
:1024A0000493FEF7B5FC049B3060FF1A084B043719
:1024B0001B78002B01D0FEF788FF2B68019A1C12B5
:1024C0001340044A9B009B580435FEF760FFC0464A
:1024D000A8020020F8CE0000A300FF1A3900200057
:1024E000FEF7AEFCE44B1B78002B01D0FEF76DFF2E
:1024F0002B68019A1C121340E04A9B009B5804353C
:10250000FEF745FFA300FE1A310020000493FEF7FA
:10251000D7FC049B3060FF1AD74B04371B78002B85
:1025200001D0FEF752FF2B68019A1C121340D34AC8
:102530009B009B580435FEF72AFFA300FF1A3900C1
:102540002000FEF751FDCC4B1B78002B01D0FEF78D
:102550003CFF2B68019A1C121340C84A9B009B58F1
:102560000435FEF714FFA300FE1A31002000049387
:10257000FEF7ACFD049B3060FF1ABF4B04371B789D
:10258000002B01D0FEF721FF2B68019A1C1213408B
:10259000BA4A9B009B580435FEF7F9FE3B1F1868AA
:1025A00000F0CEFF3A00083A12680300A400D107F9
:1025B00029D4042A0CD910680F22104001380828A9
:1025C0000FD806F0CBFE052026220E0E0E0E24009C
:1025D000AB49180009F01AFC434258413B1B8000EC
:1025E0001860A54B3F1B1B780437002B01D0FEF76A
:1025F000ECFE2B68019A1C121340A04A9B009B58CA
:102600000435FEF7C4FE9F49E3E79F49E1E79F4990
:10261000DFE79F49DDE7069B3E1DF31A964CD82B5A
:1026200003DD1A232370FEF7D0FE00F0E1FC430027
:102630000120184323783860002B02D03700FEF7C2
:10264000C4FE2B68019A1C1213408C4A9B009B58B5
:1026500037000435FEF79BFE069B3E1DF31A864CA1
:10266000D82B03DD1A232370FEF7AFFE00F0B6FC73
:10267000884B400018400123184323783860002B12
:1026800002D03700FEF7A1FE2B68019A1C121340FE
:102690007A4A9B009B5837000435FEF778FE069B6C
:1026A0003E1DF31A744CD82B03DD1A232370FEF75A
:1026B0008CFE00F09DFC784B1A68831A904201D280
:1026C000764A9B1801205B0003433B602378002B74
:1026D00002D03700FEF779FE2B68019A1C121340D6
:1026E000664A9B009B5837000435FEF750FE00F009
:1026F0007FFC694BA40018605F4B3F1B1B78002BCD
:1027000001D0FEF762FE2B68019A1C1213405B4A4F
:102710009B009B580435FEF73AFE0123A600BE1B22
:1027200020001A003100FEF779FD5D4C206864300E
:1027300002F0FAFE002802D1043DFEF759FE029B8A
:1027400021685A78574803F01EFB0123029A37008C
:10275000137000F043FC544B22681B68063253434D
:102760001818029B5860FEF743FEA600BE1B20000F
:10277000012300223100FEF751FD494C20686430EE
:1027800002F0D2FE0028D7D0464803F079F8DCE703
:10279000A4003E1BFEF7C2FD3700374B30601B78AC
:1027A0000437002B01D0FEF710FE2B68019A1C1293
:1027B0001340324A9B009B580435FEF7E8FD2E4B30
:1027C000A4001B783F1B002B01D0FEF7FEFD2B68F9
:1027D000019A1C121340294A9B009B580435FEF7AE
:1027E000D6FDA4003E1B300000F035FC3700224B24
:1027F00030601B780437002B01D0FEF7E6FD2B6814
:10280000019A1C1213401D4A9B009B580435FEF789
:10281000BEFDA4003E1B300000F01FFC3700164B2D
:1028200030601B780437002B01D0FEF7CEFD2B68FB
:10283000019A1C121340114A9B009B580435FEF765
:10284000A6FDA300FE1A31002000049300F008FC4E
:10285000049B3060FF1A084B04371B78002B01D013
:10286000FEF7B3FD2B68019A1C121340034A9B002C
:102870009B580435FEF78BFDA8020020F8CE00001F
:1028800034D100003CD1000043D100004AD1000007
:102890004FD10000FEFFFF7FD405002037894100A3
:1028A000CC050020A902002004000020A4003F1B4A
:1028B000380000F007FCFB4B1B78002B01D0FEF723
:1028C00084FD2B68019A1C121340F74A9B009B5809
:1028D0000435FEF75CFDA300FE1A310020000493CE
:1028E00000F018FC049B3060FF1AEE4B04371B7895
:1028F000002B01D0FEF769FD2B68019A1C121340D2
:10290000E94A9B009B580435FEF741FDA4003F1B9C
:10291000380000F041FCE34B1B78002B01D0FEF7A0
:1029200054FD2B68019A1C121340DF4A9B009B58F0
:102930000435FEF72CFD0121200000F015FCD94BD9
:102940001B78002B01D0FEF740FD2B68019A1C126A
:102950001340D54A9B009B580435FEF718FD002113
:10296000200000F001FCCF4B1B78002B01D0FEF7BC
:102970002CFD2B68019A1C121340CB4A9B009B58DC
:102980000435FEF704FDA4003E1B300000F026FCD9
:102990003700C44B30601B780437002B01D0FEF7A2
:1029A00014FD2B68019A1C121340BF4A9B009B58D0
:1029B0000435FEF7ECFCA4003E1B300000F022FCC6
:1029C0003700B84B30601B780437002B01D0FEF77E
:1029D000FCFC2B68019A1C121340B34A9B009B58C5
:1029E0000435FEF7D4FCA4003F1B380000F0E4FBE4
:1029F000AC4B1B78002B01D0FEF7E7FC2B68019A4B
:102A00001C121340A84A9B009B580435FEF7BFFCDC
:102A1000A4003F1B380003F011FDA24B1B78002BD4
:102A200001D0FEF7D2FC2B68019A1C1213409E4A7B
:102A30009B009B580435FEF7AAFCA4003E1B300007
:102A400003F096FD3700974B30601B780437002B5E
:102A500001D0FEF7BAFC2B68019A1C121340924A6F
:102A60009B009B580435FEF792FCA4003F1B3800E6
:102A700003F094FC8B4B1B78002B01D0FEF7A5FCD8
:102A80002B68019A1C121340874A9B009B580435FF
:102A9000FEF77DFCA4003E1B300003F095FC3700E0
:102AA000804B30601B780437002B01D0FEF78DFC83
:102AB0002B68019A1C1213407B4A9B009B580435DB
:102AC000FEF765FCA300FF1A3900200001F022FC8C
:102AD000744B1B78002B01D0FEF777FC2B68019A12
:102AE0001C121340704A9B009B580435FEF74FFCA4
:102AF000A300FF1A3900200001F020FA694B1B786F
:102B0000002B01D0FEF761FC2B68019A1C121340C8
:102B1000654A9B009B580435FEF739FCA300FF1A59
:102B20003900200001F02EFB5E4B1B78002B01D0FA
:102B3000FEF74BFC2B68019A1C1213405A4A9B006B
:102B40009B580435FEF723FCA300FF1A3900200030
:102B500001F040FB534B1B78002B01D0FEF735FCF6
:102B60002B68019A1C1213404F4A9B009B58043556
:102B7000FEF70DFCA300FE1A31002000049303F0C1
:102B80008FFD049B3060FF1A464B04371B78002BE7
:102B900001D0FEF71AFC2B68019A1C121340424A1E
:102BA0009B009B580435FEF7F2FBA300FE1A310090
:102BB0002000049303F07CFD049B3060FF1A394B26
:102BC00004371B78002B01D0FEF7FFFB2B68019A1E
:102BD0001C121340344A9B009B580435FEF7D7FB68
:102BE000A300FE1A31002000049303F069FD049B4A
:102BF0003060FF1A2B4B04371B78002B01D0FEF7F7
:102C0000E4FB2B68019A1C121340274A9B009B5837
:102C10000435FEF7BCFBA300FE1A3100200004932C
:102C200003F026FB049B3060FF1A1E4B04371B7811
:102C3000002B01D0FEF7C9FB2B68019A1C12134030
:102C4000194A9B009B580435FEF7A1FBA300FF1A0D
:102C50003900200001F0AAF9124B1B78002B01D09B
:102C6000FEF7B3FB2B68019A1C1213400E4A9B001F
:102C70009B580435FEF78BFBA300FF1A3900200098
:102C800001F0D0FA074B1B78002B01D0FEF79DFB1B
:102C90002B68019A1C121340034A9B009B58043571
:102CA000FEF775FBA8020020F8CE0000A300FE1A74
:102CB00031002000049301F031FA049B3060FF1AC8
:102CC000304B04371B78002B01D0FEF77EFB2B68BE
:102CD000019A1C1213402C4A9B009B580435FEF7A6
:102CE00056FBA300FF1A3900200001F0DFF9254B45
:102CF0001B78002B01D0FEF768FB2B68019A1C1291
:102D00001340214A9B009B580435FEF740FB069B6D
:102D1000029AFB1A9B101361A300FF1A39002000CE
:102D200002F0ECFD174B1B78002B01D0FEF74DFB9A
:102D30002B68019A1C121340134A9B009B580435C0
:102D4000FEF725FB069B029AFB1A9B101361A3005A
:102D5000FE1A31002000049302F0D0FD049B306085
:102D6000FF1A084B04371B78002B01D0FEF72DFB10
:102D70002B68019A1C121340034A9B009B58043590
:102D8000FEF705FBA8020020F8CE00000023F7B5EF
:102D90005A1E0192002B07DA01F0D2FA02F0DEFE91
:102DA00003F050F81923019300263000194B1968DD
:102DB000B14212DD184B1A6801328A420FDAF02450
:102DC0001A601D68154F6C43E35D002B1FD0E4199A
:102DD000022B06D12000FEF7B9FA019BD8E70022AA
:102DE000EDE7012B0DD1002801D100F0F7F8F0221A
:102DF0006A43BB185B680A49C31A8B4201D8022395
:102E0000BB54F0235D43054BEB5C022BE2D0013653
:102E1000CCE7C046D0050020000000203C1C00206C
:102E20003F420F00012200210A4B0B481A61195042
:102E300004301950A2210420C9005850C121C020DB
:102E40008900800258501A60044BFC311960044B11
:102E50001A70704700A000400405000000E100E087
:102E6000FB05002004207047F8B550C9012322005B
:102E70001A40101E2DD03340181E2AD06410002096
:102E80001C2C26D81D4B761035009E4200DD1D00FF
:102E90001B4F3B5D012B05D00121200004F036FEC5
:102EA00001233B55174B1B78002B01D1FFF7BAFFCD
:102EB0000023154A9E420DDCFF2514491448D65CB8
:102EC000B44202D15E007052D5540133042BF6D1C6
:102ED0000420F8BDD15C8C4203D10C4A5B009D52AA
:102EE000F6E70133042BF5D10023D15CFF2901D192
:102EF000D454F2E70133042BF7D1E9E7881300003B
:102F0000DC050020FB0500201C0000200E00002036
:102F1000DC05000070B530C9012322001A40101EE4
:102F20001BD02B40181E18D064101C2C00D9002474
:102F3000174E335D012B05D00121200004F0E6FD82
:102F40000123335569100800124A1038124B904281
:102F500004D9012252421A60042070BD1C600F483F
:102F600006F090FA0E4B18800E4B1B78002B02D106
:102F7000FFF758FFF0E701220B4B9A64A922D20019
:102F80009A588018A82280B2D2009850E4E7C04630
:102F9000DC050020908601001800002020A1070019
:102FA0000C000020FB05002000A00040030010B52D
:102FB0000120002B02DC1B30FEF7AAF910BD042013
:102FC000704710B5002803DC1C20FEF7A1F910BDE6
:102FD0000B680020DB07FAD40D30F6E70122034B23
:102FE0001A64A822D20098587047C046008000405A
:102FF00010B5FFF7F3FFFA21890006F0B9F910BD0B
:1030000000487047ACD100001D20704770B5054ED8
:103010000400335C0D008B4202D004F077FD35557F
:1030200070BDC046DC05002070B50024084D635D0E
:10303000012B09D10021200004F08EFD0021200089
:1030400004F064FD0023635501341D2CEED170BDE6
:10305000DC05002070470D2070473B2070470000C2
:10306000F8B501240B6806000D00234204D10D20A1
:10307000FEF74EF92000F8BD5B102000052BFAD8B2
:103080000E4A9B009C580E4F3B5D002B05D0002143
:10309000200004F03BFD00233B55012E06DD6B684C
:1030A000042B03D10221200004F030FD200004F0A5
:1030B000DBFB012440002043DDE7C04694D1000043
:1030C000DC050020F8B501260568354202D04468C9
:1030D000344203D10D20FEF71BF9F8BD6D101C2DF5
:1030E000FBD80A4F7B5D012B04D03100280004F08F
:1030F0000DFD7E55064964108C4202DCE143C91780
:103100002140280004F036FCE7E7C046DC0500203B
:10311000FF03000070B501240D68254204D10D2085
:10312000FEF7F6F8200070BD6D101C2D17D8002496
:10313000012804DD4C68043C63425C416400094E94
:10314000735DA34204D02100280004F0DFFC745515
:10315000280004F01FFD03000420012BE3D0002011
:10316000E1E7C046DC05002070B504000D001C2816
:103170000ED8084E335C012B04D0012104F0C6FCAC
:1031800001233355290020004D1EA94104F0E4FC21
:1031900070BDC046DC050020036810B5DA0703D413
:1031A0000D20FEF7B5F810BD4168581004394A42A9
:1031B0005141FFF7D9FFF6E737B569460A00064BDC
:1031C00030CB30C203680220042B02D100F0DAFFBA
:1031D00037BD00F0FFFFFBE75CD1000010B5084CE5
:1031E0006379002B05D00021052004F08FFC00231B
:1031F0006371052004F0CEFC43425841800010BDAD
:10320000DC05002010B5084CE37A002B05D0002126
:103210000B2004F07BFC0023E3720B2004F0BAFCCB
:1032200043425841800010BDDC050020704700007B
:10323000F7B5304D304E6B6C002B15D0A824002311
:10324000E40037596B642D4B186800280CDB2C4BBD
:1032500019784A425141C9B2197004F07DFC294BDA
:103260001B88DF19BFB23751AB6C002B39D000215E
:10327000254B264FF458A9643A780C340193244D19
:103280008A4206D02B68032B03D8224AD05C04F074
:1032900063FC2B68204A0133134004D50422013B10
:1032A0005242134301331B4900228C462B60042BEE
:1032B00018D06046C05C591CFF2802D10B000122C7
:1032C000F5E7002A00D02B60012104F045FC012322
:1032D0003B702B68114A5B009B5AE418019BA4B217
:1032E000F450F7BD01235B422B6000233B700C4B75
:1032F000F3E7C046FCA0004000A0004018000020FA
:10330000FA0500200C00002044050000F90500200B
:10331000D80500201C000020030000800E000020C3
:1033200050460000084B094AFF201A805A809A80B4
:10333000DA800023064A07491370074A087048706C
:103340008870C870136070470E000020DC05000014
:10335000F90500201C000020D80500200122024BA6
:1033600052421A607047C0461800002010B5034A48
:103370000621034802F09EF810BDC04664D100004B
:10338000CED80000E12170B54902194803F0E0FFF2
:10339000002401220320174B17491A615C500431A5
:1033A00058508018083158501A60063004F056FA08
:1033B000FF21124AA15401341D2CFBD1012200200F
:1033C0000F4B01001A6004230E4A0F4D1468002CA5
:1033D000FCD02C680002013B20431160002BF5D18A
:1033E00001220A4B1A6004F06FF901F0F5F870BD84
:1033F000C41B00200080004004050000DC05002004
:1034000000D0004000D1004008D5004004D000406A
:10341000F8B50B4E070030000D0003F0E1FF04008B
:10342000A84200DD2C003D00EB1B9C4205DD300076
:1034300003F0E0FF28700135F6E72000F8BDC04634
:10344000C41B002010B50100014803F089FF10BD26
:10345000C41B002010B5054C200003F08FFFE121B4
:103460002000490203F074FF10BDC046C41B0020B9
:10347000C3070CD4064B1B68834208D8054B1B6856
:10348000984204D8031F1B68002B00D01800704717
:1034900004060020000600200023012210B50A487F
:1034A000990001334250642BFAD1084C084B00219B
:1034B0001A602000074A08F029F9074B074A6360A1
:1034C000074B1A6010BDC046942D0020080600204E
:1034D00008000020D4090000302700000C0600205E
:1034E000FC05002010B5044B044A1A60044B054A41
:1034F0001A60FFF7D1FF10BD040600200806002067
:1035000000060020DC0F0020044B1B68186800092F
:1035100080B20238C343DB1718407047FC05002017
:1035200000B59BB00200054901A808F033FC01A8D2
:1035300002F0C2F902F086FCFCE7C04630D200007F
:103540000B4BC20704D4042804D80A4B00D00A4B02
:10355000180070470F2203681A40031D042AF7D091
:10356000064B092AF4D0064B032AF1D0054BEFE7AE
:103570000AD20000AECD0000A8CD000014D2000099
:1035800024D200001BD200000020064A0649131F67
:10359000186013681B099BB202339B00D2188A4241
:1035A000F5D370470C060020DC0F0020F7B50F2480
:1035B0000126314B314A1968314B324D1868136876
:1035C0001F002740072F26D813681B099BB2023320
:1035D0009B00D218AA42F2D300242B4EA500AD19AD
:1035E0002868FFF745FF01342860642CF6D1274C8A
:1035F0002068FFF73DFF2060254C2068002802D09E
:10360000FFF736FF20600025224B1B680093009BCC
:103610009D4214DBF7BD1B099BB29B00D3189A4255
:10362000D2D01F68374208D1B94206D2B84204D37B
:10363000043F3F68002F00D01F60043BEFE7F023FA
:103640006B43154A9B181A78002A01D10135DEE731
:103650001F693C2300266B43DB199B000193013655
:10366000BB1BF3D4019BB4001C1B0B4B1C19A069A2
:10367000FFF7FEFEA061F2E7040600200C06002022
:1036800000060020DC0F0020942D00200800002000
:10369000DC0F0020D00500203C1C0020F7B50124E1
:1036A000204246D1234B1B689C46984241D3224B73
:1036B0001B68019398423CD8031F1B68002B38D12C
:1036C0000200036800941B099BB2002B0FD10099E4
:1036D000131F196090422CD015682B1F1B6899008E
:1036E00069180C68013B14600A602A00EDE79D0030
:1036F00055192968009C214219D18C4517D8019C85
:103700008C4214D30E1F3468002C10D10F680F3474
:103710003C40072C08D92F60151F2B600B680A60EE
:103720001B099BB20A00D0E700993160CDE7013B4D
:10373000CBE7F7BD04060020000600200D4970B558
:103740000A000D4D1368141F1B0926689BB2981CB4
:10375000002E0BD000238A4200D00B002360830090
:10376000C91880001218AA42ECD370BD1B01136067
:10377000F7E7C0460C060020DC0F0020F8B5124C1D
:1037800027000F223B681D09ADB213420DD06E1CFD
:10379000B600A74204D032003900200007F0A3FF92
:1037A0000022A3190436A4191A600235AD00074B94
:1037B0007F199F42E5D31B1B9B10013B1B0123601C
:1037C000034B1C60F8BDC0460C060020DC0F002037
:1037D000FC050020F0B59BB0FFF700FC00240700BB
:1037E000214AA300D0580134FFF758FF642CF7D1C9
:1037F0001E4B1868FFF752FF1D4B1868002801D0B8
:10380000FFF74CFF00261B4B1B689E4217DBFFF7A0
:1038100095FFFFF7CBFEFFF7B1FFFFF7DFFB164B7E
:10382000C21B1B6815491B6801A81B099BB2023B00
:1038300008F0B0FA01A802F03FF81BB0F0BDF02587
:1038400075430F4BED182B78002B01D10136DAE7C9
:103850002B695C1E002CF9DBA300EB189869FFF7BD
:103860001DFF013CF6E7C046942D00200800002013
:10387000DC0F0020D0050020FC050020EAD100006C
:103880003C1C0020F7B5174D4F1C2B6806001B6829
:103890000C001B099BB201929F420BDBFFF79AFFC2
:1038A0002B681B681B099BB29F4203DB0A20FDF7B4
:1038B0002FFDFEBD2868A71CBA00DB1B81181B0169
:1038C0000B6029600021031F19600F231E400300B5
:1038D0002401264340C3083A9A189A42E9D901992B
:1038E00002C3FAE7FC050020F7B5030001221340EC
:1038F00004000D000193002B2BD1174B1B68834252
:1039000027D8164B1B68834223D90F23144F3860E6
:1039100000681840FFF7B6FF019B3C68061E3B603D
:1039200017D0236804301B099BB29D4200DD1D00A7
:10393000AA00211D251F07F0CDFEFFF725FE2E60F2
:10394000FFF734FE00232B602268064B13402360F0
:1039500034002000FEBDC046040600200006002002
:10396000DC0F0020F0FF0F000323043010B5C11757
:1039700019400918891000220420FFF783FF10BDA9
:1039800070B5050008000C00FFF7EEFF00230028CB
:1039900004D170BDE95CC21811710133A342F9DB97
:1039A000E343DB171C40002304192371F1E7F0B552
:1039B0000C009BB0022804DC1C20FDF7A9FC1BB006
:1039C000F0BD01230868184206D1042804D90F2647
:1039D00001683140042901D00E20EEE761680D0036
:1039E0001D40F9D10429F7D90A683240042AF3D1DD
:1039F000A2681A4201D10D20DFE7FFF7A1FD060002
:103A00006068FFF79DFDA768010001AC7F103000E2
:103A1000257003F034F839006423220003F094F891
:103A2000200008F0FDF901002000FFF7A9FFC6E71C
:103A300010B51C4CA544041E02D1FFF795FF0BE006
:103A400002F036FF0138062828D805F087FC09095E
:103A500011182904240000208023DB009D4410BDA0
:103A6000200002F0A1FF011B2000FFF789FFF3E710
:103A7000200002F047FF430001201843ECE78022BA
:103A80006946D200200002F054FF684608F0C8F9E9
:103A900001006846E9E704210348E6E70020CCE797
:103AA0000420D9E700FCFFFF78D2000070B50C00BD
:103AB000022803DC1C20FDF72BFC70BD01230868E5
:103AC000184206D1042804D90F2501682940042989
:103AD00001D00E20EFE761681942FAD10429F8D924
:103AE0000A682A40042AF4D1A2681A4201D10D20A2
:103AF000E1E7FFF725FD05006068FFF721FDA468F9
:103B000001006410280002F0BAFF210002F0F7FF64
:103B1000FFF78EFFD1E770B50D00012803DC1C20F4
:103B2000FDF7F6FB70BD01240868204206D1042889
:103B300004D90F2102680A40042A01D00E20EFE7C1
:103B40006A682242FAD1042AF8D913680B40042B80
:103B5000F4D1FFF7F5FC06006868FFF7F1FC0100FF
:103B6000300002F08CFF03F00EF840002043D9E74C
:103B7000F8B507000C001C20012F0BDD012508689B
:103B8000284206D1042804D90F2102680A40042AD9
:103B900003D00E20FDF7BCFBF8BD62682A42F8D1C5
:103BA000042AF6D913680B40042BF2D1FFF7C8FCA6
:103BB00006006068FFF7C4FC0100022F14D0A4685F
:103BC0002C4211D06410300002F059FF050002F0C1
:103BD0006FFE012811D1002C02DD0135012C06D128
:103BE0002800FFF725FFD7E701246442EBE7280010
:103BF00002F0E6FE013C0500F0E70228F0D1002CBF
:103C0000EEDD0135012CEBD000222800110002F07E
:103C100009FF02F0D5FE013C0500F3E710B50124D1
:103C20000868044016D04410200005F0BFFE154976
:103C300005F08AFD07F070FC04F0C2F80022124B78
:103C400006F024FE04F064F807F0F6FB43000120C0
:103C5000184310BD042810D90F2302681340042B09
:103C600007D1FFF76DFC21000A2208F0A1F904003A
:103C7000DAE7032B01D10430F5E70D20FDF748FB0F
:103C8000D2E7C046D30237390000D040086870B58B
:103C900001240500254006D1042804D90F23026819
:103CA0001340042B03D00E20FDF732FB70BDFFF74D
:103CB00047FC03782900233B5A4253411022C01885
:103CC00008F076F980239B05C218044B9A4201D96B
:103CD0001420E9E740002043E8E7C046FFFFFF3F2C
:103CE00010B5034A0621034801F0E4FB10BDC046AD
:103CF00048D2000041D200000020704710B51E20BD
:103D0000FDF706FB10BD10B51E20FDF701FB10BD31
:103D100010B51E20FDF7FCFA10BD10B51E20FDF7F2
:103D2000F7FA10BD10B51E20FDF7F2FA10BD10B560
:103D30001E20FDF7EDFA10BD10B51E20FDF7E8FAC4
:103D400010BD10B51E20FDF7E3FA10BD10B51E2002
:103D5000FDF7DEFA10BD10B51E20FDF7D9FA10BD33
:103D600010B5034A0B21034801F0A4FB10BDC04667
:103D7000B4D200000CD300000120034B1860034BA9
:103D80001B6883401843704700100020E00F00209C
:103D9000F0B5EFF310810123194083F31088134C21
:103DA000134AA4461268134E013A9340124F134A25
:103DB000002B17D0146803420FD03D682C60C0461A
:103DC000C046C046C046C046C046C046C0460C4C71
:103DD0001568246825605B08EAE765462C6014686E
:103DE0003460F8E781F31088F0BDC0460805005044
:103DF000200000200C050050EC0F0020F40F0020E4
:103E0000E80F002030B585B001AD0C22064928002E
:103E100007F060FC0024285D01210134FFF7F6F86B
:103E20000C2CF8D105B030BDA1D30000F7B56A461F
:103E30003B4B01AE13800A2393703A4B33801C2313
:103E4000B370FFF7CBF8384B384DC0182B68984249
:103E500001D200232B602C68002C41D1375D012159
:103E60003800FFF7D3F801340021380003F074FE66
:103E7000032CF3D1002401276B461E5D390030006E
:103E8000FFF7C4F801343900300003F065FE032C5D
:103E9000F2D1C8200138C046C046C046C046C04620
:103EA000C046C046C046C046C046C046C046F1D126
:103EB0006B4600211878FFF7A9F86B460021587867
:103EC000FFF7A4F86B4600219878FFF79FF8FFF7FB
:103ED00085F8FA2300241B01C01828602000FEBDCD
:103EE000FFF77CF82B6800249842F7D3032003F0F7
:103EF000BBFC0600042003F0B7FC36180A2003F0D0
:103F0000B3FC0B4B9B1B181A0A4BA04206DB186034
:103F10000023094A2B6013600124DFE71C60F7E7E8
:103F2000030400001A1B000010270000F80F0020F7
:103F3000E3030000E00F0020001000200022054BEA
:103F400010B51A60044B1B68934201D002F050FC7C
:103F5000002010BDFC0F0020E81A002010B5041E40
:103F600010DA00240A4BA400E25801239340094AC6
:103F700009491360094A1160094A0A4911600A4A4D
:103F8000136010BDFFF740F8A042EADDEAE7C04643
:103F9000C8E00000F40F002008050050EC0F0020DE
:103FA000E80F00200C05005018050050F0B53B4B01
:103FB00085B01B680C00002B03D101204042FFF7A5
:103FC000CDFF246801222700174028D0FF2360126C
:103FD000184033496714661040431F401E4005F0E7
:103FE00051FA050438002E49784305F04BFA0002D7
:103FF000054330002A49704305F044FA294B284311
:104000001B68202B06D16400A40E274BA400E358A4
:1040100000021843FFF7BCFE002005B0F0BD042CE1
:10402000FAD90F2321680B40092BF5D1636803925D
:104030005B100193019B9F42EEDABB00E3189E6880
:10404000039B1E4228D0FF237012184072101A40A2
:104050001349751440431D40009205F013FA030400
:1040600028000F496843029305F00CFA029D0002F4
:10407000054300980A49404305F004FA094B2843D8
:104080001B68202B06D17600B60E074BB600F558FC
:1040900000022843FFF77CFE0137CBE7F40F002036
:1040A000590600002000002088D5000002000868A2
:1040B00010B5C3070FD540101823012A03DD4A6845
:1040C000042A00D10833054A1360FEF7C3FFFFF747
:1040D00045FF002010BD01204042EDE720000020F8
:1040E00010B50124044002D04410200010BD042863
:1040F00010D90F2302681340042B07D1FFF720FAD1
:1041000021000A2207F054FF0400EEE7032B01D13F
:104110000430F5E70D20FDF7FBF8E6E70868F8B591
:10412000C3071AD5FFF7DCFF0300203B5E2B25D821
:104130000520434301221D180020114E9D4219D035
:1041400005211024F75C3C4200D080180139520050
:1041500064100029F7D10133F0E704280ED90F22AB
:1041600003681A40042A09D11B099BB2002B05D011
:104170000379DAE7012340001843F8BD0120FCE78A
:10418000ADD3000070B508680D00FFF7A9FF04006B
:104190006868FFF7A5FF621E0100042A14D8451EB7
:1041A000042D11D805236B439B18012215009D4057
:1041B0002B00064805682B430360054B1B68002B4A
:1041C00002D0200002F015FB002070BDFC0F002083
:1041D000E81A002070B508680D00FFF781FF0400A1
:1041E0006868FFF77DFF621E0100042A13D8451E90
:1041F000042D10D805236B439B1801229A400748D1
:10420000036893430360064B1B68002B03D0002216
:10421000200002F0EEFA002070BDC046FC0F002026
:10422000E81A0020F0B5050089B008680C00FFF717
:1042300057FF0690022D36DD6068FFF751FF0190B1
:10424000A068FFF74DFF04000127231D661E07939A
:10425000731C0293079B9E4235D00523734305933D
:10426000019B019D05330493049BAB421ED0042E99
:1042700016D86B1E042B13D80122059B2349013B42
:104280005B199A409446224A0B681068069A3A4095
:1042900003920DD062461A430A60012200280DD114
:1042A0007F000135E0E701240194CDE7029ECFE7CE
:1042B000624693430B600028F2D0039A02992800CB
:1042C00002F097FAECE7019B1E1D042E1AD8012C70
:1042D00018D1002505273B0021006B439B1999400D
:1042E0000B000A4A013511689943094B11601B689C
:1042F000002B05D0019B0022581D290002F079FAFD
:10430000052DE8D1002009B0F0BDC046FC0F00200B
:10431000E81A0020086810B5C30703D5FFF7E0FED0
:10432000054B1860054B1B68002B03D0024B186827
:1043300002F060FA002010BDFC0F0020E81A0020F7
:104340007FB5A04C2368002B0AD19F4A1268002A2F
:1043500006D19E4B1B68002B01D0FFF767FD7FBD88
:104360009B4D2A68002A26D1984A1268002A1BD041
:10437000FFF75CFD0028F2D0FFF744FD924B246864
:104380001A681C60002A16D0002C14D101AD0C2232
:104390009049280007F09EF9285D00210134FEF7BE
:1043A00035FE0C2CF8D1DAE7874A1268002AE5D1ED
:1043B000002BE3D0E0E700211A2003F0CDFB002121
:1043C0001B2003F0C9FB00211C2003F0C5FB2E6855
:1043D000012E5CD0022E00D1A2E0002E50D1013679
:1043E0003100794C03202368994303F0B5FB042086
:1043F000216801404B42594103F0AEFB1021236874
:104400000A2019404B42594103F0A6FB8021236842
:10441000090119404B425941062003F09DFB8021C0
:104420002368090219404B425941072003F094FBCD
:1044300080212368490219404B425941092003F069
:104440008BFB80212368890219404B425941192076
:1044500003F082FB80212368C90219404B42594175
:10446000182003F079FB802321681B0319404B427D
:104470005941172003F070FB31001A2003F06CFB48
:104480002B680321581C05F0E3F8296067E7022137
:104490004D4C1720236819404B42594103F05CFBF7
:1044A00008212368182019404B42594103F054FB5E
:1044B00080212368C90019404B425941042003F070
:1044C0004BFB80212368490119404B4259410A2086
:1044D00003F042FB80212368C90119404B42594136
:1044E000032003F039FB80212368890319404B42E4
:1044F0005941092003F030FB802321681B04194037
:104500004B425941192003F027FB3100062003F0EC
:1045100023FB3100072003F01FFB31001B20ADE718
:104520002021294C1720236819404B42594103F0A0
:1045300013FB40212368182019404B42594103F0D6
:104540000BFB80212368192019404B42594103F08D
:1045500003FB80212368490019404B42594109203F
:1045600003F0FAFA80212368890019404B4259412F
:10457000072003F0F1FA80212368890119404B429A
:104580005941062003F0E8FA8021236849031940C5
:104590004B4259410A2003F0DFFA80212368C90306
:1045A00019404B425941032003F0D6FA8023216879
:1045B0005B0419404B425941042003F0CDFA01211C
:1045C0001C205BE7FC0F0020F00F002000100020F3
:1045D000E40F0020A1D30000012010B54042FFF7F6
:1045E000BDFC10BD10B5034A0921034800F062FF6D
:1045F00010BDC04688D60000D0D600008023F0B59C
:1046000002255B051A690A4C0A4BA1261D51032796
:104610008025F600ED00BA43884202D300221A51E9
:10462000F0BD5F59002FFCD098518018F4E7C046C8
:104630000405000000E0014010B5002806D1C020AC
:10464000B02140028902FFF7D9FF10BDB0208021C0
:104650008002C902F7E7000043425841064B40423E
:104660001840B0239B02C018036800201A0E532A7A
:1046700001D11B02180A704700C0FEFF30B50124AB
:104680008025054B054AED009C505C59002CFCD060
:1046900001600021995030BD00E001400405000098
:1046A00043425841074B40421840B0239B02C01878
:1046B000A62310B50902DB05090A1943FFF7DEFF3F
:1046C00010BDC04600C0FEFFF0B5012480260D4B92
:1046D0000D4DF6005C51002902DC00225A51F0BD5C
:1046E000577814783F022743947824042743D478DA
:1046F000043224063C439F59002FFCD010C00139DE
:10470000E9E7C04600E001400405000070B505007F
:104710004B680A009C1C2100A400FFF7D5FF281954
:1047200070BD0000134B1B68002B0CD08022B023FF
:10473000D2029B0200280BD11A1D5B681B0E522B64
:1047400000D110007047B022C02392025B02F1E753
:1047500082420DD903681B0E522B09D143680233E4
:104760009B00C018824203D903681B0E522BE9D06C
:104770000020E7E704110020F0B50020B7B00024C6
:10478000FFF7D0FF270005002600002D2ED1284D71
:104790002868FFF761FF32003B0001900094254933
:1047A00004A807F0F7FA04A801F086F8224B642069
:1047B0001C682B68A0215A425341204A5B42134097
:1047C000B02292029B18E41A6043490204F05AFE98
:1047D000A0225202030000921949220004A807F007
:1047E000D9FA04A801F068F837B0F0BDFF226B6871
:1047F00029689C460233FF180B12013613409C4275
:1048000000DA1C00FF200A140240039262460140B5
:1048100001920091039A0B4904A807F0BBFA04A87F
:1048200001F04AF82800FFF77DFF0500ADE7C0461C
:1048300004110020DAD700000811002000C0FEFF9C
:1048400084D70000C6D7000070B50020FFF704FF32
:1048500004000120FFF700FF844200DA04000A4B45
:104860001D686A42554128001D60FFF7E5FEA02241
:104870006B4252021340054A28009B18044A611CEF
:104880001360FFF70DFF70BD0411002004800100CC
:1048900008110020F8B50020FFF7DEFE0700012018
:1048A000FFF7DAFE3E00204D0643204C0DD180215B
:1048B000C020C9024002FFF7A1FE01213000FFF72E
:1048C000EFFE1B4B2E6023601DE0874209DD0023B5
:1048D000B0212B60164B890223602368002001253C
:1048E00017E0012380212B60124BC9022360F4E7FB
:1048F000120E522A08D0002800D023600E4800F083
:10490000DBFFFFF7A1FFF8BD28005A6802329200D2
:104910009B188B4205D21A68561CE9D10028F2D0A8
:10492000D1E72160EFE7C046041100200811002004
:104930000480010004C002009FD7000070B5002071
:10494000FFF7F0FEFF260500002801D1280070BD0A
:1049500003681C143440FFF7E5FEDA2CF4D105009F
:10496000F2E700008022F0B55200A1B000216748B4
:1049700006F0CCFE802200215200654806F0C6FEFB
:10498000644BFF271B681A00049353425A411000DE
:104990000592FFF751FE049C0020631E9C415E4B74
:1049A00064421C405D4BE418FFF7C8FF0600002E70
:1049B0002DD10498FFF750FE411C0598FFF770FEBB
:1049C000059A574D534B2C601A60FEF743FD514B2F
:1049D00064201B68A0215A4253414F4A5B42134056
:1049E000B0222C6892029B18E41A6043490204F03A
:1049F00049FDA0225202030000924A49220007A862
:104A000007F0C8F907A800F057FF21B0F0BD3268E1
:104A1000131412123A403B4003921A000A3A092A30
:104A200049D83A4B039A995C002931D110223E486B
:104A300006F06CFE35002B6803991A123A40914239
:104A400009D11A143A400B2A27D0132A2DD00A2A4A
:104A500001D1354B1D602800FFF764FE051EEAD129
:104A6000314B196800290FD02000FFF74FFE0400DA
:104A70002D4B5B195968002903D02000FFF746FE33
:104A8000040004350C2DF3D1204B0121039A9954D5
:104A90003000FFF747FE060089E73B40022BDADCD7
:104AA000214A9B00D3185D60D5E7102200211E48E3
:104AB00006F02CFECFE71A00153A082AE8D8144A67
:104AC0000399525C002AE3D13500152B00D0150064
:104AD000300003681A143A40152A0FD01D2A00D15D
:104AE0000025FFF71FFE0028F3D1002D04D0200081
:104AF0002900FFF70BFE0400054BC6E7039A1B12C3
:104B00003B409A42EDD10500EBE7C046041000207F
:104B10000C1100200411002000C0FEFF04C00200A0
:104B20000811002069D70000242F002010B5FFF7DE
:104B300019FF10BDF0B585B0039203220333DC17D3
:104B4000294D1440E4182B68284F5A4253418022C3
:104B50005B42D202A4103B409B18A21C0291244E3F
:104B6000910000910190316800980A18934215D283
:104B7000FFF7F8FE2B685A42534180225B421F40E8
:104B8000D202BF183368009A9B189F4206D2194878
:104B900000F092FE0025280005B0F0BD029B3568AC
:104BA00019066B461A7BA423DB051343FF222F0053
:104BB000090C1943019B12041B04134019432800DC
:104BC000FFF75CFD0837281D21003760FFF756FD11
:104BD000002C04D00A9A21003800FFF775FD009BD5
:104BE000083BFF183760D6E70411002000C0FEFF25
:104BF0000811002043D7000070B59AB0FFF74AFEB5
:104C0000FF221E4CD2000021200006F07FFDFF2570
:104C1000FFF794FE0026002814D10200C300E358D9
:104C20000130591E8B41D218FF28F7D1144901A831
:104C300007F0B0F801A800F03FFE124800F03CFE7B
:104C40001AB070BD03681A142A400A2A0AD11A122F
:104C50002A40FF2A03D0D200A1180B71A050FFF701
:104C600061FDD8E7132AFAD11B122B40FF2BF6D097
:104C7000DB00E2181671E650F1E7C0469C250020E3
:104C80000FD8000023D800000021094B094A5960C1
:104C90000131516059680029FCD0002119610123BC
:104CA00093600222044B8131FF315A501A607047E1
:104CB000FC1000400010004000E100E00222064B22
:104CC0000121DA670022054B5A61054A11615A69D0
:104CD000002AFCD07047C04604E100E0FC10004010
:104CE0000010004010B5044C2378002B01D0FFF7D2
:104CF000E5FF0020207010BD0D1200208023012050
:104D00005B055B6E5B001843704700000120024B9F
:104D10001B685B0018437047901200200120024B73
:104D20001B685B0018437047240000200120024BE1
:104D30001B685B00184370479412002070B5040094
:104D40000D001600FEF754F9802301215B055A6E11
:104D50002670002653006170E1706272010A5A0ADF
:104D60006071A171A272010C5A0C000E5B0EA6704C
:104D70002571E1712072E272237370BD10B5044C8D
:104D8000200007F04DF801002000FEF7F9FD10BDEE
:104D9000991200200E4B10B51B680E4C5A1C0FD0F8
:104DA0000D4C002B0CD00D4C012B09D00C4C022BC0
:104DB00006D0094C042B03D00A4C052B00D1074C1C
:104DC000200007F02DF801002000FEF7D9FD10BDEE
:104DD00028000020B4D800003CD10000BFD800005B
:104DE00043D10000B9D8000070B5214C2278002AC8
:104DF0003DD1204B01215A608022D20511605A68B2
:104E0000002AFCD0002207201B4B1C4901255A50C8
:104E10000439585008315A5019481A4958501A49FB
:104E20001A485A501A495A50A622D2009D500822B8
:104E300018495A5004315850022017495850174900
:104E400017485850174804395850182016495850D8
:104E5000C12189005A500539FF3958589218024328
:104E60005A501249124A9950FFF70EFF257070BD33
:104E70000D120020FC000040001000400C05000056
:104E8000746962751C0500002405000020000402FE
:104E90002C05000014050000340500003C0500004E
:104EA000FFFF000021100100540500000E12002039
:104EB0000405000070B50E4B06001B78002B01D1D5
:104EC000FFF792FF00200B4D2C7884420ED00A4B46
:104ED000202219780323091B1940084B4901C918DE
:104EE000300006F0F7FB0120013C2C7070BDC0467D
:104EF0000D120020981200200C1200200E1200202B
:104F0000002370B588B0984235DD0D6801262C006D
:104F100034409C422FD12300042D2CD90F222B6822
:104F20001A402300092A26D16A683F2A23DD6846F1
:104F3000FFF7C0FF230000281DD06B46197833000F
:104F4000A14203DB6B461B5D5B003343A200AA1842
:104F500001349360202CF2D1092169444A780B78FE
:104F600012021A438B781B041A43CB781B06134397
:104F7000024A13600423180008B070BD9412002088
:104F800070B5454B8AB01B78002B01D1FFF72CFF81
:104F900002AC2000FFF78EFF002802D100200AB0EB
:104FA00070BD23780B2BF9D96378012BF6D1E37808
:104FB000012BF3D100231120384E394D33602B7073
:104FC00068442379374A4178136002780902114313
:104FD000827812041143C27812060A4332490A60E9
:104FE000002B0ED1152169444A780B7812021A431E
:104FF0008B781B041A43CB781B06134333600023C2
:1050000018E0012B1AD1152169444A780B78120255
:105010001A438B781B041A43CB781A211B061343BF
:1050200033600E23627C6944934200DD130000224A
:105030009A422CD100220420EA54B0E7022B03D17B
:10504000627B10331621EEE7042B0DD115210822C7
:105050006944684606F03EFB0098019902F0C8FDDD
:1050600006F0EAF93060CAE7052BC8D115210822FD
:105070006944684606F02EFB0098019902F0B8FDDD
:1050800006F0DAF93060627D0A231E21CBE7885CE6
:10509000A8540132CCE7C0460D1200209012002027
:1050A00099120020280000209412002010B5134B04
:1050B00004001B78002B01D1FFF796FEFFF7FEFDE1
:1050C00000200F4A0F49104B5450586001301060B7
:1050D00058680028FCD000201861013090601869E1
:1050E0000028FCD0094B0A481B785B011B18535061
:1050F000FFF7E4FDFFF7C8FD10BDC0460D1200200C
:105100000010004004050000FC1000400C120020BC
:105110000E12002010B588B000281DDD0A6801219C
:1051200013000B4018D1042A16D90F201468204010
:10513000092811D150683F280EDD980010188068AA
:105140000024084201D04010C4B26846C454013360
:10515000202BF2D1FFF7AAFF002008B010BD0000FD
:1051600010B5002813DD0C68E30710D56410532C2C
:105170000DD8084B1B78002B01D1FFF735FEFFF748
:105180009DFDA123044ADB00D450FFF77DFD0020E4
:1051900010BDC0460D1200200010004010B50028C0
:1051A0000EDD0C68E3070BD56410FF2C08D8054B07
:1051B0001B78002B01D1FFF717FE034A034BD45095
:1051C000002010BD0D12002000100040240500003A
:1051D00013B5002814DD0C68E30711D5094B6410E2
:1051E0000093094B0193072C0AD8084B1B78002B1E
:1051F00001D1FFF7F9FD6B46054A1957054BD15010
:10520000002016BDE2ECF0F4F8FC00040D120020C2
:10521000001000400C05000070B588B0002820DDAB
:105220000124086804401CD104281AD90F230268FD
:105230001340042B15D1FEF783F9060006F0F0FDAC
:105240000500122800D912252A0002210D326846D5
:10525000FFF774FD6B465D73A54205DC6846FFF7FA
:1052600025FF002008B070BD2300325D6B449A73A7
:105270000134F1E7F0B50D008BB0012832DD08688C
:105280000122040014402DD104282BD90F230168DA
:105290000B40042B26D16B68134223D0FEF750F944
:1052A0006E6807007310019306F0BAFD05000E2822
:1052B00000D90E252A000121113202A8FFF73EFD78
:1052C0006A46127902AB5A7302AA73129373019B56
:1052D00076141B0ED67313745574A54205DC02A810
:1052E000FFF7E4FE00200BB0F0BD3A5D02A96318A1
:1052F0009A740134F1E730B589B0002814DD0C68E8
:10530000E30711D5102268460021FFF717FD6B4611
:105310006A4665105D73684663122D0E64149373BC
:10532000D4731574FFF7C2FE002009B030BD000031
:10533000174B184A5968002903D0002159600131E0
:105340009160196900291FD0002018618023DB00BB
:10535000D3581149012B18D1A923DB00D3585B4244
:105360000B600E490B78032B01D801330B7003201F
:105370000B490B78013303400B700A495B015B1842
:10538000094953500123936070470860FAE7C0460B
:10539000FC10004000100040240000209812002063
:1053A0000C1200200E1200200405000010B5034A64
:1053B0001021034800F07EF810BDC04634D800002C
:1053C0002BD80000044A05491368C85401339B05D3
:1053D0009B0D13607047C046C8160020C8120020FD
:1053E00070B5114C114A2368834202DC002323600C
:1053F00016E0155C411C2E00FA3E012E05D899429C
:105400000FDA555C013D1F2D01D90800ECE70100C2
:10541000151A565C6E5401318B42FADC181A206062
:1054200070BD1570FAE7C046D41A0020D4160020CB
:1054300010B5FDF7D3FD064B1A68824201D9002250
:105440001A601B68C31A034898428041404210BD4D
:10545000C4120020204E000010B5094C094A2368F0
:105460001268934200D110BD074AD05CFDF7EAFFF5
:105470000028F8D0236801339B059B0D2360ECE7DF
:10548000CC160020C8160020C812002010B5040059
:10549000064B074A1B6812689B1ADB439B059B0D52
:1054A000A34200DB10BDFFF7D7FFF1E7C8160020CD
:1054B000CC16002070B5074E33680B2B08DC0C258A
:1054C0005D43054C0133285164196160A26033606B
:1054D00070BDC046D0160020342F002010B5FBF759
:1054E00019FEFFF77FF8FBF73DFEFDF73FFFFEF7E4
:1054F000F7FBFEF735FCFFF759FF00F073FF01F0F3
:105500007BF901F0C5FB10BD962210B512010021F8
:10551000034806F0FBF80022024B1A6010BDC0469B
:105520003C1C0020D0050020064B074A1B6812686F
:105530009B1ADB439B059B0D0122834200DC00226A
:1055400010007047C8160020CC160020F8B50500E2
:105550000C0016001F1E0ED10320FFF7E5FF0028E8
:1055600008D0FA20FFF72EFFE8B2FFF72BFFE0B2DA
:10557000FFF728FFF8BD501DFFF7D6FF0028F9D030
:10558000FB20FFF71FFFE8B2FFF71CFFE0B2FFF7B9
:1055900019FFF0B2FFF716FF3012C0B2FFF712FF8B
:1055A0003C00E31B9E42E5DD2078FFF70BFF013452
:1055B000F7E7000070B50024F0250B4B1B68A342F1
:1055C00002DCFFF7A1FF70BD2B006343074A9B1865
:1055D0001A78002A05D05978002311201A00FFF705
:1055E000B5FF0134E9E7C046D00500203C1C00208F
:1055F000F8B507000024F0252B0063430C4A013462
:105600009E18B74211D0317800290BD00133D15CFC
:10561000002311201A00FFF799FF2A000021300013
:1056200006F074F80A2CE7D1F8BD024B1C60F9E7CC
:105630003C1C0020D0050020F0B5150001222F00F1
:105640007A4C1740A54401900291002F11D005AB70
:105650001A706A105A70120E1A7105226912997026
:105660006D140299DD70FFF771FFCF239B009D44FD
:10567000F0BD042D2AD90F2428680440042C32D10F
:10568000022304AA28001371FDF75AFF050006F053
:10569000C7FBC82302009B00984200DD1A007C1C57
:1056A00097420DD1984206D9614804AB0322614963
:1056B000C01806F00FF8220005AB02990198D2E756
:1056C0002700611E695C05ACE155E8E7042D00D0B8
:1056D000A7E0032304AA043D13716B425D4105ABAF
:1056E00055710222E9E7092C7ED1042205AB1A701C
:1056F0006A68511000916946521209789A70009AAE
:1057000059701F2A01DD202200926A46127806ACE9
:10571000DA70009BBB4202DC05ABE21ACDE7012642
:10572000BB00EB189868064006D1042837D90F2132
:105730000368194002290CD10123237043106370C0
:1057400042121B0E4014A270E07023710534013721
:10575000DFE7042921D102232370FDF7F1FE039036
:1057600006F05EFBA31C0C2809D86070864201D1AC
:105770009C19ECE7039A925D9A550136F6E70C22E4
:105780006270039A925D9A550136092EF9D12E2343
:10579000E372237363730E34D9E7012907D103231E
:1057A000043823704342584160700234CFE709291E
:1057B00009D10423237043685A1062705B12A370EE
:1057C000E6700434C3E703290BD105232370006876
:1057D000020992B2430F92000B40D31A63701B125E
:1057E000EDE726700134B2E7032C00D03DE7052237
:1057F00005AB01091A7089B2420F890022408A1A4A
:1058000011125A709970642A00DD64220421DA7042
:10581000081F824201DC04324FE7685C58540131B2
:10582000F6E7002D00D020E753E7C046C4FCFFFF99
:1058300022030000B8CD000070B502000024F02162
:105840000D4E0800604380194578954203D001341D
:105850000A2CF6D170BDF022002105F057FF074A4F
:105860001368013BA34200D11460002329001A00F1
:105870001120FFF76BFEEDE73C1C0020D005002057
:1058800010B5B2B002236A460400137006F0C8FADD
:10589000C72800D9C7200023984207DC421C6B466A
:1058A000FE211420FFF752FE32B010BD69460133CD
:1058B0005A1EA25CCA54EFE730B5B3B002236A4661
:1058C0000500137006F0ACFA0400C72800D9C724FD
:1058D00000239C420BDC20003230FFF7D7FD621C16
:1058E0006B46FF211420FFF731FE33B030BD69460F
:1058F00001335A1EAA5CCA54EBE70000F0B5BBB0F6
:1059000004900C00012803DC1B20FBF701FD51E093
:105910002A4B08680293C30709D4042807D90F2328
:1059200002681340042B02D1FDF70AFE0290234BBC
:1059300060680393C30709D4042807D90F230268BA
:105940001340042B02D1FDF7FBFD039000271C4BF5
:105950001B680693069BBB420BDC039B194A009312
:10596000C821029B08A806F0E3F908A8FFF7A4FFE6
:10597000CAE70C267E43144B0299F618306806F0ED
:1059800045FA051E05D17368B6680793079B9D42CB
:1059900001DB0137DEE730680399059606F036FA39
:1059A0000836002808D121000498059B08310238E8
:1059B0005B6898473BB0F0BD0135E7E740D2000097
:1059C000D016002090D90000342F0020F7B5234BCB
:1059D00006001B68F02100930023009A9A4211DC14
:1059E0000024F0231A006243019201991C4A5518C1
:1059F0002F78002F12D001340A2CF3D11948FFF769
:105A00005BFF29E00A005A43154882185078B042DB
:105A100002D11278002A1FD10133DEE7F0223900CB
:105A2000280005F073FE02230D4A0199EB605354E0
:105A30000D4AF1008A58009B6E70AE70AA602F610B
:105A40006F61A34202DC054B01341C60002331006E
:105A50001A001020FFF77AFDF7BDC046D0050020E0
:105A60003C1C0020D9DD00009C25002010B5FFF76C
:105A7000A1FDFF24084AE3005B429B18074AD35C60
:105A8000043B012B03D8E043C0B2FFF79FFF013C6A
:105A9000002CEFD110BDC046FC0700009C25002063
:105AA000F7B50F00FF247F2501901E4AE300D31AAB
:105AB0001D4A9A181278062A01D0032A20D1FF2203
:105AC000D2009B18186883682B401C2B18D1C36820
:105AD0001A002A40042A13D102692A40192A0FD138
:105AE0001B0A01339B000C30C018FDF729FD037819
:105AF0000600002B10D006F093F90023B84209D01D
:105B0000013C002CD1D1F7BD019AF15CD25C9142ED
:105B1000F6D101339F42F7DCE043C0B2FFF756FFF6
:105B2000EEE7C0469C250020FC07000070B505008C
:105B3000FF24084AE3005B429B18074AD35CAB4250
:105B400003D1E043C0B2FFF741FF013C002CF0D18C
:105B500070BDC046FC0700009C250020F7B5FDF78E
:105B60003DFA574B1A68824201D900221A601A681E
:105B70005449821A8A420DD9FF2253491860D30032
:105B80005248CB1A1B181B78073B022B0CD9013A41
:105B9000002AF4D1F7BD0720FFF7C8FF4C4B27E0E0
:105BA0000820FFF7C3FF38E0FDF722FA071E00D1F7
:105BB00001270020FDF712FB01900020FDF722FBDA
:105BC000019B0090434C444D002B12D02368002BC6
:105BD0006ED12B682760002B6ED0404B01261B78BE
:105BE000002BD8D10920FFF7A1FF394B1E703B4B8A
:105BF0001E70009B002B12D02B68002B0FD1236846
:105C00002F60002B1ED0324B01261B78002BC7D1F2
:105C10000920FFF78BFF2E4B1E70304B1E70236840
:105C2000002B0FD02A4E3278002A0BD19F4200D28F
:105C300027602368FB1A312B04D90720FFF776FF72
:105C4000012333702B68002B0FD0244E3278002AAA
:105C50000BD1BB4200D92F602B68FF1A312F04D91A
:105C60000820FFF763FF012333702368002B0CD05B
:105C7000019B002B09D1164E3378002B02D107204F
:105C8000FFF754FF0023236033702B68002B00D1F3
:105C900080E7009B002B00D07CE7104C2378002B82
:105CA00002D10820FFF742FF00232B60237071E729
:105CB000009A002AA0D1B5E7009B002B9FD1AEE748
:105CC000C01200200F2700009C250020FC070000C8
:105CD000B4120020B0120020B8120020BC12002024
:105CE00037B500240500FFF765FC01A80194FDF716
:105CF00063FA21002000FEF721F9FEF721FBFDF7F2
:105D000095FAFDF70FFBFDF729FBFEF765FCFDF7A4
:105D10008BF9A54204D0FDF7BFFB0248FFF7CCFD8D
:105D200037BDC046CADD0000002310B501001A00CF
:105D30001120FFF70BFC10BD07B56B4619706946C3
:105D40005A7013128B701314120ECB700A716B46BB
:105D5000010005221320FFF7F9FB07BD10B50A006B
:105D600001001220FFF768FC10BD70B505000800A7
:105D70000C003230FFF78AFB2B00220000211B2091
:105D8000FFF7E4FB70BD10B50C00030011001420F8
:105D90002200FFF7DBFB10BD012370B5FF24084A8A
:105DA00041185B42884201D3D84370BD06781D0A72
:105DB000234073409B009B5801306B40F2E7C04684
:105DC000ACD9000013B50400FE2813D80A4BC2005A
:105DD000D05800280ED0436808309900FFF7DCFF48
:105DE00001900920FFF752FB01AB0422210017208C
:105DF000FFF7ACFB13BDC0469C250020F7B5019012
:105E0000FEF79CFD01250400FF276D42002C01D107
:105E10002800FEBD266833143B40152B0DD1210010
:105E20000198083105F0F2FF002801D135123D40FC
:105E30002000FEF777FC0400E8E71D2BF8D10125D0
:105E40006D42F5E7F0B580279FB0FFF705FBB54C35
:105E5000B54D2068FF00391A4019FDF7D9FA2368BB
:105E60000600C3182360002B0ED11FB0F0BD2068C0
:105E7000391A2818FDF7CCFA236806001B1823608E
:105E8000FDF7ACF8A94B1860002EF0DC2B78FA2B4C
:105E900000D00EE12368022B07DCFFF7C9FA0028C7
:105EA000E3D00120FFF79CFADFE76B78AC78981E0F
:105EB000182800D9F2E003F051FA0D2024282B34E1
:105EC000F13E707A7E94CDDEF1F1F1F1F1F1F1F174
:105ED000F1F1EC00FF2C0ED02000FFF7ADFC00220A
:105EE000934BE100CA505B181A7121000092130015
:105EF0001320FEF71FFE0320D4E72000FFF766FD06
:105F0000F9E72000FFF798FCF5E7FFF7AFFDF2E7B0
:105F1000FFF750FB0020FFF7E3FE8648FFF7CCFCBD
:105F2000E9E7632CE7D8844BA200D2582100152062
:105F3000FFF782FBDFE7FEF701FDFF270400002CDF
:105F4000D9D025682B143B40152B04D02000FEF738
:105F5000E9FB0400F3E72000083005F061FF0600CC
:105F60000530FFF793FAFB20FFF72CFA2D121D20C6
:105F7000FFF728FAE8B2FFF725FAF0B2FFF722FAA6
:105F80003012C0B2FFF71EFA25002B1B9E42DDDD4A
:105F9000287AFFF717FA0135F7E700211D20009155
:105FA0000B000A00FEF7C6FDFDF776FAA3E7200016
:105FB000FFF708FF9FE7FDF723F805AC5F4A642170
:105FC00000905F4B200005F0B3FE022320002370F9
:105FD00005F026FF2300020000211620FFF7B6FA85
:105FE00089E70026524AF3009B181C68002C28D031
:105FF0001B790393636808349F00B81D0293FFF771
:1060000045FAFB20FFF7DEF901207D1CFFF7DAF9E6
:10601000F0B2FFF7D7F9E8B22D12FFF7D3F9E8B2E3
:10602000FFF7D0F90398FFF7CDF9E719A7420CD88D
:10603000FFF712FA05230298584301F063FBFFF7BC
:106040000BFA0136FF2ECDD155E72078FFF7BAF9CC
:106050000134EBE70024FFF7ADFA220021000094A1
:106060002300DA20FEF766FDFF222100D20030482F
:1060700005F04CFB98E7012C02D1FEF77DFB3AE7D7
:10608000022C02D1FEF752FD35E70120FFF728FE72
:1060900031E7002321001A001A209FE71A00C83AAE
:1060A000052A00D927E7002218001100FBF766F83F
:1060B00021E7FB2B00D0F4E62268042A00DCECE6A2
:1060C0002E79E8781F4B360206439E4200DDE8E653
:1060D000331D9A4200DCE0E6EB5CFE2B00D0E0E6EC
:1060E0006878AC78771E1B2800D17DE02ED8072871
:1060F00063D0082838D001282DD1FF2C10D02000E3
:10610000FFF79AFB6D79104AB31E009221002A0016
:106110000A20FEF70FFD064BE400E0501B191D712D
:10612000701DBFE6D41A0020D4160020C41200202F
:106130009C250020ACDD0000942D0020C3DD000074
:10614000BEDD0000F6030000DA1600201D285DD039
:106150004FD31E2871D00300C83B052BE0D8404A1E
:106160003900FBF70BF8DBE7632CD9D86A79022AF0
:1061700013D0032A1BD0012AD2D1E979AB790902C5
:1061800019432B7AA4001B0419436B7A1B060B439B
:106190005B001343334AA350C2E7002FC0DDB11E9A
:1061A0003148FDF7EDFB2F4BA400E050B8E7AB7989
:1061B000A4005A1E93419B00ECE7632FB0DC05ADB1
:1061C0003A002749280005F085FA00232800EB55FE
:1061D000FFF714FE0028A3DB224B8000C2582100E9
:1061E0001520FFF729FA9BE739001D48FFF758FCF7
:1061F00096E7FF2C94D06A79022A91D81A490B208D
:1062000000912100B31EFEF795FC89E7632F00DDA6
:106210006327002305A9BB420ADBFB430022DB17EF
:106220003B40CB181A70152000917B1C2100EAE737
:10623000EA185279CA540133EDE7012C00D06FE718
:10624000002F00DC6CE76B79002B03D01C00322B95
:1062500000DD322464235C43044B1C6060E7C046CD
:10626000D9160020942D0020DA160020040000200A
:106270000122094B1A60094A1368002BFCD0032243
:10628000074B1B68D8171040C01801238010063830
:10629000400018437047C04600C0004000C10040A5
:1062A00008C500400120704710B5064C200000F0E2
:1062B0001FFE0549200000F05DFE0122034B1A601D
:1062C00010BDC0460C1B0020801A0600D81A002002
:1062D00010B501210D20FCF799FE01210E20FCF7DD
:1062E00095FE00210F20FCF791FE044C200000F0E9
:1062F00041FD1021200000F059FD10BDEC1A0020D6
:10630000F8B501250C682C4203D10D20FBF700F8ED
:10631000F8BD64102DD4FCF777FEA04229DB0021E4
:106320002000FCF773FEFA222900D200200001F0C1
:106330001BFA00281DD0002500270726FA2201217C
:106340009200200001F010FA002812D0282802DD67
:106350000123B3401F43013EF0D20E4EAF5501352D
:10636000052DE9D1012206210920FDF78BFA00282D
:1063700001D10020CCE70B23012443600023F25C11
:10638000990052004118224301338A60052BF6D14F
:10639000BEE7C046DC1A00200120704710B5046833
:1063A0000D20E30703D56410FF2C03D91720FAF75B
:1063B000AFFF10BDFFF78CFFE1B2024800F018FDFF
:1063C0000020F6E7EC1A002010B5FFF781FF00214E
:1063D000034800F00DFD43000120184310BDC046E6
:1063E000EC1A002010B5034A0A210348FFF762F8AF
:1063F00010BDC046F0DD000040DE00000D4B70B562
:106400001B6804000E001500002B01D1FFF74CFFA4
:10641000E1B2094C200000F044FEF1B2200000F08F
:1064200033FDE9B2200000F02FFD200000F0A4FEB3
:1064300070BDC046D81A00200C1B002010B50124E6
:106440000368234205D04168214202D0826822427B
:1064500003D10D20FAF75CFF10BD5810802801D938
:106460001520F7E74910FF2901D91620F2E752104D
:10647000FF2A01D91720EDE7FFF7C0FF0020EBE767
:10648000F7B501221400904222DD0D682A421FD088
:106490001D4B15411B684C68002B01D1FFF704FF11
:1064A000E9B201272500194E3D40300000F0F9FD0A
:1064B000002D0FD03C413000E1B200F0E5FC30008F
:1064C00000F05AFE0024A04202D02320FAF720FF59
:1064D0002000FEBD042CF2D90F2322681340092BA3
:1064E000EDD163685B100193019BAB42E7DDAB002C
:1064F000E3189968394204D04910C9B2300000F05D
:10650000C3FC0135F0E7C046D81A00200C1B002060
:10651000154B70B51B6805000E00002B01D1FFF76D
:10652000C3FE124CEDB22900200000F0BAFDF1B21A
:10653000200000F0A9FC0021200000F0BDFD002893
:1065400001D0404270BD72B601222900200000F047
:10655000A3FD62B6200000F088FC0028F2D02000E5
:1065600000F088FCEEE7C046D81A00200C1B002083
:1065700010B501240368234202D04168214203D1AF
:106580000D20FAF7C5FE10BD5810802801D915203E
:10659000F7E74910FF2901D91620F2E7FFF7B8FF06
:1065A00040002043EFE7000010B50D211D20FFF74C
:1065B000AFFF164C5A2809D101222A2122703D38FA
:1065C000FFF71CFF0122124B1A6010BD0F2119208A
:1065D000FFF79EFF332805D102235F22237020217D
:1065E0001A38EDE70D211E20FFF792FFC7280AD1C8
:1065F000032300222A21A9382370FFF7FFFE1B2264
:106600002A211E20DCE700232370DBE72C0000207A
:10661000E41A0020204B10B51B680400002B01D1A8
:10662000FFF7C2FF1D4B1B785BB2022B0AD0032B76
:1066300029D0012B2CD121001D200124FFF768FF58
:10664000644205E0012C13D129211920FFF760FFD6
:106650007F2801DD0138FF3803007F3301DA7F2016
:106660004042C8237F21584302F00CFF604310BD15
:10667000032C0BD12B211920FFF74AFF043CE7E73D
:106680002D211920D9E721001E20D6E7052CF7D0AF
:10669000012400206442E4E7E41A00202C000020DA
:1066A00010B50120FFF7B6FF43000120184310BDCD
:1066B00010B50320FFF7AEFF43000120184310BDC3
:1066C00010B50520FFF7A6FF43000120184310BDB9
:1066D000144B70B51B68002B02D10120FFF79AFF05
:1066E000114B1B785BB2013301D1FFF75DFF012035
:1066F000FFF790FF04000320FFF78CFF0500052043
:10670000FFF788FF6D43644340436419201804F089
:10671000C9FE01F09DFB04F08FFE430001201843E9
:1067200070BDC046E41A00202C000020F8B50123FB
:106730001C0098422BDD0F683B4228D04E68350084
:106740001D4024D1042E22D90F2231680A40092A83
:106750001DD173685C10202C00DD2024144B1B68B5
:10676000002B01D1FFF7A0FD72B67F10F9B2114FD7
:106770002200380000F090FC62B6A54214DA38001E
:1067800000F073FB002804D101246D002C4320008D
:10679000F8BD380000F06EFB0122AB004000F3189A
:1067A00010439860AD18E8E764000125EEE7C046A5
:1067B000D81A00200C1B00200020704701207047D1
:1067C000002070470020704701207047002070476C
:1067D000002070470020704700207047002070475D
:1067E000002070470020704700207047002070474D
:1067F000704770477047000010B5034A0E210348E8
:10680000FEF758FE10BDC046A4DE000014DF0000F5
:106810000378013B1F2B00D970470130F8E710B512
:10682000FFF7F6FF0378002B0BD00130222B11D19C
:106830000378002B03D0421C222B03D11000FFF75A
:10684000E7FF10BD5C2B03D14378002B00D0821CE6
:106850001000EDE73A2BF2D02C2BF0D07B2B0BD194
:10686000FFF7D6FF0378002BE9D07D2B01D1013053
:10687000E5E7FFF7D4FFF5E720225B2B14D1FFF704
:10688000C7FF0378002BDAD05D2BF0D0FFF7C7FFEE
:10689000F7E7202BD3DD2C2BD3D0190091435D29B2
:1068A000CFD0222BCDD001300378002BF1D1C6E719
:1068B000002210B5904216D0FFF7AAFF03780422F9
:1068C000222B10D0023A7B2B0DD0013A5B2B0AD041
:1068D000190030390232092905D92D2B05D141780B
:1068E000303909290AD8100010BD0522742BFAD0BE
:1068F0000132662BF7D001326E2BF4D0581E834143
:106900005A42F0E770B5FFF783FF037801222D2B81
:1069100001D18018023A00230A2502E06B430130BE
:10692000CB1801783039CCB2092CF7D95A43100072
:1069300070BDF8B50C001500FFF76AFF0378222B35
:1069400002D000232370F8BD0D236A1E2100082504
:106950000C260A279C4601300378222B02D1002303
:106960000B70F0E7002BFAD0441C5C2B0BD1437862
:10697000841C622B0ED0662B0ED06E2B0ED0722B89
:106980000ED0742B0ED0002AE9DD0B70013A0131D4
:106990002000E1E72B00F6E73300F4E73B00F2E7E5
:1069A0006346F0E70923EEE710B50400FFF737FF71
:1069B000A04202D90378202B00D910BD0138F7E797
:1069C00010B5002815D00378002B13D0FFF720FF57
:1069D0002021037802008B4300205D2B09D010009A
:1069E000FFF71DFF03782C3B5A425341C018FFF7B5
:1069F0000FFF10BD1800FCE70300002070B50C006D
:106A000081420EDD1A785B2A0BD1581CFFF700FF7C
:106A10000125AC4205D0FFF7D3FF002801D0013596
:106A2000F7E770BD70B50C001500002901D00023F8
:106A30000B70002820D00378002B1ED0FFF7E8FE53
:106A4000037806002C2B03D10130FFF7E1FE06008E
:106A5000337800207D2B0FD0844204D02A002100FF
:106A60003000FFF766FF3000FFF7D9FE03783A2BBE
:106A700002D10130FFF7CCFE70BD1800FCE7F0B585
:106A80000D0004009DB02E78002E35D02E21280058
:106A900005F0AEF9071E14D0431B0193303E092EBA
:106AA00014D82800FFF72EFF01002000FFF7A4FFF5
:106AB0000400002C20D0002F1ED0019B0133ED18C4
:106AC000E1E7280005F0ACF90190E7E723787B2B9C
:106AD00011D1601C642203A9FFF7A4FF041E0BD090
:106AE000019A290003A805F0A2F90028E1D02000AE
:106AF000FFF795FEEEE7002420001DB0F0BD70B555
:106B0000050000200C0081421DDD2800FFF7D0FEAB
:106B10000300681C012B14D00020022B13D100228B
:106B2000681C1100FFF77EFF012C0CD0FFF748FF17
:106B300000221100FFF776FF013CF5E7FFF740FF69
:106B4000013C012CFAD170BDF8B5050000200C0005
:106B500016001F0081420DDD2800FFF7A9FE03008B
:106B60000020022B06D1681C3A003100FFF75AFFC3
:106B7000012C00D1F8BDFFF723FF3A003100FFF7E9
:106B800051FF013CF4E710B50024A04218D0FFF7F4
:106B90003FFE03787B2B0AD1013000221100FFF762
:106BA00041FF00280CD0FFF73AFE0134F5E75B2BDC
:106BB00006D10130FFF704FF002801D00134F9E7C6
:106BC000200010BDF8B5002816DD0D68EB0713D5C1
:106BD0006D10013D0124FDF7B1FE0026FF27644240
:106BE00000280CD1002E21D0300005F019F9010049
:106BF0003000FCF7C5FEF8BD01256D42EAE70368E9
:106C00001A143A40152A0BD11B123B409C4200DA61
:106C10001C009D4201D106000836FDF783FDDFE729
:106C20001D2AFAD1012400266442F6E7012001342E
:106C300064002043DFE7000010B508680C00FCF793
:106C40007FFCFFF7DBF8002803DB6268024B800063
:106C5000C250002010BDC046942D002010B5086819
:106C6000FCF76EFCFFF7CAF80123002802DB024B99
:106C70008000C358180010BD942D002010B508687E
:106C8000FCF75EFCFFF7BAF8C043C00F800010BDF0
:106C900010B5034A04210348FEF70CFC10BDC046A2
:106CA000A4DF00009DDF000010B5FCF76BFBFCF7D4
:106CB00019FCFEF713FC0448FEF7FEFDFDF79CFFF0
:106CC000FEF7D4FE10BDC046F3DF000010B5FCF7A0
:106CD0005DF810BD70B5002504AC24780573A94299
:106CE00005D10A4B0A4A23210A4804F085FC0160B9
:106CF0000949920052589B0002715B58A4008371AD
:106D00006358856043710223C37170BD0BE00000BE
:106D10006AE0000019E00000C8E00000037B002BDF
:106D200004D143738373036101330373704700001D
:106D30001FB50191A02100240068C900D2B24450BF
:106D4000012A10D0A24209D0032A0AD0074A835050
:106D5000074B019AC250012343501FBD0222134327
:106D6000F4E70422FBE70622F9E7C04654050000D9
:106D70002405000010B50400FFF7D0FFA12223680E
:106D8000A179D20099506179064A20009950217961
:106D900004329950044B19685A689B68FFF7C8FF82
:106DA00010BDC0460C050000001B00204BB2002B9C
:106DB0000FDB80233F290FD81F290FD80F290FD8A9
:106DC00007290FD803290FD81B060168074A8B50E3
:106DD000704780239B04F8E7DB04F6E71B05F4E724
:106DE0005B05F2E79B05F0E7DB05EEE72405000015
:106DF0000368074A99501A00FC32D1680029FCD078
:106E0000A321C90058580023C0B2D3607047C046C0
:106E10001C05000007B58022074BD2051A6000222E
:106E20009A6002321A710F230C3200930349023B1D
:106E30000348FFF74FFF07BD001B00200030004054
:106E4000EC1A0020F8B505000E0017000024BC4223
:106E500008D02B68315D1B6828009847002801D0B6
:106E60000134F4E72000F8BD704710B51C3000F085
:106E7000BDF910BD10B51C3000F0AAF910BD10B559
:106E80001C3000F0B9F910BD70B5437E0D00002B29
:106E900001D1002070BD6430040000F0B6F9002874
:106EA000F7D12000290000F084F90120F2E700006A
:106EB000F7B50193FA23002504009B0083600B4B78
:106EC0004560083303601C300F00160000F066F9BF
:106ED0002000643000F062F96B461B79276166750B
:106EE0006576A5762000A375FEBDC046A8E000002B
:106EF0000123827DC3751B4B9200F0B5D45820222C
:106F0000210011404D1EA941457DC026AD005D59AF
:106F1000A0272A40531E9A4153421F2214402A4060
:106F20002500B6004942C135FF0531403340FF35E9
:106F30000D4EC919AD006E501100C131FF31DB1982
:106F40008900CE50CC210569084B4904E950052140
:106F50000569243BE95001690833CC500169044BB1
:106F6000CA50F0BDC8E000000C0600002405000077
:106F70000C050000A022002310B50469D200A35024
:106F80000A4CA1420FD90A4C8C425B4109495B4231
:106F90000B40CD21C9045B180469074963500521E2
:106FA0000369995010BDCC235B04F5E7A08601006E
:106FB00090D00300000098FD24050000F7B5040000
:106FC00000200D000193824265D01600402A00D9AE
:106FD000402627001C37380000F0F6F8B12322695C
:106FE000DB00D55080220123216992008B50A27EC4
:106FF000002A03D122691362226913600025731EDF
:10700000AB4207D1019B002B04D0802202212369CF
:1070100092009950012223691A622369FC33DA68CD
:10702000002A02D19A6A002AF9D09A6A002A0BD162
:10703000DA60A3232269DB00D1583800C9B20135D8
:1070400000F0B7F8B542DAD3019B2269002B0FD1CB
:107050001300FC339B6A002B0AD10133A376D36162
:107060002369FC33DA6C002AFCD00022DA640AE0DF
:1070700000230121A37651611A002369FC3399682A
:107080000029FCD09A602369FC339A6A002A01D057
:1070900000229A62E8B2FEBD10B50123FFF78EFF11
:1070A00010BD0300AC3310B504001970643000F05B
:1070B0008BF80123637610BD0023020070B5AC325B
:1070C00043760D001178B12204000069D20081508E
:1070D0008022216992008B50226901331362226958
:1070E000936026006436300000F080F8002812D04B
:1070F000300000F06DF81E4B2269D0502369FC333C
:107100001A6A002A02D19A6A002AF9D09A6A002AD9
:1071100001D11A62E5E723690122002D0DD1190082
:10712000FC31896A002908D1DA612369FC33DA6C01
:10713000002AFCD00022DA6407E05A612369FC339C
:107140009A68002AFCD000229A6000202369FC3350
:107150009A6A82420BD098622169064A8B588B50FA
:107160001800022B03D0181F431E9841033070BD36
:107170001C050000C404000010B50121FFF79CFFAE
:1071800010BD000010B51323142202490248FFF776
:107190008FFE10BD004000400C1B002010B54022A7
:1071A0000021040004F0B2FA002320002364636489
:1071B00010BD10B53F24026C531C2340446C9C420C
:1071C00001D08154036410BD0023036443647047FD
:1071D000436C026C934206D03F21C25C01330B40EA
:1071E00043641000704701204042FBE7036C406C91
:1071F000181A00D540307047436C026C934201D09E
:10720000C05C704701204042FBE73F22036C406CAA
:1072100001331340181A43425841C0B2704700006E
:1072200003210A4802680A430260094802680A43C7
:1072300002600849084A094B9B1A03DD043BC85801
:10724000D050FBDC00F012F8F8F75EFF2405004098
:10725000540500401CE600000000002068020020E9
:10726000FEE7FEE7FEE7FEE7FEE7FEE72D4B10B583
:107270001A68D2B2012A0FD12B4A126812070BD119
:107280002A4AE0241168F0220800104021422DD142
:107290002749096811422CD01A68D2B2012A12D1AA
:1072A0002149096809070ED1F020204909680140E9
:1072B000402908D11E490968014204D18020C1211A
:1072C000C005C90042501B68DBB2012B0DD1164B23
:1072D0001B681B0709D1154B1A68F0231A40A02A16
:1072E0000FD1134A12681A420ED010BD3028CFD0E9
:1072F000D2E7104A104911608021104A090211603A
:10730000CAE7D02AF1D1ECE70D4B1A68012A04D064
:107310000C4A1A601A68012AFCD1C0220A4B1A6072
:10732000E3E7C046E00F00F0E40F00F0E80F00F0E4
:10733000EC0F00F004050040DFFF07C0186C0040B0
:1073400000EC06407593000014EC064001207047E5
:1073500010B503681322DB69984710BD7047000021
:10736000054B0269D1500369FC331A6A002AFCD02C
:10737000002201201A6270471C050000030010B5AE
:107380005C331A781F231A401E3B19009140114AA2
:10739000D167C222042104699200A150026953609E
:1073A0000269D360A02300220169DB00CA500123D7
:1073B0000169094A5B428B500169084A8B50016997
:1073C0000C3A8B50016908328B501430FFF7FCFEE9
:1073D00010BDC04604E100E00C05000014050000EB
:1073E00010B51430FFF702FF10BD10B51430FFF7D1
:1073F00003FF10BD10B51430FFF7EAFE10BD00000A
:10740000030070B55E331A780469724BE2500300D2
:107410005D331A780469704BE250030061331C78C5
:1074200002696E4B012C00D09EE005005F352E787E
:10743000A225ED005651020060321578A12206699E
:10744000D200B5500269D4509623DB00994200D88F
:107450008CE096231B01994200D88AE096235B01B9
:10746000994200D888E096239B01994200D885E094
:10747000E1239B01994200D882E09623DB019942E7
:1074800000D880E0E123DB01994200D87DE096231B
:107490001B02994200D87AE0E1231B02994200D8EE
:1074A00077E096235B02994200D874E0E1235B0207
:1074B000994200D871E0E1239B02994200D86EE026
:1074C000474B994200D86CE0E123DB02994200D897
:1074D0006AE0E122002312038A425B41414A5B4297
:1074E0001340802252059B1801693F4A8B50A0230C
:1074F00004220169DB00CA5000210369FC33D96012
:107500000369FC331962012301690B6001698B6017
:10751000C1210469890062501F215C3002780A4051
:1075200093406231314AFF315350002141560029C6
:107530003CDA0F230B40083B2D4C9B089B001B198A
:1075400003242140A140FC348C40DD69A5432C007C
:10755000C0258D4029002143D9611F23017819409E
:107560001E3B8B40136070BD00246CE79E23DB0242
:10757000BAE79D231B03B7E71E4BB5E71E4BB3E7E6
:10758000EC239B03B0E71D4BAEE71D4BACE71D4B57
:10759000AAE71D4BA8E71D4BA6E71D4BA4E71D4B13
:1075A000A2E78023DB049FE71B4B9DE78C080F4B72
:1075B000A400E41803230B40FF21C025DB00994001
:1075C000AD0066598E433100C0269E4033000B4308
:1075D0006351C2E70C050000140500006C050000B3
:1075E00090D0030000D0BEFE2405000000E100E0C2
:1075F00000ED00E000B013000050270000A04E0096
:1076000000F0750000509D0000F0EB0000903A0182
:1076100000E0D70100B0AF0300705F07F7B500933B
:1076200008AB1B7800250193FA2304009B008360BC
:107630000E4B45600833036014300F001600FFF74F
:10764000ADFD23005C3327611E70009B084A9B0040
:10765000995823005D331970019B20009B009A58B4
:1076600023005E33DD701A70FEBDC0464CE10000A1
:10767000C8E00000036910B51A00FC32D2680400AB
:10768000002A0AD0A322D20099581430C9B2FFF7B9
:1076900090FD00222369FC33DA6010BD10B502486A
:1076A000FFF7E8FF10BDC046C41B0020162307B536
:1076B000022200930249013B0248FFF7AFFF07BDDA
:1076C00000200040C41B002010B5002801D004F0A9
:1076D000D9FA10BD0849094A094B10B51B688858EA
:1076E000FA22190A1B0618439200002302F002F83E
:1076F0004904C00B084310BD001001400405000000
:10770000281C002070B5041E09D0FFF7E3FF050018
:1077100000F014F8FFF7DEFF401BA042F8D370BD65
:107720000022044B9A60044A13680133DBB21360F1
:107730007047C046FC100140281C0020704770476D
:1077400010B500F061F8FFF7FAFF0120FFF7DAFF4C
:10775000FFF7AAFAFFF7BAFA024B002BFAD000E0C3
:1077600000BFF7E700000000F8B516004C1EA1416D
:107770001F220125104B8000104FC3584C4213406C
:1077800038680F499D4001F0F3FD0A21704301F074
:10779000EFFD2C400300220029000A4800F016F8F3
:1077A000FA21094C89004443386801F0E1FD0100E9
:1077B000200001F0DDFDF8BDC8E000003000002031
:1077C00040420F00100500501027000030B504683B
:1077D0000C40944206D1013B002BF8D112E0013B52
:1077E000002B0FD004680C409442F8D100240568A7
:1077F0000D40954204D101349C42F8D1002002E0B2
:10780000201C00E0181C30BDC420114B80001A5809
:1078100010491140C02212020A431A50C02180228E
:10782000490092025A501A608023A3220021DB05EE
:10783000D20099500122F9309A60074BFF3019505D
:10784000C120023180001950403019501A60704731
:1078500000E100E0FF00FFFF00100140014B186055
:107860007047C0467C000020F7B5002320285AD876
:10787000384B8000C258042A5BD007D8022A54D063
:1078800055D80423012A09D000234CE0062A54D0FD
:1078900051D31A2A53D002231B2AF5D12E4A11683C
:1078A00008294ED909294FD00A240226A0200125F3
:1078B0002A4AC00015502A482A4D07681C20BF00DC
:1078C00007402948019700685759009027481B0234
:1078D00007401F43C02300989B020340FF205751DD
:1078E0005759000207401F43019B1F43009B58014B
:1078F0006023184007433E43565101251C4B156039
:1079000058680028FCD000205860A1230125DB0026
:10791000D3585560A025ED0050511BB2A14202D0B2
:1079200015D2611ACB401800FEBD0823B6E710231C
:10793000B4E72023B2E74023B0E78023AEE701237A
:10794000ACE708240026B1E70C000126AEE7091BCE
:107950008B40E8E7C8E0000078000020007000409D
:10796000340000200405000038000020FF00FFFF65
:10797000FC700040F0B520285BD8364B8000C25820
:10798000354B1E68002E30D1C227344BBF00D8596A
:10799000334C03250440C02000022043D851C024AA
:1079A00080206400800018512E4F18602E4B803CC0
:1079B000D859FF3CA043D8510437D859A843204395
:1079C000D8510837D8590C35A84384460720654656
:1079D0002843D851A820C0001E50C1208026800016
:1079E00076021E501C601C4B1C60142500202B00CE
:1079F0001E4C2E0046433659771C1BD14343E250A0
:107A0000A0230325C132FF329200DB05D550184B6D
:107A10001A68082A14D114234343E3189A681248B9
:107A20005132FF32920059601150DA68C1239B0035
:107A3000C250F0BD9642E1D001300328D9D1F8E719
:107A4000082A02D9083AD140E5E708239A1A91405A
:107A5000E1E7C046C8E000002C1C002000E100E087
:107A6000FF00FFFF04050000009000403C000020E4
:107A70007C0000202149F0B54A6C2148002A14D02E
:107A8000A025A12600230124ED05F600C258571CAD
:107A900006D0C7187F68002F02D027009740AF514B
:107AA00014333C2BF2D100234B64A0230121DB05CE
:107AB00000260F009C4614234B43C3181A1F12685C
:107AC000104C0E4D920014195219526C002A10D00D
:107AD0001A00143A1268551C09D0103B1B68FF2B82
:107AE00005D03B00934065461A00074BEA50FC3432
:107AF000666401310429DED1F0BDC046FC9000402F
:107B00003C000020009000400C05000000B520283B
:107B100018D8104A80008358C0209A068000D217D7
:107B20000240A020C00512181F200340032909D8D5
:107B30000800C133FF339B0001F010FC0209050768
:107B40000021995000BD0C21FBE70421F9E7032136
:107B5000F7E7C046C8E00000202812D80B4B800091
:107B6000C258C02093068000DB170340A020C00548
:107B70001B181F20104001228240002902D1044915
:107B80005A507047A121C900FAE7C046C8E000007A
:107B90000C05000003000020202B12D8C021094A48
:107BA0009B009A5889009306DB170B40A021C9055A
:107BB0005B18A221C90058581F231A40D0401E3B11
:107BC00018407047C8E00000F7B506000D000C0033
:107BD0008B180193019B671B9C4207D03368217867
:107BE0001B683000984701340028F3D13800FEBDEF
:107BF000F0B5C64600B5CB0F9846404A4B005B0D2A
:107C00009A1882B00D000400132A2FDC002A49DBE9
:107C10003B4F17413E000E40064323D07F083900FA
:107C200029400C430AD03749BD438C4663445C422B
:107C30005C418023DB021341E4071D434146CE0033
:107C400031492B008E192200346875682000290004
:107C500001F0F6FE009001910098019922002B009E
:107C600003F086F802B004BC9046F0BD332A08DD6C
:107C70008023DB009A42F5D102000B0001F0E0FE08
:107C8000F0E7224A9446012263445242DA4002421B
:107C9000E8D052080242D1D094438022D2051A4142
:107CA0001443CBE74B005B080343DBD00B031B0BF8
:107CB0001C436342234380244D0C24031B0B2340AD
:107CC0006D042B4319004346DA000F4B9B181C68C8
:107CD0005D6802000B002000290001F0B1FE009059
:107CE00001910098019922002B0003F041F84246CF
:107CF0004B005B08D60733431900B3E701FCFFFFD5
:107D0000FFFF0F00EEFBFFFF80E10000EDFBFFFF38
:107D1000F8B5274A4B005B0D9A180C000700132A90
:107D200010DC002A36DB234B13410B423AD080246F
:107D300024031441002064189C43060025003000F1
:107D40002900F8BD332A0EDD80230600DB000D007C
:107D50009A42F4D102000B003800210001F070FEBD
:107D600006000D00EBE7144D0600AC460125634408
:107D70006D42DD40AC4663460D000342DFD0332345
:107D80009A1A323B93401818874200D94C1C63461C
:107D90009843D2E7C90FCC070020531CCDD1074B25
:107DA0001C43CAE706000D000028C0D1C7E7C04643
:107DB00001FCFFFFFFFF0F00EDFBFFFF0000F03FA6
:107DC00030B5214A4B0087B05B0893421EDD1F4A45
:107DD000934205DD02000B0002F0CAFF07B030BD80
:107DE00002AA00F095F803231840049A059B012885
:107DF00013D002281DD0002814D00298039900F057
:107E00006FFB80231B069C466144E7E700230022AA
:107E10000093002301F0DEF8E0E70298039900F0F8
:107E20005FFBDBE7012402980399009401F0D2F88C
:107E3000D4E7012402980399009401F0CBF8802341
:107E40001B069C466144C9E7FB21E93FFFFFEF7F2A
:107E5000F0B54746CE4680B58DB004000D0000F069
:107E600067FA294B06001B780F005BB29846013376
:107E700010D022002B002000290003F0C1FA814617
:107E8000002807D1002200232000290001F00AFC6D
:107E9000002806D1300039000DB00CBC9046994640
:107EA000F0BD01230293194B0694079503934B46AB
:107EB0000A93434604940595002B15D00023002215
:107EC0001900100002F0D8F8434608900991022BDF
:107ED0000ED103F0AFFB212303600A9B0193002B1B
:107EE0000CD1089E099FD5E700230024089309942C
:107EF00002A801F0C1F90028EFD1EAE703F09AFBEC
:107F00000A9B01930360ECE78000002090E10000F1
:107F1000F0B54E464546DE465746E0B5E14B4C00CF
:107F20008FB09046894664089C4200DC87E0DE4BB7
:107F30009C4222DCDD4A002900DC92E0DC4B02F0AE
:107F400017FFDB4B06000F009C4200D17EE1D94AAF
:107F5000D94B02F00DFF02000B00414630000A60D1
:107F60004B60390002F004FFD34BD24A02F000FF0D
:107F7000434601259860D9606BE0D04B9C4200DC01
:107F80008FE0CF4B9C4200DD55E1CE4A231592464F
:107F90009A4451460905631A19001D00040003F0B4
:107FA0004BFA03F07FFA02000B0020002900089230
:107FB000099302F0DDFE0022C34B02F067FC0F00C4
:107FC000060003F039FA03F06DFA04000D00020018
:107FD0000B00300039000A940B9502F0C9FE002214
:107FE000B94B02F053FC002200230C900D9101F0DC
:107FF00053FB002800D192E1002300222000290039
:1080000001F04AFB434243410133B04A41460192E9
:10801000022208A80092524600F07CFB4B46050065
:10802000002B16DA802243461206944642465B68CD
:10803000454263445360D3686344D36009E00B0056
:10804000020041460A604B600022002300258A603E
:10805000CB6028000FB03CBC90469946A246AB4688
:10806000F0BD934B01F0ECFC914B06000F009C42DD
:1080700000D13DE18F4A904B01F0E2FC02000B0081
:10808000414630000A604B60390002F071FE894AB7
:10809000894B01F0D5FC012543466D429860D960BB
:1080A000D7E701F049F88A4A8A4B06000F0002F030
:1080B000EDFB0022884B01F0C3FC03F0BDF9050085
:1080C00003F0F0F9794A7A4B0490059102F0DEFB57
:1080D00002000B003000390002F04AFE754A06002B
:1080E0000F0004980599744B02F0D0FB02900391A5
:1080F0001F2D00DCC7E0029A039B3000390002F01C
:1081000037FE83468A4653465B0024155B0DE31A0F
:10811000102B6CDD04980599D322674B520502F0B1
:10812000B5FB02000B00300039000292039302F00D
:108130001FFE0A0001001300069107920200390099
:10814000300002F015FE029A039B02F011FE0600B9
:108150000F0004980599614A614B02F097FB3200C9
:108160003B0002F005FE069E079F0B00020039004F
:1081700030000292039302F0FBFD4B005B0D83463F
:108180008A46E41A312C32DD04980599B822544B02
:10819000920502F07BFB03000C00020002930394A3
:1081A0000B000698079902F0E3FD02000B000600A1
:1081B0000F000698079902F0DBFD029A039B02F07C
:1081C000D7FD484A0290039104980599464B02F066
:1081D0005DFB029A039B02F0CBFD02000B00300016
:1081E00039000292039302F0C3FD83468A465A4641
:1081F0005346414630000A604B60390002F0B8FD3A
:10820000029A039B02F0B4FD44460B000200A260F8
:10821000E3604B46002B00DB1BE75B4623608023BB
:108220001B065344636080231B069C466144A06088
:10823000E1606D420DE70B00020002F099FD43463C
:1082400000259860D9601860596002E7D3221A4B64
:10825000520502F08DFD214A214B0D00040002F071
:1082600087FD02000B00414620000A604B60290098
:1082700002F07EFD1A4B194A02F07AFD43460125B1
:108280009860D960E5E602000B003000390002F08A
:108290006FFD6B1E154A9B009B5883468A46A3427E
:1082A000A5D130E7FB21E93F7BD9024000004054D3
:1082B000FB21F93F3163621A61B4D03DFB213941A2
:1082C000FFFFEF7FEAFBFFFF0000704118E20000B4
:1082D00083C8C96D305FE43F0000E03F7370032E38
:1082E0008A19A33BC14920259A837B3998E1000074
:1082F000D3220C4B520501F0A3FB0B4A0B4B04009D
:108300000D0001F09DFB02000B00414620000A60B9
:108310004B60290002F02CFD034A044BB9E603230D
:1083200073E6C04661B4D03D7370032E8A19A33B37
:10833000F8B54746CE46674B80B50A000F001900D6
:1083400005003940994200D19BE004000100002F54
:1083500069DD3F1500D1B4E05F4B12039C468023DA
:10836000120B5B0313435B00CA0F67449B184A0060
:10837000F80703D5D20F5B009B188A0079108C4652
:10838000002180201624894680030D189D4202DCBE
:1083900029185B1B8144D50F5B00013C5B1952001F
:1083A0004008002CF1D100208046802020250027A5
:1083B000000609E08B425CD0D40F5B00013DE3185E
:1083C00052004008002D16D0C4198B42F2DD271848
:1083D0000E00002C49DB5B1AA242894149425B1A1C
:1083E000121BD40F5B00013D80443100E3185200A2
:1083F0004008002DE8D113434ED143465B0837496E
:108400004A468846494652104244C90702D580214F
:1084100009060B4361460F05BD18180029000CBC66
:1084200090469946F8BD7B005B0803433900002B5A
:10843000F5D0002F3CD1E30A153A6405002BFAD0A1
:108440008020400303423FD1002700E00F005B0083
:10845000791C0342FAD0250020208D40401A2900C3
:10846000D71B2200C2401A4376E7FE43F60F8E194F
:10847000B1E79442A0D82718002CF6DB1E00002399
:10848000AEE702003B002800390002F0FFF92A00A5
:108490003B0001F0D5FAC2E74346013303D043461F
:1084A00001335B08ABE7012398460023C144A6E7EC
:1084B0003B00020002F05CFC02000B0001F0DCFD5E
:1084C000ADE713000022BBE70127210020207F42F7
:1084D000C6E7C0460000F07F01FCFFFF0000E03F60
:1084E000F0B54746CE4680B587B000920193754BF4
:1084F0004F00814688467F089F4263DC02F09CFF64
:10850000002800D1D4E04A4643464846414602F09E
:10851000BDF904000D006C4A6C4B02F0B7F96C4ACF
:108520006C4B01F08DFA22002B0002F0AFF96A4A81
:108530006A4B02F01DFC22002B0002F0A7F9684AEA
:10854000684B01F07DFA22002B0002F09FF9664A89
:10855000664B02F00DFC22002B0002F097F9644AF2
:10856000644B01F06DFA22002B0002F08FF90290AB
:1085700003910022604B2000290002F087F9029A43
:10858000039B06000F002000290002F07FF9009AEB
:10859000019B04000D004846414602F077F90200B5
:1085A0000B002000290002F0E3FB02000B0030006A
:1085B000390002F0DDFB02000B0000204F4902F001
:1085C000D7FB70E002000B0002F060F904000D0020
:1085D0003D4A3E4B02F05AF93D4A3E4B01F030FA1B
:1085E00022002B0002F052F93B4A3C4B02F0C0FB48
:1085F00022002B0002F04AF9394A3A4B01F020FAE6
:1086000022002B0002F042F9374A384B02F0B0FB4F
:1086100022002B0002F03AF9354A364B01F010FAED
:108620002B00220002F032F9354B029003919F4259
:108630009FDD344B00229F423DDC334900207B18F4
:108640002E4916001F0002F093FB049005910022B2
:10865000294B2000290002F019F932003B0002F0FA
:1086600087FB029A039B06000F002000290002F0FE
:108670000DF9009A019B04000D004846414602F0A6
:1086800005F902000B002000290002F071FB020036
:108690000B003000390002F06BFB02000B00049865
:1086A000059902F065FB07B00CBC90469946F0BDF9
:1086B00000201249F7E7154B002604920593144F4A
:1086C000C5E7C046FFFF3F3ED43888BEE9FAA8BDE3
:1086D000C4B1B4BD9EEE213EAD529C804F7E923E11
:1086E0009015CB19A001FA3E7751C1166CC1563FC7
:1086F0004C5555555555A53F0000E03F0000F03F53
:108700003233D33F0000E93F0000E0FF0000E73FC5
:108710000000D23FF0B5DE464E4645465746E0B52E
:10872000DC4CA5440D9114001900A49A0993DA4B6E
:108730009200D6584D1E03901821E01E0696029511
:1087400000F0A0FEC3430100DB1719404B1C9A0048
:108750009B1ADB001B190B9105934C1B771918D43E
:10876000A59BA5009C463F1922AE6544013707E052
:10877000286802F097FE013403C60435BC4208D0D5
:10878000002CF5DA00200021013403C60435BC4278
:10879000F6D1069B002B01DA00F0FDFB069B039946
:1087A0000133DB009A46099BDA00944600920022CE
:1087B000914672AA0492B94A6144934688469AAB9C
:1087C00063449B44029B002B00DABCE15D4600261B
:1087D0000027039C4D442A686B6803CC02F056F8CE
:1087E00002000B003000390001F02AF9083D0600B4
:1087F0000F004445EFD1049B4B441E605F6008238B
:108800009C46E144D145DDD10EA80421844649426D
:1088100061448C46069A93009C44614684460A91C2
:108820000399083B63448C460C93009B009263447D
:108830009B46009A0498D10003008C46634408913B
:108840001E685F68002A33DD954980468C46624485
:10885000D300984470AB9A460EAB99460022914BD8
:108860003000390002F012F802F0E6FD02F01AFEC4
:1088700000228D4B04000D0002F008F802000B00EE
:108880003000390002F074FA02F0D6FD4B4601C305
:108890009946434620001A685B68290001F0D0F829
:1088A00008235B429C46E04406000F00D045D5D12A
:1088B000059B30001A003900984600F0DFFCFF23CA
:1088C00000229B0504000D0001F0E0FF00F038FCE1
:1088D0000022764B01F0DAFF02000B002000290095
:1088E00002F046FA0D00040002F0A6FD814602F0F7
:1088F000D9FD02000B002000290002F039FA060021
:1089000040460F00002800DCEEE0009B18215A1EB4
:1089100092000EAB9B58091A1D000D41A9448D40D1
:108920005D1B0EAB9D5017231B1A1D41002D2DDD25
:1089300001239C46009BE144002B00DC1CE20E9CC2
:108940000123002C00D0B5E0009A012A09D099003B
:108950000EAA54580133002C00D0ACE0009A9A4281
:10896000F5D1059B002B0EDD012B00D1A8E1022BD8
:1089700009D1009B0EA95A1E92000EAB9B5807937B
:108980009B029B0A8B50022D00D1C1E000230022E4
:108990003000390000F080FE009B002800D194E2F6
:1089A000069A591E8A4210DC414A0A9894460EAA39
:1089B0006344944600229B0063441C68043B2243AA
:1089C0008342FAD1002A00D0C0E0069B0EAA013BE8
:1089D0009B00D358002B00D0B3E001220C9B043B3A
:1089E000596801320029FAD0009B9C46624411006C
:1089F00007921A0001338B4246DC0B98634680468F
:108A0000A59C4344A046099C9B00A1464A44984427
:108A1000D30022AA9146049A99449446089BA59AA9
:108A200063448446614494469A468B0063440093B1
:108A30004346586802F036FD4B4618605960029B69
:108A4000002B24DB4D46039C0026002701E028680C
:108A500069680CCC01F01AFF02000B0030003900ED
:108A600000F0EEFF083D06000F005C45EFD15346D5
:108A70009E60DF6004239C460433E0449C46009BD8
:108A8000E144E2449845D3D1079B0093D1E6002608
:108A90000027ECE794FDFFFF60E3000018FEFFFFF6
:108AA000FFFFFF1F0000703E0000704100002040EB
:108AB000FFFFFF3F002180225204141B0EAA5450D6
:108AC000009999420EDD0EA884469B000EAA8900EB
:108AD000D25861446344CF4800E01A68821A04C344
:108AE0008B42FAD101243CE7059B002B06D1009B69
:108AF0000EAA013B9B00D558ED1517E70022C64B87
:108B0000300000F0EDFD002800D024E100253DE715
:108B100032003B000020C14902F02AF906000F0094
:108B2000002C00D132E7059A0020BC4900F0A6FBDA
:108B300002000B003000390002F01AF906000F00A5
:108B400024E7012250E70026002754E64B46059A09
:108B5000079388468B000EA9CB58183A08950592C2
:108B6000002B0DD18C464146AD4B43449B006344E2
:108B7000043B58680139183A0028F9D08846059214
:108B8000059A0020A54900F079FB434604000D003A
:108B9000002B00DA05E29E000EAB9C464346DB004C
:108BA00066449C46059370AB9946049F67440097C2
:108BB000306802F077FC22002B0001F067FE0022F3
:108BC00038607960974B2000290001F05FFE083F74
:108BD00004000D00043EB945EAD14AAB03939B461D
:108BE00000239A46069B424699464346013202922A
:108BF00004934B46002B00DAAAE080208A4B009DAC
:108C00009846C005894900260027002408E008236B
:108C10009C460835E044544511DC434618685968C1
:108C20002A686B6801F032FE02000B003000390048
:108C300000F006FF013406000F00A145E7DA5B46AD
:108C4000C0C39B4601239C46009BE244083B009323
:108C5000029B9A45CDD1049B9846A49B022B00DD34
:108C60008EE0002B37DC1FD1059B00271D00039BE6
:108C700000249C461E006544083E2A686B68380044
:108C8000210000F0DDFE083D07000C00AE42F4D1EB
:108C9000089B002B03D080231B069C4664443A00AB
:108CA00023000D990A604B600720079B18409B2307
:108CB0009B009D443CBC90469946A246AB46F0BD05
:108CC000009B0EA95A1E92000EAB9B5807935B02A5
:108CD0005B0A8B5057E64346002B00DA70E1002018
:108CE0000021DB004AAAD61848AF32687368083EF4
:108CF00000F0A6FEB742F8D1089B002B00D025E17A
:108D00000B0002004A984B990D9C2260636002F0B0
:108D10002FF8434607000C00002B13DD01254CAE55
:108D2000B14638002E0021004C4601360CCC00F034
:108D300087FEA146B045F7DA089B07000C00002B20
:108D400000D015E13A0023000D998A60CB60ABE7B3
:108D50000026002773E701239C46009BE14402257F
:108D6000002B00DDEBE532003B0000202B4901F039
:108D7000FFFF06000F0009E60024F2E54AAB03936B
:108D8000A49B032B00D08FE74346002B00DC14E1AB
:108D9000039ADB009B46130091465B441E685F68A4
:108DA000234B43440293DB00994448AB9A464B461D
:108DB0005C681B681800210032003B0000900191A4
:108DC00000F03EFE04000D0002000B000098019927
:108DD00001F0CEFF3B00320000F032FE4B469860BF
:108DE000D9601C605D6008235B429C46E14426001C
:108DF0002F00CA45DBD14346012B00DCE3E0039A98
:108E000013005B441E685F68029BDB0099464A447E
:108E1000904610E0FFFFFF000000E03F0000F03F41
:108E2000FFFFFF3F0000703E20E30000FB21F93F01
:108E3000FFFFFF1F984643465C681B68180021002F
:108E400032003B000090019100F0FAFD04000D009B
:108E500002000B000098019901F08AFF32003B00EC
:108E600000F0EEFD4346039A9860D9601C605D6097
:108E7000083B26002F009A42DCD14D46944600263E
:108E800000244746083565442A686B683000210095
:108E900000F0D6FD083D06000C00AF42F4D1039B64
:108EA0004A9F5D689968D868089B002B65D080222E
:108EB000120694460D9B6544604464441F605D60E7
:108EC0009960D8601E615C61EEE69A464B46079356
:108ED000059B30005A423900089500F0CFF9002276
:108EE0003A4B06000F0000F0FBFB002824D0384B63
:108EF00000223000390001F0C9FC02F09DFA524610
:108F00000400950002F0CEFA0022304B01F0BEFCC6
:108F100002000B003000390001F02AFF02F08CFA49
:108F20000EAA50510122059B5244183390460593D6
:108F300093000EAAD45023E65346300039009C001B
:108F400002F07AFA0EAB1851D04619E680230D9A3A
:108F50001B06CB18106053600B0002004A984B9917
:108F600001F006FF434607000C00002B00DDD5E6AC
:108F700080231B069C466444E4E62B003A000D9DCA
:108F80002A606B600A000300AA60EB6032002300D5
:108F90002A616B6188E6099BDB00009372AB049346
:108FA00032E4A49B022B00DDE8E6002B00DD92E614
:108FB00000D079E6002700246AE6002600246EE748
:108FC0000020002198E60026340068E70000704188
:108FD0000000703EF0B5CE46474680B587B000929F
:108FE0000193474A4B00814688465B08934207DC61
:108FF0004146484602F020FA4146031E484666D0E4
:109000004A4643464846414601F040FC04000D00F4
:1090100002000B004846414601F038FC394A3A4B01
:1090200006000F002000290001F030FC374A384BC1
:1090300001F09EFE22002B0001F028FC354A364B41
:1090400000F0FEFC22002B0001F020FC334A344BE0
:1090500001F08EFE22002B0001F018FC314B324A49
:1090600000F0EEFC0E9B02900391002B34D0009890
:10907000019900222D4B01F009FC029A039B0490F8
:1090800005913000390001F001FC02000B0004984A
:10909000059901F06DFE22002B0001F0F7FB009A0C
:1090A000019B01F065FE224A04000D00214B3000B7
:1090B000390001F0EBFB02000B002000290000F05A
:1090C000BFFC02000B004846414601F051FE07B0CC
:1090D0000CBC90469946F0BD02000B002000290010
:1090E00001F0D4FB124A134B01F042FE32003B0068
:1090F00001F0CCFB4A46434600F0A2FCE7E7C0463D
:10910000FFFF3F3E7CD5CF5A3AD9E53DEB9C2B8AF9
:10911000E6E55A3E7DFEB157E31DC73ED561C11954
:10912000A0012A3F1111813FA6F810110000E03F75
:10913000495555555555C53F49004B0819007047CD
:10914000474AF0B54F4691464B005B0D9944464661
:10915000D6464A46C0B505000C000E0088460700FA
:10916000132A27DC002A4BDB3E4B13419A460B00A7
:1091700052461340034318D03B4A3C4B2800210081
:1091800000F05EFC0022002300F0A0FA002847D087
:10919000002C04DA80234A465B0313419844464678
:1091A000534600279E43380031001CBC9046994628
:1091B000A246F0BD332A08DD8023DB009945F4D1B7
:1091C00002000B0000F03CFCEFE7294A9446012224
:1091D00063445242DA4092460242E6D0224A234B8E
:1091E0002800210000F02CFC0022002300F06EFA81
:1091F000002815D0002C1EDB534646469F430FE047
:10920000194A1A4B2800210000F01AFC0022002302
:1092100000F05CFA002803D0002C04DB00270026B5
:1092200038003100C1E76400640825430027002DA1
:10923000F6D0104EF4E74B46142B0BD03422D21A42
:10924000012393405D19BD4208D201239C462F00A3
:10925000E044D1E7133B9C46E044CDE72F00CBE749
:1092600001FCFFFFFFFF0F009C7500883CE4377E88
:10927000EDFBFFFF0000F0BF002070474B0070B512
:109280005B0D14000A00002B1AD14B005B0803434E
:1092900015D0234B002201F0F9FA224B9C422DDB22
:1092A0000A004B005B0D363B1F4DE318AB422ADC36
:1092B000002B0DDD1D4C1B0522401A43110070BD13
:1092C0001B4DAB42F0D102000B0000F0B9FBF6E7FA
:1092D0001D00353519DA174B02009C4209DD0B00E1
:1092E0001548164900F032F8134A144B01F0CEFA33
:1092F000E5E70B001248134900F028F8104A114B1B
:1093000001F0C4FADBE70200E9E7084C36332240FB
:109310001B051343190000220B4B01F0B7FACEE7EF
:1093200000005043B03CFFFFFE070000FFFF0F802E
:10933000FF07000050C300009C7500883CE4377EA6
:1093400059F3F8C21F6EA5010000903C30B54A00E9
:10935000DB0FDB0752081A43110030BD02B471461F
:1093600049084900095C49008E4402BC7047C04668
:10937000002243088B4274D303098B425FD3030A54
:109380008B4244D3030B8B4228D3030C8B420DD367
:10939000FF22090212BA030C8B4202D312120902F5
:1093A00065D0030B8B4219D300E0090AC30B8B4233
:1093B00001D3CB03C01A5241830B8B4201D38B03E1
:1093C000C01A5241430B8B4201D34B03C01A524186
:1093D000030B8B4201D30B03C01A5241C30A8B42C9
:1093E00001D3CB02C01A5241830A8B4201D38B02B4
:1093F000C01A5241430A8B4201D34B02C01A524158
:10940000030A8B4201D30B02C01A5241CDD2C309C9
:109410008B4201D3CB01C01A524183098B4201D345
:109420008B01C01A524143098B4201D34B01C01A30
:10943000524103098B4201D30B01C01A5241C308A8
:109440008B4201D3CB00C01A524183088B4201D317
:109450008B00C01A524143088B4201D34B00C01A03
:109460005241411A00D20146524110467047FFE76F
:1094700001B5002000F0F0F802BDC0460029F7D089
:1094800076E7704703460B437FD4002243088B42A4
:1094900074D303098B425FD3030A8B4244D3030B7B
:1094A0008B4228D3030C8B420DD3FF22090212BA40
:1094B000030C8B4202D31212090265D0030B8B42BC
:1094C00019D300E0090AC30B8B4201D3CB03C01AA6
:1094D0005241830B8B4201D38B03C01A5241430B81
:1094E0008B4201D34B03C01A5241030B8B4201D371
:1094F0000B03C01A5241C30A8B4201D3CB02C01ADC
:109500005241830A8B4201D38B02C01A5241430A53
:109510008B4201D34B02C01A5241030A8B4201D342
:109520000B02C01A5241CDD2C3098B4201D3CB01E9
:10953000C01A524183098B4201D38B01C01A524198
:1095400043098B4201D34B01C01A524103098B429C
:1095500001D30B01C01A5241C3088B4201D3CB0087
:10956000C01A524183088B4201D38B00C01A52416A
:1095700043088B4201D34B00C01A5241411A00D21A
:1095800001465241104670475DE0CA0F00D0494283
:10959000031000D34042534000229C4603098B42F3
:1095A0002DD3030A8B4212D3FC22890112BA030A7B
:1095B0008B420CD3890192118B4208D389019211FD
:1095C0008B4204D389013AD0921100E08909C30982
:1095D0008B4201D3CB01C01A524183098B4201D384
:1095E0008B01C01A524143098B4201D34B01C01A6F
:1095F000524103098B4201D30B01C01A5241C308E7
:109600008B4201D3CB00C01A524183088B4201D355
:109610008B00C01A5241D9D243088B4201D34B0070
:10962000C01A5241411A00D20146634652415B10B2
:10963000104601D34042002B00D549427047634693
:109640005B1000D3404201B5002000F005F802BDD8
:109650000029F8D016E770477047C046D0400B1C71
:109660001141203A03D49C461341184363465242A9
:10967000934018437047C0468446101C62468C468F
:10968000191C634600E0C0461FB501F097F800289A
:1096900001D40021C8421FBD10B500F0EFFF4042C9
:1096A000013010BD10B501F089F8002801DB002061
:1096B00010BD012010BDC04610B501F07FF8002894
:1096C00001DD002010BD012010BDC04610B501F025
:1096D00011F8002801DC002010BD012010BDC0469B
:1096E00010B501F007F8002801DA002010BD0120B4
:1096F00010BDC046F0B5CE46474615042D0C2E00D1
:1097000080B50704140C3F0C9946030C7E435D435F
:10971000674363437F19340CE4199C46A54203D97F
:1097200080235B029846C4444B4643435143250C77
:1097300036046544360C2404A4195B19591820001A
:109740000CBC90469946F0BDF0B54E46574645468E
:10975000DE46E0B543025B0A450083B00F1C994624
:109760002D0EC60F002D57D0FF2D24D08020DB00FA
:10977000C0041843002381469A469B467F3D7C02E5
:109780007A00FB0F640A120E984623D0FF2A4BD0B2
:10979000E30080240020E4047F3A1C43AD186B1CD6
:1097A00047460193534677403A000F2B48D87D49EE
:1097B0009B00CB589F46002B00D085E008339A468B
:1097C000063B9B467C027A00FB0FFF25640A120EC3
:1097D0009846DBD1002C00D090E0524601231A437A
:1097E00092460120DBE74C4658461700022824D059
:1097F000032800D1CFE00022002301284DD15802D8
:10980000D205400AFF071043384303B03CBC9046E2
:109810009946A246AB46F0BD002B5BD104239A4685
:10982000033B00259B46AAE7FF35002C60D152463A
:1098300002231A4392460220B1E7FF220023DEE70B
:109840004B461B0C9C464B462604360C18046146BE
:109850003300220C6446000C43434E4350435443B0
:1098600080191A0C1218964203D9802149028C469D
:1098700064441B041B0C1004C01883015E1EB3411A
:10988000800E1843130C1B199B0103431C0023017A
:1098900079D5012362081C401443019A7F32002AC3
:1098A0004DDD630704D00F232340042B00D0043484
:1098B000230103D53C4B019A1C408032FE2ABCDCBC
:1098C000A3015B0AD2B29AE70C239A46093BFF2513
:1098D0009B4654E7180001F071FE4A46431F762567
:1098E0009A4000236D4291462D1A9A469B4646E7C0
:1098F000524603231A439246032050E7200001F00A
:109900005DFE431F2D1A9C40763D002047E78023D3
:109910000027DB03FF2272E7424666E74C4632002F
:10992000584662E780234A46DB031A4222D01C4293
:1099300020D123435B025B0A4746FF225FE70123F6
:109940009A1A1B2A21DC23000199D3409E318C40B6
:109950001A0023005C1EA34113435A0704D00F22B0
:109960001A40042A00D004335A0111D49B015B0A27
:10997000002244E780234A46DB0313435B025B0A71
:109980003700FF223BE7019587E70022002336E7F7
:109990000122002333E78023DB0323435B025B0ABE
:1099A000FF222CE770E30000FFFFFFF770B50028EF
:1099B0003DD0C317C5185D40C40F280001F0FEFD5F
:1099C0009E22121A962A07DCD2B2082833DD083804
:1099D00085406802400A23E0992A0BDD052329000F
:1099E0001B1AD94003001B339D402B005D1EAB4169
:1099F00019430D00052801DD431F9D402B000F4931
:109A00000B406E0709D00F263540042D05D00433D6
:109A10005D0102D59F220B40121A9B01580AD2B257
:109A20004002D205400AE4071043204370BD0024E1
:109A300000220020F4E76802400AF1E7FFFFFFFB85
:109A4000F0B54F464646D6460C000903C0B5490A54
:109A5000470F5E0039431F03DB0F9C4665007B0AFE
:109A6000570F1F436D0DE40F760DA146C000B84699
:109A7000D200AB1B64457BD0002B5FDD002E00D0F5
:109A8000A4E03E00164300D112E15E1E002E00D07D
:109A90009EE1871A4346B84280410125C91A4042D7
:109AA000091A0B0200D431E149024E0A002E00D1FE
:109AB0006EE1300001F082FD0300083B1F2B00DD4A
:109AC00061E120223900D21A9E40D1409F400E43CE
:109AD0009D4200DD51E15D1B6B1C1F2B00DD7CE115
:109AE0002021C91A3D0030008F408840DD40791E9A
:109AF0008F41310007222843D940002507433A40CF
:109B0000002A09D00F233B40042B05D03B1DBB424C
:109B1000BF417F42C9191F000B0200D426E26A1C14
:109B2000C64B55056D0D9A4200D106E1C44AFF08A7
:109B30000A40530752023B43120B8EE0002B00D029
:109B4000B8E06B1C5B055B0D012B00DC30E1871A74
:109B50004346B842B641CB1A76429E1B330200D52B
:109B60004CE13B003343A1D100220024002570E0EA
:109B7000002B00DCE5E0002E00D183E0AF4EB542C3
:109B800060D0802636043743B846382B00DC3EE1EF
:109B9000434613431F007A1E97413F188742804176
:109BA000404209180B0200D4B0E0A44B01359D429D
:109BB00000D1C3E0A24A7B080A4001210F401F43A5
:109BC0005108D30707221F433A4099E79B4EB542FD
:109BD00038D0802636043743B846382B00DDDCE029
:109BE0001F2B00DC30E11E004746203EF740BC46FC
:109BF000202B04D04026F31A46469E4032431700DD
:109C000063467A1E97411F43CCE0002B00D104E24B
:109C10004346134300D159E14B07C0081843802342
:109C2000C9081B03194208D04546ED081D4204D15E
:109C30004346D008590708432900420FC9007F4D09
:109C40001143C0004B07CA087C49C00803438D423A
:109C500068D012036D05120B6D0D00211203180060
:109C6000130B0A0D12051A43764B2D0513402B4397
:109C70005B00E4075B08234319001CBC904699462F
:109C8000A246F0BD3E00164312D05E1E002E00D04C
:109C900000E187188742804141444042091801256C
:109CA0000B0233D5022585E7644633004146100098
:109CB0001D00C7E7002D00D0DAE00C000443F3D00C
:109CC0005C1C00D19FE15D4CA64200D12FE1DB433B
:109CD000382B00DD66E11F2B00DD83E12024050029
:109CE000E41A0F00DD40D940A0404346A7405B1A6C
:109CF000441EA04198462F433843171ABA42924156
:109D000043465242991A64463500CAE607223A4051
:109D1000002A00D0F6E64B07CA084849FF083B4333
:109D20008D4296D11900114300D19EE18021090393
:109D30000A431203120B414D8FE715000022002346
:109D40008BE7002B00D0C7E06B1C5F057F0D012F58
:109D500000DCF1E0394DAB4200D1B9E085180A00D2
:109D6000854289414244494251180722CF076D0874
:109D70002F4349083A401D00C2E607223049ED1A38
:109D800031403A40BCE63E002838864000279FE636
:109D9000380001F013FC20308EE6434613431F00C9
:109DA0007A1E9741C71BB84280414042091A78E6A3
:109DB0000E003B0006431343002D61D1002E00D05E
:109DC000F4E0002B00D11BE164463900100039E7B4
:109DD0001A4FBB427AD03300FFE630001F3DE84007
:109DE000202B03D04021CB1A9E4037437B1E9F413E
:109DF000072207433A400021002589E7171A434606
:109E0000BA42B641591A76428E1B64464EE61F2B63
:109E100000DDADE020264746F61AB740B9461700E8
:109E2000B246DF404E463E4337005646B240561ECD
:109E3000B24117434246DA408918AEE6FF070000F8
:109E4000FFFF7FFFFFFF0F8020264746F61AB7402F
:109E5000B9461700B246DF404E463E4337005646ED
:109E6000B240561EB24117434246DA40891A99E77A
:109E70007F4CA6425BD0802424045B42214327E729
:109E8000002E0CD1002B00D1CBE06446390010002D
:109E9000774DD7E6764FBB4218D0330075E6002BDE
:109EA00014D04B07C00818438023C9081B0319426C
:109EB00007D0FC081C4204D17907D0080843E146CA
:109EC00021004C46420FC9001143C000684DB9E65D
:109ED0001D0000220023C0E6002D5BD10D000543CC
:109EE00000D1E2E65D1C00D1B0E0614DAE421FD072
:109EF000DB43382B71DC1F2B00DD96E020250F00A3
:109F0000ED1AAF40B9460700AA46DF404D463D4333
:109F10002F005546A840D940451EA8418844074314
:109F2000BF18974292415142414435003AE6644697
:109F300035004146100085E60B000343002D00D09C
:109F400063E6002BF5D04346134300D17AE6871829
:109F50008742804107224144404209183A400B029F
:109F600000D4D5E6434B01351940C9E5380069E610
:109F70001E004746203EF740BC46202B04D040261A
:109F8000F31A46469E403243170063467A1E9741B5
:109F90001F4302E6364DAE42CAD080252D045B42F7
:109FA0002943A6E70843411E8841A6E6002B00D1BD
:109FB00048E6871A4346B842B641CB1A76429E1B02
:109FC00033024BD5171A4346BA429241591A5242AC
:109FD000891A072264463A4092E501430F00791E30
:109FE0008F419DE71C000F00203CE740202B03D051
:109FF0004024E31A99400843411E884138437CE6D7
:10A000000022002425E6171A4346BA429241591A03
:10A010005242891A6446350043E541461000144D0A
:10A0200010E680220024120380E61D000F00203D70
:10A03000EF40BC46202B03D04025EB1A9940084343
:10A0400007006346781E87411F4369E787189742D8
:10A050009B4141445B42C9183500A3E53B003343B3
:10A06000CED0072231003A4052E600231A00F4E530
:10A07000FF070000FFFF7FFFF0B55746DE464E4664
:10A080004546E0B5834607000E03480085B092467A
:10A090001C00360B400DCD0F002800D19DE0954BE4
:10A0A000984239D08023F6001B041E43924A7B0F4E
:10A0B00033439946944603006344009300230026EB
:10A0C000FF00029323031B0B98466300E40F5246E4
:10A0D0005B0D019400D1B3E086498B4200D19EE034
:10A0E0004246D100802212040A435146490F1143CF
:10A0F0008B46814952468C4600996344CB1A002115
:10A10000D20000932B0063409A460F2E00D905E140
:10A110007A4BB6009B599F465B463343994600D025
:10A12000B8E002230826002700900293CAE7CB4636
:10A130003A0002990195019B9A46022927D00329EA
:10A1400000D180E2012944D06D49009B8C466344D4
:10A150001C00002C38DD530700D013E2D2085B4608
:10A16000DB0109D55946674B19408B468021C90050
:10A170008C46009B63441C00634B9C4207DC5B469F
:10A1800064055F075B0217431B0B620D02E00023AF
:10A190000027584A00211B031C0B0B0D1B052343F2
:10A1A00014055A4A380013401C4353466400DB0729
:10A1B00064081C43210005B03CBC90469946A24669
:10A1C000AB46F0BD0122524201231B1B382B00DCA1
:10A1D000ADE1002200230027DCE75B4633439946CC
:10A1E0005ED0002E00D18AE1300001F0E7F90300D3
:10A1F0000B3B1C2B00DD7BE11D22D31A5A460100CC
:10A20000DA4008398E4013005F46334399468F4049
:10A210003F4B00261B1A00930023029352E741464E
:10A2200053460B433B499B468C46009B634400933B
:10A230005B46002B3BD1022300221E43022161E733
:10A24000434613439B4637D04346002B00D162E17F
:10A25000404601F0B3F903000B3B1C2B00DD53E13A
:10A2600002004146083A914088461D21CB1A5146CA
:10A27000D9400B0041460B439B46534693401A007E
:10A28000009B25499C46604403008C466344009330
:10A29000002137E70323B14600900C26029311E713
:10A2A0000023009301330426002702930AE70323C7
:10A2B000C3461E43032125E701331E43002201212B
:10A2C00020E700239A46802300271B03094A61E701
:10A2D000802349461B03194200D1E2E05946194246
:10A2E00000D0DEE00B431B0317001B0BA246014A04
:10A2F00050E7C046FF07000001FCFFFFB0E300008D
:10A30000FF030000FFFFFFFEFE070000FFFF0F80BE
:10A310000DFCFFFF01F8FFFFF3030000D94500D952
:10A32000CBE000D1C6E03C0048460027009B013B43
:10A3300000935B46160E1B021E431302984633041D
:10A340001B0C9946310C0191FFF798F84A4642439D
:10A350000B04210C050019438A4207D98919013DD4
:10A360008E4203D88A4201D9851E8919881A01991B
:10A37000FFF784F809048C464A46210464464243A8
:10A38000090C030021438A4204D98919013B8E42FA
:10A3900000D8F1E02D041D43AB464346891A4246DE
:10A3A000280C12041D0C5B46140C22001B041B0C11
:10A3B0005A4303946B434443029568431B19150C9D
:10A3C000EB189C4203D980246402A44660441C0C10
:10A3D00015041B042D0C20185D19814277D373D00E
:10A3E0000C1AA24A7D1BAF42BF419446009B7F429C
:10A3F0006344E01B1C00864200D1DBE00199FFF7BB
:10A400003DF84A4642430B04290C070019438A428F
:10A4100007D98919013F8E4203D88A4201D9871E84
:10A420008919881A0199FFF729F809044A468946CB
:10A4300029044D464243090C030029438A4207D9A7
:10A440008919013B8E4203D88A4201D9831E89199A
:10A450003F04891A3A00039F1A43380013041B0C67
:10A46000584381460298150C6F4343434543484681
:10A47000000C8446DB1963449F4203D980204002CC
:10A480008446654448461F0C00041B04000C7D19DB
:10A490001818A94200D284E000D17FE001231A43BA
:10A4A00057E680234A461B0313431B031B0BAA4694
:10A4B0006F4A6FE6BA4200D935E74B46DC075808C9
:10A4C0007B081C43FF0734E70024AF4289D247448E
:10A4D0004745A4415B466442A4196418013BA64267
:10A4E0001ED2A0426DD800D1B6E0241A9B4678E770
:10A4F00003005A46283B9A400027914688E6584672
:10A5000001F05CF8203072E603005246283B9A4086
:10A5100093460022B4E6504601F050F820309AE607
:10A52000A642E2D1B845DCD9341A9B4659E71F2B25
:10A5300065DC504C0099A4465C46614408008C40A0
:10A5400011008240D940501E82410C4314435A46A8
:10A55000DA401300620709D00F222240042A05D0F6
:10A560002200141D9442894149425B181A0262D5A7
:10A570000122002300270DE68A4200D80AE7831E45
:10A58000891907E70F231340042B00D1E6E5171DB7
:10A590009742924153429B44FA08E0E5002800D1DB
:10A5A000D7E57118531EB14227D3A94215D358D00D
:10A5B0001A0073E7002B00DC04E6012300229B4411
:10A5C000CDE502234744474589415B429C464942C9
:10A5D00089190C19E344241A03E743465F004745F1
:10A5E0009B41B8465B429E19023A8919A94200D0A4
:10A5F00054E7404500D051E7ABE51A00F6E71F21CC
:10A600005F4649420C1BE740202B07D01A49009BAC
:10A610008C46634418005B4683401A43501E8241B7
:10A620003A4307270023174009D00F210023114088
:10A630001400042995D122005F075B021B0BD2088E
:10A6400017430022A6E5802359461B030B431B0337
:10A6500017001B0B064A9DE5BD42B2D89B4600245D
:10A66000BFE68045B9D31A00C3E7C046FF03000028
:10A67000FF0700001E0400003E040000F0B54F4636
:10A680004646D6468446C0B58046194E18030F0389
:10A690004D00000B5C0082463F0B6D0DC90F9146CB
:10A6A000640DDB0F0120B5420AD0B44203D0A542AD
:10A6B00001D157450CD01CBC90469946A246F0BD2E
:10A6C00066463E43F7D1AC42F5D154461443F2D12D
:10A6D0000120C845EFD1994207D0002DEBD1634648
:10A6E0001F433800471EB841E5E70020E3E7C046B6
:10A6F000FF070000F0B54F464646D6464D00C0B5B0
:10A700000E03C90F8A462C491F035C008046360B96
:10A710006D0D91463F0B640DDB0F8D421ED08C42B8
:10A7200016D0002D1ED130438446002C01D13A436F
:10A7300023D06246002A1AD09A4529D051460220D9
:10A740000139084001381CBC90469946A246F0BD2C
:10A7500039001143E5D002204042F4E73043FAD1FA
:10A76000AC420FD0002C0FD13A43E7D00CE00122CD
:10A77000013B934318000130E5E763460020002BBE
:10A78000E1D0DBE73A43E6D19A45D7D1A542D5DC03
:10A79000A54205DBBE42D1D808D00020BE42D2D2AD
:10A7A00050460123013898430130CCE7C845C5D84D
:10A7B0000020C845F4D3C6E7FF070000F0B54F46B8
:10A7C0004646D6464D00C0B50E03C90F8A462E49EF
:10A7D0001F035C008046360B6D0D91463F0B640DE8
:10A7E000DB0F8D4218D08C4211D0002D18D1304390
:10A7F0008446002C1ED13A431CD163460020002B16
:10A8000030D0514602200139084001382AE0390091
:10A810001143EAD0022025E03043FBD1AC4226D0E0
:10A82000002C26D13A4324D1514602200139084058
:10A83000013817E06246002A0FD09A45E1D1A542BF
:10A8400005DBBE42DDD819D00020BE420AD25046F8
:10A85000012301389843013004E00122013B934376
:10A86000180001301CBC90469946A246F0BD3A4300
:10A87000D0D19A45C5D1A542C3DCE0E7C845C0D8D0
:10A880000020C845E3D3EDE7FF070000F0B55746C9
:10A89000DE464E464546E0B5834606000F034800B7
:10A8A00087B092461D003F0B400DCC0F002800D111
:10A8B0006FE0DE4B984238D08023FF001B041F431B
:10A8C000730F3B430193DA4B0027994600239B46C5
:10A8D000F60081442B0369001B0B52469846490D34
:10A8E000ED0F002900D185E0D04B994200D173E0F3
:10A8F0004346DA0080231B0413435246CC48520FD0
:10A9000084461343524600206144D200894421000A
:10A91000694000918C46012149448A460F2F00D995
:10A9200090E0C449BF00CF59BF465B463B4301930B
:10A9300000D06AE102230827002681469B46C9E72A
:10A9400032005846019B61460091022800D175E013
:10A95000032800D1FEE1012800D02CE100230027CC
:10A96000002600253F032A0D3F0BB34812053A434A
:10A9700002401B051343009A5B00D1075B080B43A1
:10A980003000190007B03CBC90469946A246AB4641
:10A99000F0BD5B463B43019300D12FE1002F00D176
:10A9A000A5E1380000F00AFE03000B3B1C2B00DD84
:10A9B00096E11D22D31A5A460100DA405E46083954
:10A9C0008F4013008E403B4301939C4B00271B1A82
:10A9D000994600239B467DE7414653460B439349E6
:10A9E0008C46E144002B00D01AE1022202201743DA
:10A9F00000228CE7134300D10DE14346002B00D128
:10AA000081E1404600F0DAFD02000B3A1C2A00DD2D
:10AA100072E10100434608398B4098461D239A1A7B
:10AA20005346D3401A004346134352468A40494690
:10AA3000081A824989468144002068E77B4B002739
:10AA400000268EE7140C1204120C1100370C360489
:10AA5000350C794328008C462E00604360448346C1
:10AA600056432100300C80465846794340440291B9
:10AA7000844506D98846802149028C46E0444146F7
:10AA800002913604010C360C00048B4681191E0C11
:10AA90001B041B0C0391190079438C462800754355
:10AAA0006544A8465843050C45447743A94203D959
:10AAB000802149028C466744290C8C4639000004E9
:10AAC000000C2D042D186144AB44059159460491A6
:10AAD00001990F043F0C080C390051434243904642
:10AAE00002008C46090C8B4662437C4344445C4420
:10AAF000A04503D98021490288464244210C88465A
:10AB000061460904090C8C4639005943434370439C
:10AB10007E430F0CF6182404BE19644442448C464C
:10AB2000B34203D980235B0298464044029B6146AE
:10AB30009846049B370443449B46AB45AD416B426A
:10AB40000D0405992D0C8C467F196744FD18A84605
:10AB50005D462D19A542A44193466442A446C344D0
:10AB6000DC448F42BF4198459B4193459241A445A7
:10AB7000A4415B427F421F43360C52426442BF19DC
:10AB80002243BF18624638184302D20D039913437B
:10AB90006A020A43501E82416146ED0D2A434E026D
:10ABA0003243D90100D4B3E00126500832400243B9
:10ABB000DE0732435B08224C5444002C62DD51070F
:10ABC00009D00F201040042805D0101D904292415A
:10ABD00052429B180200D90104D580241948E40090
:10ABE000034054441848844200DD27E75E075B02B7
:10ABF000D2081F0B630516435B0DB2E6002399468E
:10AC00000133042700269B4664E60323019781460F
:10AC10000C279B465EE6012201201743002276E6C0
:10AC2000032303201F43434671E6C046FF0700008D
:10AC300001FCFFFFF0E30000FFFF0F800DFCFFFFB2
:10AC4000FF030000FFFFFFFEFE0700000023802738
:10AC500000933F030026434B83E6019B3200A4464A
:10AC6000584670E6AC466EE6802701993F033942AC
:10AC70002DD03B422BD11F433F033F0B00951600C5
:10AC8000384B6EE601252D1B382D00DD66E61F2DA5
:10AC900040DC35481C005044160082408440EE40A1
:10ACA000501E824134431443EB40620709D00F2207
:10ACB0002240042A05D02200141D944280414042C3
:10ACC0001B181A023ED501230027002649E68027DB
:10ACD000019B3F031F433F033F0B0094214B40E682
:10ACE00003005A46283B9A40002601926DE65846DA
:10ACF00000F064FC203057E603005246283B9A409F
:10AD00001300002293E6504600F058FC20307BE60A
:10AD1000CA4650E71F201E004042041BE640202D7B
:10AD200003D0124C5444A3401A43501E8241324374
:10AD300007260027164009D00F20002310401400DA
:10AD40000428B9D122005E075B021F0BD20816430C
:10AD5000002306E680273F031F433F033F0B1600F7
:10AD6000004BFEE5FF0700001E0400003E0400004B
:10AD7000F8B557464E464546DE460C000903E0B599
:10AD8000490A460F5F0031431E03DB0F760A9B46DC
:10AD9000530F3343C84E6500C000E40FD2006D0D61
:10ADA000A24681467F0D9C469046B74200D1B9E04D
:10ADB0005B46012673409B46EE1BA34500D183E012
:10ADC000002E63DD002F00D0B1E06346134300D1B5
:10ADD00023E1731E002B00D0BAE1861A6346B0420D
:10ADE00080410125C91A4042091A0B0200D447E1EB
:10ADF00049024B0A98464346002B00D189E1404660
:10AE000000F0DCFB0300083B1F2B00DD7CE120226F
:10AE10003000D21A4146D040994002009E400A4379
:10AE20009D4200DD6AE15D1B6B1C1F2B00DD94E180
:10AE3000202110003500C91A8E40DA408840DD40DC
:10AE4000711E8E411100072228430025064332401F
:10AE5000002A09D00F233340042B05D0331DB34201
:10AE6000B641764289191E000B0200D43DE26A1CED
:10AE7000914B55056D0D9A4200D119E18F4AF608A4
:10AE80000A40570752023743120B9BE0002E00D0B6
:10AE9000C5E06E1C7605760D012E00DC48E16746A4
:10AEA000861ACB1BB042BF417F42B8461F004346C3
:10AEB000FF1A3B00B8461B0200D55FE137439AD129
:10AEC00000220024002579E0002E00DCFAE0002FAB
:10AED00000D18DE0784B9D4267D0802367461B04EC
:10AEE0001F43BC46382E00DC52E1634613435A1E12
:10AEF00093411E1886428041404209180B0200D43B
:10AF0000BEE06D4B01359D4200D1D2E06B4A730823
:10AF10000A4001210E401E435108D30707221E4359
:10AF2000324095E71E00164300D045E740E7624BEC
:10AF30009D423AD0802367461B041F43BC46382EEF
:10AF400000DDEBE01F2E00DC3AE133006746203BDA
:10AF5000DF403B00202E05D04027BF1B6646BE4089
:10AF6000324390464646721E96413343DAE0002B48
:10AF700000D114E26346134300D168E180234E07F9
:10AF8000C008C9081B030643194208D06046C00820
:10AF9000184204D163460100D2085E071643F3004D
:10AFA0009946C900720F444D11434B46DE08424B8F
:10AFB0004F073743CA089D4200D16EE012036D056A
:10AFC000120B6D0D00211203130B0A0D12051A430B
:10AFD0003B4B2D0513402B435B00E4075B082343E9
:10AFE000380019003CBC90469946A246AB46F8BDD5
:10AFF0006346134311D0731E002B00D007E186185F
:10B000008642804161444042091801250B0237D530
:10B0100002257BE73E00614691463500C5E75C4668
:10B02000002D00D0E1E00B000343F3D0731C00D1EE
:10B03000ACE1214B9F4200D13AE1F343382B00DDD4
:10B040006FE11F2B00DD8CE120250E00ED1AAE40D4
:10B05000B0460600AA46DE40454635432E0055461A
:10B06000D940A8406346451EA8415B1A9C46304320
:10B07000161AB242924163465242991A3D00B4E612
:10B0800007223240002A00D0E4E60B4BF6084F07B7
:10B090003743CA089D4200D090E73B00134300D1DC
:10B0A000A6E180231B031A431203120B024D89E70A
:10B0B00015000022002785E7FF070000FFFF7FFF44
:10B0C000FFFF0F80002E00D0C7E06B1C5E05760DE1
:10B0D000012E00DCF0E0C84DAB4200D1B9E085188C
:10B0E0000A00854289416244494251180722CE072D
:10B0F0006D082E43490832401D00A9E6BF49ED1AEC
:10B10000114007223240A3E6320028388240002650
:10B1100086E6300000F052FA203073E663461343AF
:10B120005A1E9341C61AB04280414042091A5CE659
:10B130000E00674606431743002D5ED1002E00D057
:10B14000F3E0002F00D11EE15C46614691462CE7FA
:10B15000A94FBE427BD01E00F1E610001F3DE84023
:10B16000202B03D04021CB1A9A401643731E9E41D8
:10B170000722064332400021002583E7161A634662
:10B18000B2428041591A40420B1A98465C4632E658
:10B190001F2E00DDABE02027BB1B9A4663465746B7
:10B1A000BB40994613004F46F3401F433B005746B0
:10B1B000BA40571EBA4113436246F240891898E6D6
:10B1C0002027BB1B9A4663465746BB40994613004F
:10B1D0004F46F3401F433B005746BA40571EBA4103
:10B1E00013436246F240891A9CE7834B9F425FD02B
:10B1F00080252D047342294320E7002E0CD1002F17
:10B2000000D1D0E05C46614691467B4DCDE67A4F59
:10B21000BE421CD01E0065E6002F18D0C0084E07A5
:10B2200006438020C9080003014208D06346DC08B9
:10B23000044204D12100DA46D2085E071643F30027
:10B24000994601245346C900720F11431C406A4DB0
:10B25000ABE61D0000220027B4E6002D59D10B00FB
:10B26000034300D1D6E6731C00D1B2E0624B9F428B
:10B270001ED0F343382B6FDC1F2B00DD97E0202519
:10B280000E00ED1AAE40B0460600AA46DE40454626
:10B2900035432E005546A840D940451EA8418C4450
:10B2A0000643B61896429241514261443D0025E65C
:10B2B0003D006146914678E60B000343002D00D027
:10B2C00055E6002BF5D06346134300D16DE6861892
:10B2D0008642804161444042091800220B0200D49A
:10B2E000D0E6464B01351940B2E5B1465DE6330084
:10B2F0006746203BDF403B00202E05D04027BF1B88
:10B300006646BE40324390464646721E96413343DF
:10B31000EFE5394B9F42CBD080252D047342294362
:10B32000A8E70843411E8841A2E6002F00D13CE671
:10B330006346861ACF1AB0429B415B42FB1A98467D
:10B340001B024ED5161A6346B2429241591A524216
:10B35000891A5C4600227BE501430E00711E8E4176
:10B360009FE71D000E00203DEE40B046202B04D08C
:10B370004025EB1A99400843814648464346411E02
:10B380008841184374E60022002417E6161A634623
:10B39000B2429241591A5242891A3D0025E561464E
:10B3A0009146154D01E680220024120379E61D0026
:10B3B0000E00203DEE40B046202B04D04025EB1A75
:10B3C0009940084381464E464346711E8E411E43B6
:10B3D00067E7861896429B4161445B42C9183D006D
:10B3E0008CE547463743CED007224146324049E6F6
:10B3F00000273A00E6E5C046FF070000FFFF7FFF99
:10B4000070B50C4E0D031C0349005B002D0B490D5C
:10B41000240B5B0DB14208D0064900208B4203D1BA
:10B4200014432000441EA04170BD05430120002D9F
:10B43000FAD1F1E7FF07000030B5144D0A034B00C5
:10B44000120B5B0DC90F0024AB4211DD104CA3425F
:10B4500010DC8024640322430E4CE41A1F2C0CDD04
:10B460000D48C31ADA4013005C42002900D11C00C9
:10B47000200030BD094BCC18FAE7094DE040AC463E
:10B4800063449A4013000343EEE7C046FE03000006
:10B490001D0400003304000013040000FFFFFF7FC1
:10B4A000EDFBFFFF70B500282DD0C317C5185D4018
:10B4B000C40F280000F082F8154B1B1A5B055B0DCA
:10B4C0000A2815DD0B38854000222D032D0B0021A5
:10B4D00010002D030A0D2D0B12052A430D4D1B05DF
:10B4E0002A4013435B00E4075B082343190070BD47
:10B4F00002002900153291400A000B21081AC540AC
:10B500002D032D0BE3E70024002300250022DEE7B6
:10B510001E040000FFFF0F804100090E4B1C70B598
:10B52000DBB24602750AC40F012B14DDE0239B0039
:10B530006D07360BCB1800210A0D280012051C4D93
:10B5400032435B052A405B0813435B00E4075B085A
:10B550002343190070BD002914D1002D1ED02800EE
:10B5600000F02CF80A281CDC0B232A001B1ADA40F6
:10B57000030015339D400F4B12031B1A5B05160B7E
:10B580005B0DD8E7002D06D0320B802636036D0701
:10B590001643094BCFE7084B0026CCE700230026D3
:10B5A000C9E703002A000B3B9A400025E3E7C046A9
:10B5B000FFFF0F8089030000FF0700001C2101230B
:10B5C0001B04984201D3000C10391B0A984201D386
:10B5D000000A08391B09984201D30009043902A264
:10B5E000105C40187047C0460403020201010101CB
:10B5F000000000000000000030B51C00094B0500F1
:10B600001B6885B0D868084B002A01D1074B1A0087
:10B610000292019300912B002200054900F026F8C8
:10B6200000F0A6FD8400002030E4000040D20000BD
:10B630003DE40000014B18687047C04684000020BC
:10B64000084B10B50400002B02D0002100E000BF21
:10B65000054B1868836A002B00D09847200001F042
:10B660005DFBC046000000006CE400000EB403B5B2
:10B67000010003AB044804CB0068019300F076F8A6
:10B6800002B008BC03B018478400002070B5002643
:10B690000C4D0D4C641BA410A64209D1002601F0EC
:10B6A0003FFB0A4D0A4C641BA410A64205D170BD95
:10B6B000B300EB5898470136EEE7B300EB589847D4
:10B6C0000136F2E754020020540200205402002008
:10B6D00064020020002310B59A4200D110BDCC5C5A
:10B6E000C4540133F8E710B5884202D98B18984248
:10B6F00003D3002307E08B5C8354013AFBD210BDD7
:10B70000CC5CC45401339A42FAD1F8E70300121812
:10B71000934200D1704719700133F9E7936810B56F
:10B72000013B9360002B04DA9469A34207DB0A29EA
:10B7300005D01368581C10601970080010BD00F087
:10B740004BFC0100F9E7F8B506000F001400D5180E
:10B75000AC4201D1002007E021783A003000FFF729
:10B76000DDFF0134431CF3D1F8BD0000F0B59FB0FC
:10B7700002900F0016000593002805D083690493FA
:10B78000002B01D100F0F4FD7B4B9F425BD1029B6B
:10B790005F68BB891B0762D53B69002B5FD0002324
:10B7A00006AC6361203363761033A37635002B78C3
:10B7B000002B01D0252B5CD1AB1B04930CD03200A5
:10B7C00039000298FFF7BFFF431C00D1C4E0626953
:10B7D000049B9446634463612B78002B00D1BBE04B
:10B7E000012200235242626002A9543252186E1C98
:10B7F0002360E360A3601370A365317805225F487E
:10B8000000F0D4FE751C002835D12268D30604D57B
:10B81000532302A95B1820211970130704D5532361
:10B8200002A95B182B21197033782A2B2CD03500F4
:10B8300000210A20E3682A786E1C303A092A64D96C
:10B8400000292ED026E04E4B9F4202D1029B9F68DA
:10B850009FE74C4B9F429CD1029BDF6899E73900E0
:10B86000029800F00FFC002899D0012040421FB040
:10B87000F0BD01359BE7414B2268C01A012383408C
:10B88000134323602E00B8E7059B191D1B68059123
:10B89000002B01DB099304E05B42E36002231343C6
:10B8A00023602B782E2B0AD16B782A2B35D1059B60
:10B8B00002351A1D1B680592002B2BDB0793324EB5
:10B8C00029780322300000F071FE002806D04023C2
:10B8D000801B8340226801351343236029780622A8
:10B8E0002A486E1C217600F061FE00283AD0284BD1
:10B8F000002B25D10722059B07339343083305937B
:10B900006369039A9B18636150E7434301219B18C5
:10B91000350090E701235B42D0E700230A201A009C
:10B920000135636029786E1C3039092903D9002B51
:10B93000C5D00792C3E74243012352183500F1E70F
:10B9400005AB00933A00134B2100029800E000BFC2
:10B950000390039B0133D3D1BB895B0600D584E7F9
:10B960000B9884E705AB00933A000A4B210002983C
:10B9700000F080F8ECE7C046C4E4000070E400008A
:10B98000E4E40000A4E4000076E400007AE40000AF
:10B990000000000047B70000F7B5150001938A6862
:10B9A0000B6900900C00934200DA130022002B6018
:10B9B00043321278002A01D001332B6023689B06A2
:10B9C00002D52B6802332B60062723681F4027D03F
:10B9D000230043331B785A1E93412268920630D4C9
:10B9E0002200019943320098089EB047431C25D09D
:10B9F000062320682A68E16803400025042B03D150
:10BA00008D1AEB43DB171D40A3682269934201DDC9
:10BA10009B1AED180027BD4220D1002010E001370D
:10BA2000E3682A689B1ABB42D2DD22000123193247
:10BA300001990098089EB047431CF0D10120404274
:10BA4000FEBD3020E1184331087021005A1C4531F9
:10BA50000978A218433202331170C1E72200012392
:10BA60001A3201990098089EB047431CE6D001376E
:10BA7000D1E70000F0B589B004920A004332059383
:10BA8000039002920A7E0C000E9B6E2A00D186E083
:10BA90001FD8632A33D008D8002A00D18CE0582A56
:10BAA0004DD0250042352A7030E0642A01D0692A41
:10BAB000F7D1196825680A1D280629D508681A6073
:10BAC000002803DA2D23029A404213706B4E0A2796
:10BAD0004FE0732A74D008D86F2A1FD0702AE0D1A3
:10BAE000202209680A43226003E0752A16D0782ACA
:10BAF000D7D12200782145321170614E22E0250015
:10BB00001A684235111D196013682B70012365E016
:10BB100008681A606906D3D500B2D1E719682568AC
:10BB2000081D186008682E0605D5544E08276F2A90
:10BB30001BD00A2719E06D06F7D580B2F5E745312D
:10BB40004E4E0A7018682268011D006819601506BB
:10BB500021D5D30702D520231A43226010270028BD
:10BB600003D1202322689A4322602300002243331A
:10BB70001A706368A360002B58DB0422216891438C
:10BB80002160002854D1029D002B5AD02500337823
:10BB900042352B7055E05506DBD580B2D9E71A68DF
:10BBA0000D68101D4969186013682E0601D51960CB
:10BBB00002E06D06FBD519800023029D23614FE052
:10BBC0001A68111D1960156800216268280000F0CC
:10BBD000EDFC002801D0401B6060636823610023F6
:10BBE000029A13703CE023692A0004990398059D8A
:10BBF000A847431C3ED023689B0715D4079BE068E9
:10BC0000984239DA180037E02200012319320499EA
:10BC10000398059EB047431C2CD00135E368079A72
:10BC20009B1AAB42F0DCE9E70025F7E70028ADD02E
:10BC3000029D3900FDF722FC735C013D2B7000284A
:10BC4000F7D1082F09D12368DB0706D5636822697D
:10BC5000934202DC3023013D2B70029B5B1B23616E
:10BC6000059B07AA00932100049B0398FFF794FE0D
:10BC7000431CB8D10120404209B0F0BD81E400006E
:10BC800092E400000D4B70B51C680500A36B002BFF
:10BC90000FD1182000F06EFC094BA0630360094B24
:10BCA00001224360084B83600B23838100230261E0
:10BCB00043610022A36B1D615A6170BD84000020A6
:10BCC0000E33CDAB34126DE6ECDE0500124B10B531
:10BCD0001C68A36B002B0FD1182000F04BFC0F4BFE
:10BCE000A06303600E4B012243600E4B83600B2365
:10BCF0008381002302614361A46B0B4A206961695F
:10BD00000A4BFDF7F7FC01220023801859412061FE
:10BD100061614800400810BD840000200E33CDABA7
:10BD200034126DE6ECDE05002D7F954C2DF4515854
:10BD30000CB430B5164B9DB00C1E1D6808DA8B2371
:10BD400001202B6040421DB030BC08BC02B0184737
:10BD5000822302A99B008B810023029008619C42F0
:10BD600000D0631E8B604B6101235B42CB81209A24
:10BD700021AB2800019300F055FD431C01DA8B2311
:10BD80002B60002CDFD00023029A1370DBE7C04643
:10BD9000840000200EB400B50B499CB01DAB02908E
:10BDA0000690079104910948094904CB0591006860
:10BDB00002A9019300F036FD0023029A13701CB013
:10BDC00008BC03B01847C046FFFFFF7F8400002077
:10BDD0000802FFFF020010B51378541C002B05D198
:10BDE000CC5CD4540133002CFAD110BD2200F3E70F
:10BDF000C9B20378002B04D08B4200D170470130C8
:10BE0000F7E74B42594149420840F7E702780B787F
:10BE1000002A03D0013001319A42F7D0D01A70477E
:10BE20000023C25C0133002AFBD1581E7047002357
:10BE300030B59A420AD0013AC45CCD5CAC4204D120
:10BE4000934202D00133002CF6D1631B180030BDA1
:10BE500030B50500002A00D130BD0C78013A6B1CCA
:10BE60002C700131002C05D19A189A42F4D01C7024
:10BE70000133FAE71D00EDE710B50378002B0FD171
:10BE80000B785A4253415B42184010BD0023CA5CF4
:10BE9000002AFAD0C45C944201D10133F7E70130A3
:10BEA0000378002BF2D11800EFE70000F0B51F0077
:10BEB0000E0087B00590019102920C98347800F042
:10BEC000EAFA082200194378751C134036D12D2C4C
:10BED00036D1B51C74780126002F62D0102F09D1FD
:10BEE000302C07D120222B789343582B54D1102784
:10BEF0006C7802352D4B3900F31818000393FDF7C9
:10BF0000BDFA049101210023494202008C46180029
:10BF10002100303909291AD80C00A74223DD591C09
:10BF200009D06346824206D302D10499A14202DBC2
:10BF30000123784320182C780135E9E72E00BCE76F
:10BF40002B2C01D01E00C7E7B51C7478FAE721003E
:10BF50004139192901D8373CDFE721006139192916
:10BF600001D8573CD9E75A1C08D1059A23331360EE
:10BF7000029B0398002B09D107B0F0BD002E00D022
:10BF80004042029A002AF7D0002B01D06B1E019389
:10BF9000029B019A1A60EFE73024002FAAD10827EC
:10BFA000A8E7302C9ED00A27A4E7C046FFFFFF7FFA
:10BFB00037B51300064A05001068046A002C00D14A
:10BFC000044C0A0000942900FFF770FF3EBDC046F4
:10BFD00084000020E8000020F8B505000E001400E1
:10BFE000002804D08369002B01D100F0C1F9224B55
:10BFF0009C422DD16C68A369A360A3891B0731D52E
:10C000002369002B2ED023682269F7B2981A63693E
:10C01000F6B2834205DC2100280000F03BF900283D
:10C0200026D1A3680130013BA36023685A1C22601B
:10C030001F706369834204D0A389DB071AD50A2ED7
:10C0400018D12100280000F025F9002812D00FE0B7
:10C050000A4B9C4201D1AC68CDE7094B9C42CAD146
:10C06000EC68C8E72100280000F00CF80028CAD0CE
:10C07000012676423000F8BDC4E40000E4E400008C
:10C08000A4E40000364B70B51D6806000C00002DBE
:10C0900005D0AB69002B02D1280000F069F9314BC3
:10C0A0009C420FD16C680C23E25E93B219072DD429
:10C0B000D90611D409230120336037331343A381F8
:10C0C000404270BD284B9C4201D1AC68EBE7274B46
:10C0D0009C42E8D1EC68E6E75B0713D5616B002969
:10C0E00008D023004433994202D0300000F06AFAAD
:10C0F000002363632422A3899343A3810023636005
:10C10000236923600823A2891343A3812369002B99
:10C110000BD1A0218022A389890092000B40934279
:10C1200003D02100300000F0E1F90123A28913407F
:10C1300011D00023A36063695B42A36100202369DF
:10C140008342BED10C23E25E1306BAD540231343CB
:10C15000A3810138B5E7920700D46369A360EDE7D6
:10C1600084000020C4E40000E4E40000A4E4000033
:10C1700010B5062000F090FC012000F0CFFD00007B
:10C18000F7B58A8905000C00130760D44B68002BB3
:10C1900004DC0B6C002B01DC0020FEBDE76A002FE5
:10C1A000FAD000232E682B6080235B01216A1A409D
:10C1B00034D0606DA3895B0706D56368C01A636BD2
:10C1C000002B01D0236CC01A0200216A0023280032
:10C1D000E76AB847A189431C06D12B681D2B30D8CC
:10C1E0002B4ADA40D3072CD50023636023692360F0
:10C1F000CB0405D5431C02D12B68002B00D1606510
:10C20000616B2E600029C7D023004433994202D0CD
:10C21000280000F0D7F900206063BEE70123280062
:10C22000B847431CC6D12B68002BC3D01D2B01D0AF
:10C23000162B01D12E60AFE74023A2891343A381BF
:10C24000ABE740230B430120A3814042A5E70F69E0
:10C25000002FA1D00B680F60DB1B01930023920716
:10C2600000D14B69A360019B002B00DC94E7019B8C
:10C270003A00216A2800A66AB047002803DC402360
:10C28000A2891343DFE7019B3F181B1A0193EAE7DA
:10C29000010040200B6970B505000C00002B01D196
:10C2A000002070BD002804D08369002B01D100F06C
:10C2B0005FF80B4B9C4209D16C680C22A35E002BEB
:10C2C000EED021002800FFF75BFFEAE7054B9C4218
:10C2D00001D1AC68F1E7044B9C42EED1EC68ECE78D
:10C2E000C4E40000E4E40000A4E40000002310B56E
:10C2F000040003604360836081814366C2810361FF
:10C3000043618361190008225C30FFF7FFF9054B98
:10C3100024626362044BA362044BE362044B236315
:10C3200010BDC046D9CA000001CB000039CB0000C7
:10C3300065CB000010B5024900F08CF810BDC04676
:10C3400095C2000070B568254A1E55430E002900AD
:10C35000743100F081F9041E08D000212A00016028
:10C3600046600C30A0606832FFF7D0F9200070BD45
:10C37000836913B50400002B28D18364C36403656B
:10C38000134B144A1B6882620193984201D1012326
:10C390008361200000F020F86060200000F01CF8AD
:10C3A000A060200000F018F80022E060042160681E
:10C3B000FFF79CFF01220921A068FFF797FF0222E7
:10C3C0001221E068FFF792FF0123A36113BDC0466D
:10C3D0006CE4000035C30000F8B51C4B07001E6874
:10C3E000B369002B02D13000FFF7C2FF4836B468B2
:10C3F0007368013B04D53368002B07D03668F6E735
:10C400000C22A55E002D0DD06834F2E7042138001F
:10C41000FFF798FF30600028F0D10C2304003B6048
:10C420002000F8BD20000A4B656625606560A560A8
:10C43000E36025616561A561082229005C30FFF792
:10C4400065F96563A563A564E564E9E76CE400004C
:10C450000100FFFFF7B504000700002601914834F2
:10C46000002C01D13000FEBD6368A5680093009BDD
:10C47000013B009301D52468F2E7AB89012B08D971
:10C480000E22AB5E013304D029003800019B98478F
:10C4900006436835EBE7EC300068704770B50E0076
:10C4A0001D000E23C95E96B01400002907DA002390
:10C4B0002B60B3891B0611D48023DB000FE06A4692
:10C4C00000F088FB0028F2DBF022019B12021340EF
:10C4D000054A9B185A4253412B60EDE74023002048
:10C4E000236016B070BDC04600E0FFFFF7B502261E
:10C4F0008B8905000C00334206D0230047332360AC
:10C50000236101236361F7BD01AB6A46FFF7C6FFF4
:10C5100000990700280000F09FF8002808D10C229D
:10C52000A35E9A05EFD4032293431E43A681E4E75A
:10C530000F4BAB628023A28920601343A381009B31
:10C5400020616361019B002B0DD00E23E15E28006A
:10C5500000F052FB002806D00322A38993431A005F
:10C5600001231343A381A0893843A081CBE7C046B0
:10C5700035C3000010B5034B0100186800F06CF8DB
:10C5800010BDC0468400002082B0002900D101A95E
:10C59000101E06D0002B06D013780B601078431EB7
:10C5A000984102B0704702204042FAE7C9B28218AF
:10C5B000904201D10020704703788B42FBD00130BC
:10C5C000F6E7000070B50500002910D00C1F2368A5
:10C5D000002B00DAE418280000F034FB1D4A136831
:10C5E000002B05D163601460280000F02CFB70BDA7
:10C5F000A34209D9216860188342F3D118685B68A7
:10C6000041182160EEE713005A68002A01D0A242C7
:10C61000F9D919685818A0420BD120680918581880
:10C6200019608242E0D110685268411819605A605E
:10C63000DAE7A04202D90C232B60D5E72168601805
:10C64000824203D1106852684118216062605C60C8
:10C65000CAE7C046301C0020032370B5CD1C9D43A3
:10C66000083506000C2D1ED20C25A9421DD830001D
:10C6700000F0E8FA254A14682100002919D1244C59
:10C680002368002B03D1300000F0CAF92060290094
:10C69000300000F0C5F9431C2BD10C23300033606F
:10C6A00000F0D1FA03E0002DDFDA0C233360002024
:10C6B00070BD0B685B1B19D40B2B03D90B60CC1816
:10C6C000256003E04B688C420DD11360300000F010
:10C6D000BAFA200007220B30231D9043C31AE7D07B
:10C6E0005A42E250E4E763600C00EFE70C0049684F
:10C6F000C3E70323C41C9C43A042E1D0211A3000AD
:10C7000000F08EF9431CDBD1C7E7C046301C002087
:10C71000341C0020F8B507000D001600002905D1D3
:10C720001100FFF799FF04002000F8BD002A03D193
:10C73000FFF748FF3400F7E700F086FA2C00B0421C
:10C74000F2D231003800FFF787FF041EECD0290039
:10C750003200FEF7BFFF29003800FFF733FFE3E7A1
:10C76000F0B58E6885B007000C00039201939E42DD
:10C770003CD890238A89DB001A4234D0032509690A
:10C7800023685B1A0293636902985D43EB0F5D199E
:10C79000019B6D1001331B18AB4200D91D005305DE
:10C7A00032D529003800FFF757FF061E09D10C23A8
:10C7B0003B6040230120A28940421343A38105B07E
:10C7C000F0BD029A2169FEF785FFA389144A1A4039
:10C7D00080231343A381029B2661F61826606561BE
:10C7E000019EED1AA560019B9E4200D9019E320078
:10C7F00003992068FEF777FFA36800209B1BA360C6
:10C8000023689E192660DAE72A003800FFF782FFC6
:10C81000061EE0D121693800FFF7D4FEC7E7C04605
:10C820007FFBFFFFF0B59FB0029005938B890F004F
:10C8300016001B0611D50B69002B0ED14021FFF706
:10C840000BFF38603861002805D10C23029A0138AB
:10C8500013601FB0F0BD40237B61002306AC636111
:10C86000203363761033A37635002B78002B01D06C
:10C87000252B46D1AB1B04930CD032003900029813
:10C88000FFF76EFF431C00D1AEE06269049B944643
:10C89000634463612B78002B00D1A5E001220023C3
:10C8A0005242626002A9543252186E1C2360E36047
:10C8B000A3601370A365317805225448FFF776FE14
:10C8C000751C00281FD12268D30604D5532302A962
:10C8D0005B1820211970130704D5532302A95B1894
:10C8E0002B21197033782A2B16D0350000210A200D
:10C8F000E3682A786E1C303A092A4ED9002918D0EC
:10C9000010E00135B1E7414B2268C01A0123834092
:10C91000134323602E00CEE7059B191D1B6805916C
:10C92000002B01DB099304E05B42E3600223134325
:10C9300023602B782E2B0AD16B782A2B35D1059BBF
:10C9400002351A1D1B680592002B2BDB0793304E16
:10C95000297803223000FFF729FE002806D0402363
:10C96000801B834022680135134323602978062207
:10C9700028486E1C2176FFF719FE00283CD0264B74
:10C98000002B25D10722059B0733934308330593DA
:10C990006369039A9B18636166E7434301219B180F
:10C9A0003500A6E701235B42D0E700230A201A00E6
:10C9B0000135636029786E1C3039092903D9002BB1
:10C9C000C5D00792C3E74243012352183500F1E76F
:10C9D00005AB00933A00114B2100029800E000BF24
:10C9E0000390039B0133D3D1BB890B985B0600D422
:10C9F0002FE7012040422CE705AB00933A00074B9C
:10CA000021000298FFF736F8EAE7C04670E400001C
:10CA100076E400007AE400000000000061C7000036
:10CA2000002370B5064C05000800236000F060F993
:10CA3000431C03D12368002B00D02B6070BDC0467F
:10CA4000C42F002070B504000D001F2904D916233F
:10CA500003600120404270BD436C002B04D08A006B
:10CA60009B181A68002A08D1200000F031F82A002B
:10CA70000100200000F01AF8EDE70020012AEAD0BA
:10CA8000511C03D1162301302360E4E70024280061
:10CA90001C6090472000DEE710B5034B01001868CA
:10CAA000FFF7D0FF10BDC04684000020002370B502
:10CAB000064C050008001100236000F001F9431C3A
:10CAC00003D12368002B00D02B6070BDC42F002041
:10CAD00010B500F0E5F810BD70B50C000E25495FEB
:10CAE00000F0BAF8002803DB636D1B18636570BDA6
:10CAF000A389024A1340A381F9E7C046FFEFFFFF75
:10CB0000F8B51F008B8905000C001600DB0505D564
:10CB10000E23C95E0022022300F080F8A389054A93
:10CB200028001340A38132000E23E15E3B0000F099
:10CB30002BF8F8BDFFEFFFFF70B50C000E25495F25
:10CB400000F06CF8A389421C03D1054A1340A3816D
:10CB500070BD802252011343A3816065F8E7C0468F
:10CB6000FFEFFFFF10B50E23C95E00F021F810BDE6
:10CB70000B1E04D0FF2A04D98A2303608B3B1800C4
:10CB800070470A700123FAE770B50500080011002C
:10CB90000022064C22601A0000F0B8F8431C03D1B2
:10CBA0002368002B00D02B6070BDC046C42F00202E
:10CBB000002370B5064C05000800236000F060F803
:10CBC000431C03D12368002B00D02B6070BDC046EE
:10CBD000C42F0020002370B5064C0500080011008A
:10CBE000236000F055F8431C03D12368002B00D0CC
:10CBF0002B6070BDC42F0020002370B5064C0500CB
:10CC00000800236000F054F8431C03D12368002B74
:10CC100000D02B6070BDC046C42F002070B5050049
:10CC2000080011000022064C22601A0000F050F8A3
:10CC3000431C03D12368002B00D02B6070BDC0467D
:10CC4000C42F0020704770470B1F1B68181F002B54
:10CC500001DA0B58C018704770B5050008001100C4
:10CC60000022064C22601A0000F03AF8431C03D15F
:10CC70002368002B00D02B6070BDC046C42F00205D
:10CC800058220120014B40421A607047C42F0020F7
:10CC900058220120014B40421A607047C42F0020E7
:10CCA00058220120014B40421A607047C42F0020D7
:10CCB0005822024B00201A607047C046C42F002043
:10CCC00058220120014B40421A607047C42F0020B7
:10CCD00058220120014B40421A607047C42F0020A7
:10CCE00058220120014B40421A607047C42F002097
:10CCF000044A1368002B00D1034B18181060180069
:10CD00007047C046381C0020C82F00205822012040
:10CD1000014B40421A607047C42F0020FEE7C04616
:10CD2000F8B5C046F8BC08BC9E467047F8B5C0468A
:10CD3000F8BC08BC9E467047646174610000000046
:10CD4000BCCD0000EF010000C5CD0000E3020000F3
:10CD5000CDCD000019090000D4CD0000290A000043
:10CD6000D9CD000041050000E4CD000053030000D0
:10CD7000E9CD0000810C0000F5CD00001F0200008D
:10CD8000FFCD0000210800000DCE0000CD06000000
:10CD90001ACE00000305000072616E646F6D0061C1
:10CDA0006C6C006C6173740066616C736500747206
:10CDB000756500252E3135732E2E2E006D616B6545
:10CDC0004C697374006164644C6173740064656CD5
:10CDD000657465006A6F696E00636F707946726F83
:10CDE0006D546F0066696E64006A6F696E53747289
:10CDF000696E677300756E69636F64654174007571
:10CE00006E69636F6465537472696E67006E6577EF
:10CE100042797465417272617900667265654D652B
:10CE20006D6F7279000000008DCE00002D110000A2
:10CE300092CE00004B110000CDCD00004F1100003C
:10CE400098CE000031110000A2CE00005311000066
:10CE5000ABCE000057110000B5CE00005B11000002
:10CE6000C0CE00005F110000CCCE000035110000E4
:10CE7000D5CE000043110000DFCE000039110000C4
:10CE8000EACE00004711000066696C65006F7065AE
:10CE90006E00636C6F736500656E644F6646696C07
:10CEA0006500726561644C696E650072656164421B
:10CEB0007974657300617070656E644C696E6500AD
:10CEC000617070656E6442797465730066696C6543
:10CED00053697A650073746172744C697374006E7F
:10CEE000657874496E4C6973740073797374656DF9
:10CEF000496E666F0000000090130000A013000050
:10CF0000BA1300003814000070140000A6140000CA
:10CF1000DE1400000415000040150000821500001A
:10CF2000D81500001C16000088160000D01600005E
:10CF3000F61600002E170000741700009A17000064
:10CF4000C8170000F617000038180000BC180000D1
:10CF50008E190000181A00006E1A0000BA1A00009C
:10CF6000DA1A0000FC1A0000AE1B0000F41B0000DF
:10CF70006C1C00009A1C0000CA1C0000001D000070
:10CF8000841D0000EC1D0000321E00007A1E00000F
:10CF9000F01E0000661F0000AE1F0000F41F00001E
:10CFA0002A20000070200000B620000008210000A8
:10CFB0005C210000B0210000EE210000582200009A
:10CFC0008E220000D62200001E23000066230000EF
:10CFD000A0230000E8230000302400009C2500006E
:10CFE000C81700002E1700009824000090130000BE
:10CFF000D8240000042500003A2500006625000022
:10D000009013000090130000901300009013000094
:10D0100016260000582600009E260000EE2600007E
:10D020001A2700006A27000090270000BE27000092
:10D030009013000090130000E22700001228000067
:10D0400042280000AC280000D62800000C2900006F
:10D05000362900005E29000086290000B62900005C
:10D06000E6290000102A00003A2A00006A2A00007F
:10D07000942A000090130000901300009013000009
:10D080009013000090130000C42A0000F02A000052
:10D090001C2B0000482B0000742B0000AA2B000062
:10D0A000E02B0000162C00004C2C0000782C000017
:10D0B000AC2C0000E22C0000901300009013000044
:10D0C00090130000901300009013000090130000D4
:10D0D00090130000901300009013000090130000C4
:10D0E00090130000901300009013000090130000B4
:10D0F0000E2D0000442D00005B2564206974656DD1
:10D10000206C6973745D00282564206279746573EE
:10D110002900286F626A65637420747970653A200B
:10D1200025642900537461636B20756E64657266B3
:10D130006C6F7700626F6F6C65616E006E756D620B
:10D14000657200737472696E67006C697374006253
:10D150007974652061727261790000000700000037
:10D1600003000000B6D10000652E0000BED1000013
:10D17000152F0000C7D10000BF2F0000D0D1000044
:10D18000692E0000D9D10000C32F0000E1D10000BA
:10D19000AD2F0000000000000100000002000000B0
:10D1A00003000000040000000A0000006D696372C3
:10D1B0006F3A62697400686173546F6E6500706CD9
:10D1C0006179546F6E6500686173536572766F00A4
:10D1D000736574536572766F00646163496E697438
:10D1E00000646163577269746500474320746F6F10
:10D1F0006B2025642075736563733B2066726565DB
:10D2000020256420776F726473003C496E746567F3
:10D2100065723E003C4C6973743E003C4F626A6527
:10D2200063743E003C4279746541727261793E00DC
:10D230000D0A564D2050616E69633A2025730D0A20
:10D24000006D6973630000007DD200008D3C00001A
:10D2500086D200001D3C00008AD20000713B000015
:10D2600092D20000173B00009CD20000AD3A0000B3
:10D27000A8D20000AF3900006E756C6C006865784C
:10D28000546F496E740073696E006A736F6E476500
:10D2900074006A736F6E436F756E74006A736F6E9D
:10D2A00056616C75654174006A736F6E4B657941A8
:10D2B0007400000010D30000F93C000018D30000F7
:10D2C000FD3C000022D300001B3D00002BD30000DA
:10D2D000253D000036D300002F3D000042D3000062
:10D2E000393D000057D30000433D00006CD30000DF
:10D2F0004D3D000078D30000573D000088D300006A
:10D30000073D000094D30000113D00006E657400DD
:10D31000686173576946690073746172745769462E
:10D32000690073746F70576946690077696669535D
:10D330007461747573006D794950416464726573EA
:10D3400073006874747053657276657247657452C1
:10D3500065717565737400726573706F6E64546F78
:10D360004874747052657175657374006874747074
:10D37000436F6E6E65637400687474704973436FB5
:10D380006E6E65637465640068747470526571755F
:10D390006573740068747470526573706F6E736532
:10D3A000001A1B1C03040607090A171819000000BD
:10D3B000000008080800080A4A4000000A5FEA5F07
:10D3C000EA0ED92ED36E19324489330C924C924D09
:10D3D0000808000000048808080408048484880001
:10D3E0000A448A4000048EC48000000004880000C3
:10D3F0000EC000000000080001224488100C925268
:10D40000524C048C84848E1C824C901E1EC244920A
:10D410004C06CA525FE21FF01EC13E02448ED12E5E
:10D420001FE24488100ED12ED12E0ED12EC48800BA
:10D430000800080000048004880244880482000E6A
:10D44000C00EC008048244880ED126C0040ED13517
:10D45000B36C0C925ED2521C925C925C0ED0101097
:10D460000E1C9252525C1ED01C901E1ED01C90109E
:10D470000ED013712E12525ED2521C8808081C1F47
:10D48000E242524C1254981492101010101E113B8C
:10D4900075B131113935B3710C9252524C1C925CFA
:10D4A00090100C92524C861C925C92510ED00C82C1
:10D4B0005C1FE4848484125252524C1131312A444C
:10D4C000113135BB7112524C9252112A4484841E80
:10D4D000C488101E0EC808080E10080482410EC22F
:10D4E00042424E048A400000000000001F080480F1
:10D4F0000000000ED2524F10101C925C000ED01093
:10D500000E02424ED24E0C925C900E06C81C880849
:10D510000ED24EC24C10101C92520800080808028D
:10D520004002424C10149814920808080806001B88
:10D5300075B131001C925252000C92524C001C9258
:10D540005C90000ED24EC2000ED010100006C8042F
:10D550009808080EC807001252524F0011312A4491
:10D5600000113135BB00124C8C9200112A449800F6
:10D570001EC4881E06C48C8486080808080818087B
:10D580000C881800000C83600000000001000000FF
:10D59000020000000300000004000000050000007D
:10D5A000060000000700000008000000090000005D
:10D5B0000A0000000B0000000C0000000D0000003D
:10D5C0000E0000000F00000010000000120000001C
:10D5D0001400000016000000180000001A000000EF
:10D5E0001C0000001E0000002000000023000000BE
:10D5F00026000000290000002C0000002F00000081
:10D6000032000000360000003A0000003E0000003A
:10D6100042000000460000004B00000050000000E7
:10D62000550000005A000000610000006800000082
:10D630006F000000760000007D0000008400000004
:10D640008B0000009200000099000000A000000084
:10D65000A7000000AE000000B5000000BC00000004
:10D66000C3000000CA000000D1000000D800000084
:10D67000DF000000E6000000ED000000F400000004
:10D68000FB000000FF000000D8D60000793D00003C
:10D69000E3D6000015430000EDD600003D3F00003A
:10D6A000FAD600008541000001D70000D5410000F6
:10D6B0000AD700002542000016D700001D410000D7
:10D6C00027D70000AD3F000034D70000AD40000078
:10D6D000646973706C6179006C696768744C657615
:10D6E000656C006D62446973706C6179006D6244B1
:10D6F0006973706C61794F6666006D62506C6F740F
:10D70000006D62556E706C6F74006D62447261776B
:10D710005368617065006D625368617065466F7231
:10D720004C6574746572006E656F506978656C53F2
:10D73000656E64006E656F506978656C53657450F2
:10D74000696E004E6F7420656E6F75676820726F2A
:10D750006F6D206576656E20616674657220636FFB
:10D760006D70616374696F6E00436F6D7061637497
:10D77000656420466C61736820636F646520737410
:10D780006F72650A2564206279746573207573650C
:10D790006420282564252529206F66202564004201
:10D7A0006164207265636F726420666F756E6420B9
:10D7B000647572696E6720696E697469616C697AF3
:10D7C0006174696F6E00256420256420256420281B
:10D7D000256420776F726473290025642072656365
:10D7E0006F7264732C20256420776F7264732C2011
:10D7F0006D617849442025642C20636F6D706163EE
:10D8000074696F6E206379636C65732025640052C0
:10D810006573746F72656420256420736372697028
:10D820007473005374617274656400726164696F2B
:10D8300000000000C4D80000E54C0000D1D8000072
:10D84000814F0000E1D80000014F0000EFD8000038
:10D8500015510000FAD800000D4D00000AD9000053
:10D86000954D00001ED900007D4D00002DD900000F
:10D87000F752000039D900007552000042D900006B
:10D88000195200004DD900006151000058D9000024
:10D890009D51000061D90000D15100006AD90000FB
:10D8A0001D4D000079D90000FD4C000082D9000018
:10D8B0002D4D00006E6F6E65006F746865720070AC
:10D8C0006169720064697361626C65526164696F59
:10D8D000006D65737361676552656365697665643C
:10D8E000007061636B65745265636569766500708D
:10D8F00061636B657453656E640072656365697618
:10D900006564496E74656765720072656365697602
:10D9100065644D6573736167655479706500726500
:10D92000636569766564537472696E670073656ECA
:10D9300064496E74656765720073656E64506169F1
:10D94000720073656E64537472696E6700736574F8
:10D950004368616E6E656C0073657447726F7570B5
:10D9600000736574506F776572007369676E616CE0
:10D97000537472656E67746800646576696365499F
:10D9800044006C6173744D6573736167654944004D
:10D99000556E6B6E6F776E207072696D6974697603
:10D9A00065205B25733A25735D00000000000000D0
:10D9B000963007772C610EEEBA51099919C46D079C
:10D9C0008FF46A7035A563E9A395649E3288DB0EF7
:10D9D000A4B8DC791EE9D5E088D9D2972B4CB609DA
:10D9E000BD7CB17E072DB8E7911DBF906410B71DB7
:10D9F000F220B06A4871B9F3DE41BE847DD4DA1AF0
:10DA0000EBE4DD6D51B5D4F4C785D38356986C1320
:10DA1000C0A86B647AF962FDECC9658A4F5C011499
:10DA2000D96C0663633D0FFAF50D088DC8206E3B77
:10DA30005E10694CE44160D5727167A2D1E4033C89
:10DA400047D4044BFD850DD26BB50AA5FAA8B535B0
:10DA50006C98B242D6C9BBDB40F9BCACE36CD8329F
:10DA6000755CDF45CF0DD6DC593DD1ABAC30D92646
:10DA70003A00DE518051D7C81661D0BFB5F4B42149
:10DA800023C4B3569995BACF0FA5BDB89EB8022846
:10DA90000888055FB2D90CC624E90BB1877C6F2FCB
:10DAA000114C6858AB1D61C13D2D66B69041DC76C6
:10DAB0000671DB01BC20D2982A10D5EF8985B1719F
:10DAC0001FB5B606A5E4BF9F33D4B8E8A2C907784E
:10DAD00034F9000F8EA8099618980EE1BB0D6A7FE5
:10DAE0002D3D6D08976C6491015C63E6F4516B6B9E
:10DAF00062616C1CD83065854E0062F2ED95066C53
:10DB00007BA5011BC1F4088257C40FF5C6D9B065C7
:10DB100050E9B712EAB8BE8B7C88B9FCDF1DDD6224
:10DB2000492DDA15F37CD38C654CD4FB5861B24D8A
:10DB3000CE51B53A7400BCA3E230BBD441A5DF4A54
:10DB4000D795D83D6DC4D1A4FBF4D6D36AE9694317
:10DB5000FCD96E34468867ADD0B860DA732D0444C2
:10DB6000E51D03335F4C0AAAC97C0DDD3C710550ED
:10DB7000AA41022710100BBE86200CC925B5685794
:10DB8000B3856F2009D466B99FE461CE0EF9DE5EDD
:10DB900098C9D9292298D0B0B4A8D7C7173DB3598E
:10DBA000810DB42E3B5CBDB7AD6CBAC02083B8ED1F
:10DBB000B6B3BF9A0CE2B6039AD2B1743947D5EA2C
:10DBC000AF77D29D1526DB048316DC73120B63E35B
:10DBD000843B64943E6A6D0DA85A6A7A0BCF0EE4BA
:10DBE0009DFF099327AE000AB19E077D44930FF075
:10DBF000D2A3088768F2011EFEC206695D5762F76C
:10DC0000CB67658071366C19E7066B6E761BD4FEA8
:10DC1000E02BD3895A7ADA10CC4ADD676FDFB9F985
:10DC2000F9EFBE8E43BEB717D58EB060E8A3D6D647
:10DC30007E93D1A1C4C2D83852F2DF4FF167BBD175
:10DC40006757BCA6DD06B53F4B36B248DA2B0DD878
:10DC50004C1B0AAFF64A0336607A0441C3EF60DF1B
:10DC600055DF67A8EF8E6E3179BE69468CB361CB04
:10DC70001A8366BCA0D26F2536E2685295770CCC29
:10DC800003470BBBB91602222F260555BE3BBAC56A
:10DC9000280BBDB2925AB42B046AB35CA7FFD7C25B
:10DCA00031CFD0B58B9ED92C1DAEDE5BB0C2649B4C
:10DCB00026F263EC9CA36A750A936D02A906099C7F
:10DCC0003F360EEB8567077213570005824ABF95F2
:10DCD000147AB8E2AE2BB17B381BB60C9B8ED29275
:10DCE0000DBED5E5B7EFDC7C21DFDB0BD4D2D386CC
:10DCF00042E2D4F1F8B3DD686E83DA1FCD16BE813F
:10DD00005B26B9F6E177B06F7747B718E65A08880F
:10DD1000706A0FFFCA3B06665C0B0111FF9E658FA0
:10DD200069AE62F8D3FF6B6145CF6C1678E20AA04A
:10DD3000EED20DD75483044EC2B30339612667A7D0
:10DD4000F71660D04D476949DB776E3E4A6AD1AE1F
:10DD5000DC5AD6D9660BDF40F03BD83753AEBCA9AE
:10DD6000C59EBBDE7FCFB247E9FFB5301CF2BDBD1B
:10DD70008AC2BACA3093B353A6A3B4240536D0BA24
:10DD80009306D7CD2957DE54BF67D9232E7A66B3C1
:10DD9000B84A61C4021B685D942B6F2A37BE0BB46E
:10DDA000A18E0CC31BDF055A8DEF022D416C6C2038
:10DDB0007461736B732073746F7070656400763177
:10DDC000303700202573202573004D656D6F727903
:10DDD00020636C6561726564004E6F2066726565D4
:10DDE000207461736B20656E747269657300000046
:10DDF00048DE0000D166000055DE000071620000C0
:10DE000061DE0000A166000067DE0000B166000070
:10DE10006DDE0000C166000073DE0000A562000038
:10DE20007DDE00002D67000085DE000081640000BB
:10DE30008EDE00000163000096DE000099630000A2
:10DE400073656E736F727300616363656C65726195
:10DE500074696F6E0074656D70657261747572655A
:10DE60000074696C74580074696C74590074696C3E
:10DE7000745A00746F756368526561640069326337
:10DE80005265616400693263577269746500726536
:10DE90006164444854006D6963726F70686F6E65A9
:10DEA0000000000018DF0000B967000026DF000056
:10DEB000BD6700002FDF0000C967000039DF0000E8
:10DEC000CD67000042DF0000D167000047DF00009F
:10DED000D56700004CDF0000D967000058DF000064
:10DEE000DD6700005FDF0000E167000068DF000021
:10DEF000E56700006DDF0000E967000078DF0000E3
:10DF0000ED67000082DF0000C16700008CDF0000C9
:10DF1000C567000074667400656E61626C65446973
:10DF200073706C6179006765745769647468006721
:10DF300065744865696768740073657450697865CD
:10DF40006C006C696E65007265637400726F756E4B
:10DF50006465645265637400636972636C65007420
:10DF60007269616E676C65007465787400746674BC
:10DF7000546F756368656400746674546F75636884
:10DF80005800746674546F756368590074667454ED
:10DF90006F75636850726573737572650076617230
:10DFA00073000000C4DF00007D6C0000CEDF0000C5
:10DFB0005D6C0000D7DF0000396C0000E3DF00007B
:10DFC000C56B000076617245786973747300766181
:10DFD000724E616D6564007365745661724E616D59
:10DFE0006564007661724E616D65466F72496E645C
:10DFF00065780057656C636F6D6520746F204D699F
:10E0000063726F426C6F636B732100705F73706932
:10E0100020213D204E554C4C002F686F6D652F67B9
:10E0200069742F2E706C6174666F726D696F2F70DA
:10E0300061636B616765732F6672616D65776F727F
:10E040006B2D61726475696E6F6E6F726469636E59
:10E050007266352F6C69627261726965732F5350F5
:10E06000492F5350492E63707000535049436C61DF
:10E0700073733A3A535049436C617373284E524656
:10E080005F5350495F547970652A2C2075696E740E
:10E09000385F742C2075696E74385F742C20756934
:10E0A0006E74385F7429000000000000000000005A
:10E0B000896E0000456E00006B6E0000756E0000FA
:10E0C0007F6E0000696E0000030000000200000087
:10E0D0000100000004000000050000001100000025
:10E0E0000C0000000B000000120000000A000000FD
:10E0F000060000001A0000001400000017000000D5
:10E10000160000001500000010000000FFFFFFFFD8
:10E11000FFFFFFFF000000001E00000019000000CC
:10E1200018000000070000000800000009000000BF
:10E130000D0000000E0000000F0000001C00000099
:10E140001B0000001D000000130000000000000084
:10E150000000000061730000C97B0000E173000053
:10E16000F5730000EB7300005D7300005173000055
:10E17000017400007D7300004D730000000000007A
:10E18000000000000000304300000000000030C329
:10E190007371727400000000FB21F93FFB210940FC
:10E1A0007CD91240FB2119407A6A1F407CD9224059
:10E1B000BBFD2540FB2129403A462C407A6A2F407E
:10E1C0005C4731407CD932409C6B3440BBFD3540CC
:10E1D000DB8F3740FB2139401BB43A403A463C4084
:10E1E0005AD83D407A6A3F404C7E40405C474140AF
:10E1F0006C1042407CD942408CA243409C6B44400E
:10E20000AC344540BBFD4540CBC64640DB8F474064
:10E21000EB584840FB21494083F9A200444E6E0070
:10E22000FC291500D1572700DD34F50062DBC00062
:10E230003C999500419043006351FE00BBDEAB006A
:10E24000B761C5003A6E2400D24D42004906E00095
:10E2500009EA2E001C92D100EB1DFE0029B11C0022
:10E26000E83EA700F535820044BB2E009CE98400FF
:10E27000B4267000417E5F00D69139005383390087
:10E280009CF439008B5F840028F9BD00F81F3B0027
:10E29000DEFF97000F980500112FEF000A5A8B0040
:10E2A0006D1F6D00CF7E360009CB2700464FB700AB
:10E2B0009E663F002DEA5F00BA277500E5EBC700B8
:10E2C0003D7BF100F739070092528A00FB6BEA00B0
:10E2D0001FB15F00085D8D00300356007BFC4600D7
:10E2E000F0AB6B0020BCCF0036F49A00E3A91D0010
:10E2F0005E619100081BE60085996500A0145F002F
:10E300008D40680080D8FF0027734D00060631005D
:10E31000CA561500C9A873007BE260006B8CC00070
:10E3200000000040FB21F93F000000002D44743E36
:10E33000000000809846F83C0000006051CC783B1B
:10E3400000000080831BF0390000004020257A384F
:10E35000000000802282E336000000001DF36935D2
:10E36000020000000300000004000000060000009E
:10E3700040980000EA970000EA9700001899000012
:10E38000E6970000E69700000E990000189900003B
:10E39000E69700000E990000E6970000189900002B
:10E3A0001C9900001C9900001C9900002499000091
:10E3B0001CA300008EA10000D2A1000036A1000025
:10E3C000D2A10000C2A20000D2A1000036A100002C
:10E3D0008EA100008EA10000C2A2000036A10000A4
:10E3E0002EA100002EA100002EA10000D0A200004E
:10E3F00044AA000046A9000046A9000064AC000041
:10E4000040A9000040A900004CAC000064AC000032
:10E4100040A900004CAC000040A9000064AC000022
:10E420005AAC00005AAC00005AAC000068AC0000C6
:10E430002C2066756E6374696F6E3A200061737389
:10E44000657274696F6E2022257322206661696C83
:10E4500065643A2066696C6520222573222C206C45
:10E46000696E65202564257325730A0088000020E5
:10E47000232D302B2000686C4C00656667454647AD
:10E480000030313233343536373839414243444530
:10E49000460030313233343536373839616263649F
:10E4A00065660000000000000000000000000000A1
:10E4B000000000000000000000000000000000005C
:10E4C000000000000000000000000000000000004C
:10E4D000000000000000000000000000000000003C
:10E4E000000000000000000000000000000000002C
:10E4F000000000000000000000000000000000001C
:10E50000000000004300504F5349580000202020D5
:10E5100020202020202028282828282020202020D3
:10E5200020202020202020202020202020881010A3
:10E5300010101010101010101010101010040404FF
:10E5400004040404040404101010101010104141BD
:10E5500041414141010101010101010101010101AB
:10E5600001010101010101011010101010104242BF
:10E57000424242420202020202020202020202027B
:10E58000020202020202020210101010200000001B
:10E59000000000000000000000000000000000007B
:10E5A000000000000000000000000000000000006B
:10E5B000000000000000000000000000000000005B
:10E5C000000000000000000000000000000000004B
:10E5D000000000000000000000000000000000003B
:10E5E000000000000000000000000000000000002B
:10E5F000000000000000000000000000000000001B
:10E60000000000000000000000000000000000000A
:04E610000000000006
:08E61400F41AFF7F0100000071
:10E61C00FFFFFFFFD007000001000000E803DC054E
:10E62C00DC05DC05DC050000FFFFFFFFFFFFFFFF43
:10E63C001800000019FCFFFFFFFFFFFFFF000000A8
:10E64C000024F4000200000003000000FFFFFFFFA5
:10E65C0000000000010000000000020001000000AA
:10E66C00FFFFFFFF0000000002000000000004009C
:10E67C0002000000FFFFFFFF00000000030000008D
:10E68C0000000800030000000A0000000800000061
:10E69C00010000008800002000000000C4E400001D
:10E6AC00E4E40000A4E4000000000000000000000E
:10E6BC00000000000000000000000000000000004E
:10E6CC00000000000000000000000000000000003E
:10E6DC00000000000000000000000000000000002E
:10E6EC00000000000000000000000000000000001E
:10E6FC0000000000000000004300000000000000CB
:10E70C0000000000000000000000000000000000FD
:10E71C0000000000000000004300000000000000AA
:10E72C0000000000000000000000000000000000DD
:10E73C00000000000000000043000000000000008A
:10E74C0000000000000000000000000000000000BD
:10E75C00000000000000000043000000000000006A
:10E76C00000000000000000000000000000000009D
:10E77C00000000000000000043000000000000004A
:10E78C00000000000000000000000000000000007D
:10E79C00000000000000000043000000000000002A
:10E7AC00000000000000000000000000000000005D
:10E7BC00000000000000000043000000000000000A
:10E7CC00000000000000000000000000000000003D
:10E7DC00000000000000000071CB000089C50000A3
:10E7EC00000000000CE50000BACD000040D2000093
:10E7FC0040D2000040D2000040D2000040D20000C5
:10E80C0040D2000040D2000040D2000040D20000B4
:10E81C00FFFFFFFFFFFFFFFFFFFFFFFFFFFF0000FA
:10E82C000100415343494900000000000000000072
:10E83C0000000000000000000000000000000000CC
:10E84C000000415343494900000000000000000053
:10E85C0000000000000000000000000000000000AC
:10E86C0000000000E9000000156E0000857100003A
:08E87C00AD760000C1000000B0
:040000030000722166
:00000001FF
